:020000040800F2
:1000000000060020E1010008B10E0008310E0008D2
:10001000890E0008310E00085D0E0008E30100089B
:10002000E3010008E3010008E3010008852100085E
:10003000E3010008E3010008E3010008E301000810
:10004000E3010008E3010008E3010008E301000800
:10005000E3010008E30100084D320008793200088E
:10006000A5320008D1320008FD320008E301000883
:10007000E3010008E3010008E3010008E3010008D0
:10008000E3010008E3010008E3010008E3010008C0
:10009000E3010008E3010008E30100082933000838
:1000A000E3010008E3010008E3010008E3010008A0
:1000B000C1300008E3010008E3010008E301000883
:1000C000E3010008E3010008E3010008E301000880
:1000D000E3010008E3010008E3010008E301000870
:1000E00091330008E3010008E3010008E301000880
:1000F000E3010008E3010008E3010008E301000850
:10010000E3010008E3010008E3010008E30100083F
:10011000E3010008E3010008E3010008E30100082F
:10012000E3010008E3010008E3010008E30100081F
:10013000E3010008E3010008E3010008E30100080F
:10014000E3010008E3010008E3010008BD280008FE
:10015000E3010008E3010008E3010008E3010008EF
:10016000E3010008E3010008E3010008E3010008DF
:10017000E3010008E3010008E3010008E3010008CF
:10018000E3010008E3010008E3010008E3010008BF
:10019000E3010008E3010008E3010008E3010008AF
:1001A000E3010008E3010008E3010008E30100089F
:1001B000E3010008E3010008E3010008E30100088F
:1001C000E3010008E3010008E3010008E30100087F
:1001D000E3010008E3010008E3010008E30100086F
:1001E00002E000F000F8FEE772B63A4880F30888B3
:1001F000394880F3098839484EF60851CEF200019B
:10020000086040F20000CCF200004EF63471CEF2ED
:1002100000010860BFF34F8FBFF36F8F40F2000003
:10022000C0F2F0004EF68851CEF200010860BFF334
:100230004F8FBFF36F8F4FF00000E1EE100A4EF6C4
:100240003C71CEF200010860062080F31488BFF3F1
:100250006F8F02F017F801F0F3FF02F095FE4FF0F8
:1002600055301F491B4A91423CBF41F8040BFAE745
:100270001C49194A91423CBF41F8040BFAE71A495C
:100280001A4A1B4B9A423EBF51F8040B42F8040B2A
:10029000F8E700201749184A91423CBF41F8040B87
:1002A000FAE701F0D1FF02F0C3FE144C144DAC424A
:1002B00003DA54F8041B8847F9E700F041F8114CC1
:1002C000114DAC4203DA54F8041B8847F9E701F0FA
:1002D000B9BF000000060020002200200000000836
:1002E0000000002000060020B8370008002200208F
:1002F0004022002040220020A82D0020E00100081C
:10030000E0010008E0010008E00100082DE9F04FDD
:100310002DED108AC1F80CD0C3689D46BDEC108A43
:10032000BDE8F08F002383F311882846A047002002
:1003300001F034FBFEE701F0AFFA00DFFEE700005A
:1003400038B501F0EFFE054601F012FF0446D8B9BA
:100350000F4B9D421AD001339D4218BF044641F213
:10036000883504BF01240025002001F0E5FE0CB112
:1003700000F076F800F032FD00F0A4FB284600F013
:10038000C3F800F06DF8F9E70025EDE70546EBE767
:10039000010007B008B500F067FBA0F12003584248
:1003A000584108BD07B541F21203022101A8ADF87A
:1003B000043000F077FB03B05DF804FB38B5202370
:1003C00083F311881748C3680BB101F06DFB164A1F
:1003D000144800234FF47A7101F02AFB002383F3C1
:1003E0001188124C236813B12368013B23606368B2
:1003F00013B16368013B63600D4D2B7833B96368BB
:100400007BB9022000F05AFC322363602B78032B67
:1004100007D163682BB9022000F050FC4FF47A73C7
:10042000636038BD40220020BD0300085C2300202B
:1004300054220020084B187003280CD8DFE800F085
:1004400008050208022000F027BC022000F012BCC0
:10045000024B00225A607047542200205C23002087
:10046000244B254A10B51C461968013140D004338D
:100470009342F9D16268214B9A4239D9204B9B684B
:1004800003F1006303F580339A4231D2002000F07B
:1004900033FB0220FFF7CEFF1A4B1A6C00221A64BE
:1004A000196E1A66196E596C5A64596E5A665A6EEC
:1004B0005A6942F080025A615A6922F080025A61F8
:1004C0005A691A6942F000521A611A6922F0005200
:1004D0001A611B6972B64FF0E0232021C3F8084D62
:1004E000D4E9003281F311889D4683F308881047D0
:1004F00010BD00BF0000010820000108FFFF000838
:1005000000220020003802402DE9F04F93B0AA4BA2
:1005100000902022FF210AA89D6800F009FCA74A4C
:100520001378A3B9A6480121C3601170202383F377
:100530001188C3680BB101F0B7FAA24AA0480023A2
:100540004FF47A7101F074FA002383F31188009B51
:1005500013B19D4B009A1A609C4A009C1378032BA0
:100560001EBF00231370984A4FF0000A18BF536053
:10057000D3465646D146012000F08EFB24B1924B63
:100580001B68002B00F01182002000F06DFA039030
:10059000039B002BF2DB012000F06CFB039B213B53
:1005A000162BE8D801A252F823F000BF0906000874
:1005B00031060008C5060008770500087705000821
:1005C000770500084F0700081F09000839080008D0
:1005D0009B080008C3080008E90800087705000820
:1005E000FB080008770500086D090008A906000847
:1005F00077050008B109000815060008A9060008DB
:10060000770500089B0800080220FFF7C3FE0028BA
:1006100040F0F581009B0221BAF1000F08BF1C4693
:1006200005A841F21233ADF8143000F03BFAA2E70E
:100630004FF47A7000F018FA071EEBDB0220FFF788
:10064000A9FE0028E6D0013F052F00F2DA81DFE89D
:1006500007F0030A0D10133605230593042105A89E
:1006600000F020FA17E054480421F9E75848042123
:10067000F6E758480421F3E74FF01C08404600F025
:100680003DFA08F104080590042105A800F00AFAD3
:10069000B8F12C0FF2D1012000FA07F747EA0B0B53
:1006A0005FFA8BFB4FF0000900F08EFB26B10BF0D8
:1006B0000B030B2B08BF0024FFF774FE5BE74648D3
:1006C0000421CDE7002EA5D00BF00B030B2BA1D1FD
:1006D0000220FFF75FFE074600289BD0012000F0B4
:1006E0000BFA0220FFF7A6FE00265FFA86F84046C6
:1006F00000F012FA044690B10021404600F01CFAC6
:1007000001360028F1D1BA46044641F21213022103
:1007100005A8ADF814303E4600F0C4F92BE70120DF
:10072000FFF788FE2546244B9B68AB4207D9284635
:1007300000F0E4F9013040F067810435F3E7234B22
:1007400000251D70204BBA465D603E46ACE7002E8A
:100750003FF460AF0BF00B030B2B7FF45BAF022079
:10076000FFF768FE322000F07FF9B0F10008FFF6D5
:1007700051AF18F003077FF44DAF0F4A926808EBB2
:10078000050393423FF646AFB8F5807F3FF742AF8F
:10079000124B0193B84523DD4FF47A7000F064F9F1
:1007A0000390039A002AFFF635AF019B039A03F8E2
:1007B000012B0137EDE700BF002200205823002065
:1007C00040220020BD0300085C23002054220020AA
:1007D00004220020082200200C22002058220020A1
:1007E000C820FFF7D7FD074600283FF413AF1F2DA1
:1007F00011D8C5F1200242450AAB25F0030028BFFD
:10080000424683490192184400F06CFA019A8048EC
:10081000FF2100F08DFA4FEAA8037D490193C8F348
:100820008702284600F08CFA064600283FF46DAF98
:10083000019B05EB830537E70220FFF7ABFD00289E
:100840003FF4E8AE00F0A4F900283FF4E3AE00273F
:10085000B846704B9B68BB4218D91F2F11D80A9B12
:1008600001330ED027F0030312AA134453F8203C9F
:1008700005934046042205A900F01CFB043780467E
:10088000E7E7384600F03AF90590F2E7CDF8148032
:10089000042105A800F006F906E70023642104A856
:1008A000049300F0F5F800287FF4B4AE0220FFF7BF
:1008B00071FD00283FF4AEAE049800F051F90590A8
:1008C000E6E70023642104A8049300F0E1F800287F
:1008D0007FF4A0AE0220FFF75DFD00283FF49AAE42
:1008E000049800F04DF9EAE70220FFF753FD0028D5
:1008F0003FF490AE00F05CF9E1E70220FFF74AFD1B
:1009000000283FF487AE05A9142000F057F9042110
:100910000746049004A800F0C5F83946B9E732202C
:1009200000F0A2F8071EFFF675AEBB077FF472AEAB
:10093000384A926807EB090393423FF66BAE0220F8
:10094000FFF728FD00283FF465AE27F003074F446A
:10095000B9453FF4A9AE484600F0D0F8042105900F
:1009600005A800F09FF809F10409F1E74FF47A7047
:10097000FFF710FD00283FF44DAE00F009F9002804
:1009800044D00A9B01330BD008220AA9002000F0B2
:10099000D7F900283AD02022FF210AA800F0C8F990
:1009A000FFF700FD1C4800F0FFFF13B0BDE8F08F1B
:1009B000002E3FF42FAE0BF00B030B2B7FF42AAE6F
:1009C0000023642105A8059300F062F8074600287B
:1009D0007FF420AE0220FFF7DDFC804600283FF4C4
:1009E00019AEFFF7DFFC41F2883000F0DDFF05981B
:1009F00000F01CFA464600F0E7F93C46BBE5064627
:100A000052E64FF0000905E6BA467EE637467CE638
:100A10005822002000220020A086010070B50F4B54
:100A20001B780133DBB2012B0C4611D80C4D296821
:100A30004FF47A730E6AA2FB03320146224628461F
:100A4000B047844204D1074B00221A70012070BDC8
:100A50004FF4FA7000F0A8FF0020F8E71022002001
:100A6000502500209023002007B5002302460121D5
:100A70000DF107008DF80730FFF7D0FF20B19DF88A
:100A8000070003B05DF804FB4FF0FF30F9E700000A
:100A90000A4608B50421FFF7C1FF80F00100C0B28B
:100AA000404208BD30B4054C2368DD69044B0A465A
:100AB000AC460146204630BC604700BF50250020B0
:100AC000A086010070B501F01FFA094E094D308073
:100AD000002428683388834208D901F00FFA2B6874
:100AE00004440133B4F5803F2B60F2D370BD00BFE6
:100AF000922300206423002001F0C8BA00F10060B6
:100B000000F580300068704700F10060920000F549
:100B1000803001F047BA0000054B1A68054B1B886E
:100B20009B1A834202D9104401F0E8B900207047B3
:100B3000642300209223002038B5084D044629B1D3
:100B400028682044BDE8384001F0F8B928682044FE
:100B500001F0DCF90028F3D038BD00BF6423002089
:100B600010F003030AD1B0F5047F05D200F1005064
:100B7000A0F51040D0F80038184670470023FBE776
:100B800000F10050A0F51040D0F8100A70470000A6
:100B9000064991F8243033B10023086A81F82430E3
:100BA0000822FFF7B1BF0120704700BF6823002073
:100BB000014B1868704700BF002004E070B52A4B55
:100BC0001B68C3F30B0204461B0C62B140F21340D6
:100BD000824230D040F2194082422ED040F2214071
:100BE00082422CD10322214D0C2000FB0252556879
:100BF00042F20102934224D0B3F5805F23D041F248
:100C00000102934221D041F2030293421FD041F2EC
:100C10000702934214BF3F233123013C0C44013DA2
:100C20000A46A24215D215F9016F501C9EB100F878
:100C3000016C0246F5E70122D5E70222D3E70C4D0D
:100C4000D6E73323E9E74123E7E75A23E5E75923CA
:100C5000E3E7104605E02C258442157001D9901C6D
:100C60005370401A70BD00BF002004E0BC3400087F
:100C700090340008022804D1054B4FF000729A61AD
:100C800070470128FCD1034B4FF08042F7E700BFCB
:100C90000004024000000240022804D1054B4FF43A
:100CA00000729A6170470128FCD1034B4FF48042D7
:100CB000F7E700BF0004024000000240022805D10F
:100CC000064A536983F40073536170470128FCD1CD
:100CD000034A536983F48043F6E700BF00040240EF
:100CE0000000024010B50023934203D0CC5CC454F2
:100CF0000133F9E710BD000010B5013810F9013FCC
:100D00003BB191F900409C4203D11AB10131013A43
:100D1000F4E71AB191F90020981A10BD1046FCE7CB
:100D200003460246D01A12F9011B0029FAD1704776
:100D300002440346934202D003F8011BFAE77047CE
:100D40002DE9F8431F4D144695F8242007468846A0
:100D500052BBDFF870909CB395F824302BB9202259
:100D6000FF2148462F62FFF7E3FF95F82400C0F10A
:100D70000802A24228BF2246D6B24146920005EBA5
:100D80008000FFF7AFFF95F82430A41B1E44F6B295
:100D9000082E17449044E4B285F82460DBD1FFF7B5
:100DA000F7FE0028D7D108E02B6A03EB82038342C9
:100DB000CFD0FFF7EDFE0028CBD10020BDE8F883AF
:100DC0000120FBE768230020024B1A78024B1A70BF
:100DD000704700BF902300201022002010B50F4C58
:100DE0000F4800F0F7F821460D4800F01FF924687D
:100DF0000C48626DD2F8043843F00203C2F804389C
:100E000000F0D2FD0849204600F016FA626DD2F8D3
:100E1000043823F00203C2F8043810BDB0350008CE
:100E20005025002040420F00B835000870470000F0
:100E300000B59BB0EFF3098168226846FFF752FFC7
:100E4000EFF30583044B9A6BDA6A9A6A9A6A9A6A94
:100E50009A6A9A6A9B6AFEE700ED00E000B59BB0D3
:100E6000EFF3098168226846FFF73CFFEFF3058343
:100E7000044B9A6B9A6A9A6A9A6A9A6A9A6A9B6A05
:100E8000FEE700BF00ED00E000B59BB0EFF3098185
:100E900068226846FFF726FFEFF30583034B5A6B82
:100EA0009A6A9A6A9A6A9A6A9B6AFEE700ED00E07B
:100EB000FEE7000030B5094D0A4491420DD011F80B
:100EC000013B5840082340F30004013B2C4013F041
:100ED000FF0384EA5000F6D1EFE730BD2083B8ED80
:100EE000026843681143016003B11847704700006E
:100EF00013B5446BD4F894341A681178042915D1C9
:100F0000217C022912D11979128901238B401342C5
:100F10000CD101A904F14C0001F03CFFD4F8944439
:100F2000019B21790246206800F0CEF902B010BD85
:100F3000143001F0BFBE00004FF0FF33143001F059
:100F4000B9BE00004C3001F091BF00004FF0FF33FC
:100F50004C3001F08BBF0000143001F08DBE00005A
:100F60004FF0FF31143001F087BE00004C3001F02B
:100F70005DBF00004FF0FF324C3001F057BF000062
:100F80000020704710B5D0F894341A6811780429FD
:100F9000044617D1017C022914D1597952890123C1
:100FA0008B4013420ED1143001F020FE024648B1AE
:100FB000D4F894444FF4807361792068BDE8104000
:100FC00000F070B910BD0000406BFFF7DBBF000000
:100FD000704700007FB5124B036000234360C0E9F7
:100FE0000233012502260F4B05740446029001933B
:100FF00000F18402294600964FF48073143001F00A
:10100000D1FD094B0294CDE9006304F523724FF43E
:101010008073294604F14C0001F098FE04B070BDC5
:10102000EC340008C90F0008F10E00080B682022FC
:1010300082F311880A7903EB820290614A790932BE
:1010400043F822008A7912B103EB820398610223EC
:101050000374C0F89414002383F3118870470000D0
:1010600038B5037F044613B190F85430ABB9201D56
:1010700001250221FFF734FF04F1140025776FF0FA
:10108000010100F0B9FC84F8545004F14C006FF0F9
:101090000101BDE8384000F0AFBC38BD10B50121FA
:1010A00004460430FFF71CFF0023237784F85430F4
:1010B00010BD000038B504460025143001F08AFD4B
:1010C00004F14C00257701F059FE201D84F854509E
:1010D0000121FFF705FF2046BDE83840FFF752BF6A
:1010E00090F8443003F06003202B07D190F845209E
:1010F000212A4FF0000303D81F2A06D8002070478A
:10110000222AFBD1C0E90E3303E0034A826307229F
:10111000C2630364012070471122002037B5D0F864
:1011200094341A681178042904461AD1017C0229E2
:1011300017D11979128901238B40134211D100F183
:101140004C05284601F0DAFE58B101A9284601F005
:1011500021FED4F89444019B21790246206800F0D6
:10116000B3F803B030BD0000F0B500EB810385B0EB
:101170009E6904460D46FEB1202383F3118804EBDB
:101180008507301D0821FFF7ABFEFB685B691B6814
:1011900006F14C001BB1019001F00AFE019803A971
:1011A00001F0F8FD024648B1039B2946204600F0B5
:1011B0008BF8002383F3118805B0F0BDFB685A69F2
:1011C0001268002AF5D01B8A013B1340F1D104F1CB
:1011D0004402EAE7093138B550F82140DCB1202358
:1011E00083F31188D4F894241368527903EB8203B3
:1011F000DB689B695D6845B104216018FFF770FEEC
:10120000294604F1140001F0FBFC2046FFF7BAFE6A
:10121000002383F3118838BD7047000001F0A8B89F
:10122000012303700023C0E90133C36183620362B9
:10123000C36243620363704738B50446202383F3D7
:1012400011880025C0E90355C0E90555416001F04A
:101250009FF80223237085F3118838BD70B500EB29
:10126000810305465069DA600E46144618B1102213
:101270000021FFF75DFDA06918B110220021FFF7E2
:1012800057FD31462846BDE8704001F04BB90000DB
:10129000826802F0011282600022C0E904228261A9
:1012A00001F0CCB9F0B400EB81044789E468012572
:1012B000A4698D403D43458123600023A2606360A3
:1012C000F0BC01F0E7B90000F0B400EB810407893D
:1012D000E468012564698D403D4305812360002356
:1012E000A2606360F0BC01F061BA000070B5022337
:1012F000002504460370C0E90255C0E90455C564E1
:10130000856180F8345001F0A9F863681B6823B147
:1013100029462046BDE87040184770BD037880F824
:1013200050300523037043681B6810B504460BB1A9
:10133000042198470023A36010BD000090F85020BE
:10134000436802701B680BB1052118477047000005
:1013500070B590F83430044613B1002380F834306F
:1013600004F14402204601F08BF963689B68B3B92D
:1013700094F8443013F0600535D00021204601F088
:10138000DDFB0021204601F0CFFB63681B6813B131
:10139000062120469847062384F8343070BD204645
:1013A00098470028E4D0B4F84A30E26B9A4288BFEC
:1013B000E36394F94430E56B002B4FF0200380F297
:1013C0000381002D00F0F280092284F8342083F399
:1013D00011880021D4E90E232046FFF775FF002372
:1013E00083F31188DAE794F8452003F07F0343EA9A
:1013F000022340F20232934200F0C58021D8B3F5B7
:10140000807F48D00DD8012B3FD0022B00F0938075
:10141000002BB2D104F14C02A2630222E2632364E6
:10142000C1E7B3F5817F00F09B80B3F5407FA4D185
:1014300094F84630012BA0D1B4F84C3043F00203AD
:1014400032E0B3F5006F4DD017D8B3F5A06F31D0AF
:10145000A3F5C063012B90D8636894F846205E68BA
:1014600094F84710B4F848302046B047002884D09C
:101470004368A3630368E3631AE0B3F5106F36D0E3
:1014800040F6024293427FF478AF5C4BA3630223A1
:10149000E3630023C3E794F84630012B7FF46DAF7C
:1014A000B4F84C3023F00203C4E90E55A4F84C30D4
:1014B000256478E7B4F84430B3F5A06F0ED194F802
:1014C000463084F84E30204601F020F863681B68EF
:1014D00013B1012120469847032323700023C4E958
:1014E0000E339CE704F14F03A3630123C3E7237882
:1014F000042B10D1202383F311882046FFF7C8FE68
:1015000085F311880321636884F84F5021701B68AC
:101510000BB12046984794F84630002BDED084F873
:101520004F300423237063681B68002BD6D0022140
:1015300020469847D2E794F848301D0603F00F0183
:1015400020460AD501F08EF8012804D002287FF445
:1015500014AF2B4B9AE72B4B98E701F075F8F3E7A4
:1015600094F84630002B7FF408AF94F8483013F01D
:101570000F01B3D01A06204602D501F0F3FAADE709
:1015800001F0E6FAAAE794F84630002B7FF4F5AEB6
:1015900094F8483013F00F01A0D01B06204602D566
:1015A00001F0CCFA9AE701F0BFFA97E7142284F829
:1015B000342083F311882B462A4629462046FFF71C
:1015C00071FE85F31188E9E65DB1152284F83420B7
:1015D00083F311880021D4E90E232046FFF762FE31
:1015E000FDE60B2284F8342083F311882B462A462B
:1015F00029462046FFF768FEE3E700BF1C350008D8
:10160000143500081835000838B590F83430044611
:10161000002B3ED0063BDAB20F2A34D80F2B32D83B
:10162000DFE803F0373131082232313131313131E5
:1016300031313737C56BB0F84A309D4214D2C36898
:101640001B8AB5FBF3F203FB12556DB9202383F31C
:1016500011882B462A462946FFF736FE85F3118866
:101660000A2384F834300EE0142384F83430202325
:1016700083F3118800231A4619462046FFF712FE0D
:10168000002383F3118838BD036C03B1984700230E
:10169000E7E70021204601F051FA0021204601F041
:1016A00043FA63681B6813B1062120469847062356
:1016B000D7E7000010B590F83430142B044629D039
:1016C00017D8062B05D001D81BB110BD093B022B42
:1016D000FBD80021204601F031FA0021204601F01C
:1016E00023FA63681B6813B1062120469847062336
:1016F00019E0152BE9D10B2380F83430202383F334
:10170000118800231A461946FFF7DEFD002383F3F4
:101710001188DAE7C3689B695B68002BD5D1036C3D
:1017200003B19847002384F83430CEE7024B0022FF
:10173000C3E900339A6070479423002000230374A8
:101740008268054B1B6899689142FBD25A68036016
:1017500042601060586070479423002008B5202331
:1017600083F31188037C032B05D0042B0DD02BB9F8
:1017700083F3118808BD436900221A604FF0FF33DC
:101780004361FFF7DBFF0023F2E7D0E9003213608B
:101790005A60F3E7002303748268054B1B6899685D
:1017A0009142FBD85A6803604260106058607047ED
:1017B00094230020054B19690874186802681A60A0
:1017C0005360186101230374FEF7A0BD9423002029
:1017D00030B54B1C0B4D87B0044610D02B690A4A1C
:1017E00001A800F025F92046FFF7E4FF049B13B1A0
:1017F00001A800F059F92B69586907B030BDFFF70F
:10180000D9FFF8E7942300205D17000838B50C4D88
:1018100041612B6981689A689142044603D8BDE80A
:101820003840FFF78BBF1846FFF7B4FF01232C6148
:10183000014623742046BDE83840FEF767BD00BF6F
:1018400094230020044B1A681B6990689B68984297
:1018500094BF0020012070479423002010B5084C4D
:10186000236820691A6822605460012223611A7477
:10187000FFF790FF01462069BDE81040FEF746BD26
:101880009423002008B5FFF7DDFF18B1BDE808403C
:10189000FFF7E4BF08BD0000FFF7E0BFFEE7000070
:1018A00010B50C4CFFF742FF00F0B4F80A49802253
:1018B000204600F03BF8012344F8180C037400F0B4
:1018C00071FC002383F3118862B60448BDE8104020
:1018D00000F04CB8BC23002020350008303500084B
:1018E00000F01CB9EFF3118020B9EFF3058320223B
:1018F00082F311887047000010B530B9EFF305840A
:10190000C4F3080414B180F3118810BDFFF7BAFFC7
:1019100084F31188F9E70000034A516853685B1AA1
:101920009842FBD8704700BF001000E0826002229E
:10193000028270478368A3F17C0243F80C2C026991
:1019400043F83C2C426943F8382C074A43F81C2CD6
:10195000C26843F8102C022203F8082C002203F876
:10196000072CA3F1180070472503000810B52023A9
:1019700083F31188FFF7DEFF00210446FFF746FFDF
:10198000002383F31188204610BD0000024B1B6921
:1019900058610F20FFF70EBF94230020202383F30C
:1019A0001188FFF7F3BF000008B50146202383F339
:1019B00011880820FFF70CFF002383F3118808BD6E
:1019C00049B1064B42681B6918605A601360436056
:1019D0000420FFF7FDBE4FF0FF3070479423002036
:1019E0000368984206D01A68026050605961184630
:1019F000FFF7A4BE7047000038B504460D462068C6
:101A0000844200D138BD036823605C604561FFF704
:101A100095FEF4E7054B03F11402C3E905224FF0EC
:101A2000FF310022C3E90712704700BF9423002052
:101A300070B51C4EC0E9032305460C4601F090FA30
:101A4000334653F8142F9A420DD13062C5E9012470
:101A50002A600A2C2CBF00190A30C6E90555BDE8DA
:101A6000704001F06BBA316A431AE31838BF1C4664
:101A70009368A34202D9081901F06EFA73699A6853
:101A800094420CD85A68AC602B606A6015609A6802
:101A90005D60121B9A604FF0FF33F36170BD1B68ED
:101AA000A41AECE79423002038B51B4C63699842D4
:101AB0000DD0D0E9003213605A6000228168C26004
:101AC0009A680A449A604FF0FF33E36138BD2246BA
:101AD000036842F8143F002193425A60C16003D169
:101AE000BDE8384001F032BA9A688168256A0A4434
:101AF0009A6001F035FA63699A68411B8A42E5D918
:101B0000AB181D1A092D206A98BF01F10A02BDE821
:101B10003840104401F020BA942300202DE9F04110
:101B2000184C002704F11406656901F019FA236ABC
:101B3000AA68C11A8A4215D813442362D5E9003233
:101B400013605A606369D5F80C80EF60B34201D12D
:101B500001F0FCF987F311882869C047202383F33B
:101B60001188E1E76169B14209D013441B1ABDE84D
:101B7000F0410A2B2CBFC0180A3001F0EDB9BDE8C6
:101B8000F08100BF9423002000207047FEE7000092
:101B9000704700004FF0FF307047000002290CD062
:101BA000032904D00129074818BF00207047032AE1
:101BB00005D8054800EBC200704704487047002074
:101BC000704700BF1436000820220020C8350008E6
:101BD00070B59AB00546084601A9144600F0C2F84F
:101BE00001A8FFF79DF8431C5B00C5E90034002203
:101BF000237003236370C6B201AB02341046D1B226
:101C00008E4204F1020401D81AB070BD13F8011B12
:101C100004F8021C04F8010C0132F0E708B5202397
:101C200083F311880348FFF779FA002383F31188BF
:101C300008BD00BF5025002090F8443003F01F027B
:101C4000012A07D190F845200B2A03D10023C0E9CF
:101C50000E3315E003F06003202B08D1B0F84830B4
:101C60002BB990F84520212A03D81F2A04D8FFF762
:101C700037BA222AEBD0FAE7034A82630722C2630B
:101C800003640120704700BF1822002007B5052912
:101C900017D8DFE801F0191603191920202383F360
:101CA0001188104A01900121FFF7D8FA01980E4AD5
:101CB0000221FFF7D3FA0D48FFF7FCF9002383F365
:101CC000118803B05DF804FB202383F311880748D3
:101CD000FFF7C6F9F2E7202383F311880348FFF7E3
:101CE000DDF9EBE7683500088C3500085025002049
:101CF00038B50C4D0C4C0D492A4604F10800FFF78D
:101D000067FF05F1CA0204F110000949FFF760FFFF
:101D100005F5CA7204F118000649BDE83840FFF71E
:101D200057BF00BF182A0020202200204835000895
:101D3000523500085D35000870B5044608460D466A
:101D4000FEF7EEFFC6B22046013403780BB9184601
:101D500070BD32462946FEF7CFFF0028F3D101209F
:101D6000F6E700002DE9F04705460C46FEF7D8FFE0
:101D70002B49C6B22846FFF7DFFF08B10636F6B298
:101D800028492846FFF7D8FF08B11036F6B2632E6F
:101D90000BD8DFF88C80DFF88C90234FDFF894A00D
:101DA0002E7846B92670BDE8F08729462046BDE862
:101DB000F04701F065BB252E2ED10722414628466B
:101DC000FEF79AFF70B9194B224603F10C0153F844
:101DD000040B42F8040B8B42F9D11B7813700735C2
:101DE0000D34DDE7082249462846FEF785FF98B9FD
:101DF0000F4BA21C197809090232C95D02F8041CB4
:101E000013F8011B01F00F015345C95D02F8031CD3
:101E1000F0D118340835C3E704F8016B0135BFE78A
:101E2000343600085D3500084A3600083C360008A4
:101E3000107AFF1F1C7AFF1FBFF34F8F024AD3682F
:101E4000DB03FCD4704700BF003C024008B5094BDF
:101E50001B7873B9FFF7F0FF074B1A69002ABFBF61
:101E6000064A5A6002F188325A601A6822F4806287
:101E70001A6008BD762C0020003C02402301674513
:101E800008B50B4B1B7893B9FFF7D6FF094B1A69BE
:101E900042F000421A611A6842F480521A601A68CD
:101EA00022F480521A601A6842F480621A6008BDF7
:101EB000762C0020003C02400B28F0B516D80C4CC4
:101EC0000C4923787BB90C4D0E460C234FF0006271
:101ED00055F8047B46F8042B013B13F0FF033A440A
:101EE000F6D10123237051F82000F0BD0020FCE75B
:101EF000A82C0020782C00205C360008014B53F8F9
:101F0000200070475C3600080C2070470B2810B585
:101F1000044601D9002010BDFFF7CEFF064B53F851
:101F200024301844C21A0BB90120F4E712680132B8
:101F3000F0D1043BF6E700BF5C3600080B2838B54B
:101F4000044628D8FFF7CEFCFFF776FFFFF77EFFA9
:101F5000124AF323D360E300DBB243F4007343F08F
:101F600002031361136943F480331361054620466D
:101F7000FFF762FFFFF7A0FF094B53F8241000F0B2
:101F8000E9F82846FFF77CFFFFF7B6FC2046BDE8DE
:101F90003840FFF7BBBF002038BD00BF003C024007
:101FA0005C36000812F001032DE9F04105460E46AB
:101FB00014464BD18218B2F1016F61D8314B1B68C6
:101FC00013F001035CD0304FFFF78CFCFFF73EFFAE
:101FD000F323FB60FFF730FF314640F20128032C6A
:101FE00018D824F00104284E0C446D1A40F2011850
:101FF000A142336905EB01072AD123F001033361C4
:10200000FFF73EFFFFF778FC0120BDE8F081043CBC
:102010000435E4E7AB07E4D13B6923F440733B614B
:102020003B6943EA08033B6151F8046B2E60BFF340
:102030004F8FFFF701FF2B689E42E8D03B6923F0EA
:1020400001033B61FFF71CFFFFF756FC0020DCE7B4
:1020500023F440733361336943EA080333610B8827
:102060003B80BFF34F8FFFF7E7FE3F8831F8023B1D
:10207000BFB2BB42BCD0336923F001033361E1E757
:102080001846C2E700380240003C0240084908B543
:102090000B7828B11BB9FFF7D9FE01230B7008BDDF
:1020A000002BFCD0BDE808400870FFF7E9BE00BF78
:1020B000762C002010B50244064BD2B2904200D1DB
:1020C00010BD441C00B253F8200041F8040BE0B2EC
:1020D000F4E700BF502800400F4B30B51C6F2404BC
:1020E00007D41C6F44F400741C671C6F44F4004454
:1020F0001C670A4C236843F4807323600244084B36
:10210000D2B2904200D130BD441C00B251F8045B01
:1021100043F82050E0B2F4E700380240007000407D
:102120005028004007B5012201A90020FFF7C2FF97
:10213000019803B05DF804FB13B50446FFF7F2FF06
:10214000A04205D0012201A900200194FFF7C4FF9D
:1021500002B010BD70470000034B1A681AB9034A59
:10216000D2F874281A607047AC2C0020003002406E
:1021700008B5FFF7F1FF024B1868C0F3407008BDC7
:10218000AC2C0020EFF3098305494A6B22F00102D1
:102190004A63683383F30988002383F31188704707
:1021A00000EF00E0202080F3118862B60C4B0D4A4E
:1021B000D96821F4E0610904090C0A43DA60D3F814
:1021C000FC20094942F08072C3F8FC200A6842F002
:1021D00001020A601022DA7783F82200704700BFFC
:1021E00000ED00E00003FA05001000E010B5202328
:1021F00083F311880E4B5B6813F4006314D0F1EE87
:10220000103AEFF30984683C4FF08073E361094BA7
:10221000DB6B236684F30988FFF714FB10B1064BD0
:10222000A36110BD054BFBE783F31188F9E700BFFD
:1022300000ED00E000EF00E0370300083A0300087B
:1022400070470000FEE700000A4B0B480B4A904223
:102250000BD30B4BDA1C121AC11E22F003028B4265
:1022600038BF00220021FEF763BD53F8041B40F87D
:10227000041BECE7F8370008A82D0020A82D00204B
:10228000A82D00207047000070B5D0E915439E6866
:1022900000224FF0FF3504EB42135101D3F800093F
:1022A0000028BEBFD3F8000940F08040C3F8000901
:1022B000D3F8000B0028BEBFD3F8000B40F08040DD
:1022C000C3F8000B013263189642C3F80859C3F8EB
:1022D000085BE0D24FF00113C4F81C3870BD000059
:1022E0001D4B03EB80022DE9F043D2F80CC05D6D6D
:1022F000DCF81420461CD2F800E005EB063605EBAE
:102300004018516871450AD3D5F83438012202FAD1
:1023100000F023EA0000C5F83408BDE8F083BCF8FB
:102320001040AEEB0103A34228BF2346D8F818495A
:10233000A4B2B3EB840FF0D89468A4F1040959F85F
:10234000047F3760A4EB09071F44042FF7D81C440F
:102350000B4494605360D4E7B02C0020890141F015
:102360002001016103699B06FCD41220FFF7D4BA57
:1023700010B5054C2046FEF753FF4FF0A0436365B0
:10238000024BA36510BD00BFB02C0020B036000882
:1023900070B50378012B054650D12A4B446D984205
:1023A0001BD1294B5A6B42F080025A635A6D42F09E
:1023B00080025A655A6D5A6942F080025A615A6920
:1023C00022F080025A610E2143205B6900F0D4FBA9
:1023D0001E4BE3601E4BC4F800380023C4F8003ED7
:1023E000C02323606E6D4FF40413A3633369002B85
:1023F000FCDA012333610C20FFF78EFA3369DB0727
:10240000FCD41220FFF788FA3369002BFCDA00268F
:10241000A6602846FFF738FF6B68C4F81068DB68D1
:10242000C4F81468C4F81C684BB90A4BA3614FF098
:10243000FF336361A36843F00103A36070BD064BE3
:10244000F4E700BFB02C00200038024040140040E8
:1024500003002002003C30C0083C30C0F8B5446D99
:10246000054600212046FFF779FFA96D00234FF0B4
:1024700001128F68C4F834384FF00066C4F81C2885
:102480004FF0FF3004EB431201339F42C2F8006962
:10249000C2F8006BC2F80809C2F8080BF2D20B6848
:1024A0006A6DEB65636210231361166916F01006FE
:1024B000FBD11220FFF730FAD4F8003823F4FE6382
:1024C000C4F80038A36943F4402343F01003A36128
:1024D0000923C4F81038C4F814380A4BEB604FF0E5
:1024E000C043C4F8103B084BC4F8003BC4F8106963
:1024F000C4F80039EB6D03F1100243F48013EA6570
:10250000A362F8BD8C36000840800010426D90F840
:102510004E10D2F8003823F4FE6343EA0113C2F8E8
:10252000003870472DE9F84300EB8103456DDA6808
:10253000166806F00306731E022B05EB41130C46CA
:1025400080460FFA81F94FEA41104FF00001C3F8BD
:10255000101B4FF0010104F1100398BFB60401FAFB
:1025600003F391698EBF334E06F1805606F500469F
:1025700000293AD0578A04F15801490137436F5076
:10258000D5F81C180B43C5F81C382B180021C3F8CC
:10259000101953690127611EA7409BB3138A928BC0
:1025A0009B08012A88BF5343D8F85C20981842EA58
:1025B000034301F1400205EB8202C8F85C002146AA
:1025C00053602846FFF7CAFE08EB8900C3681B8AE0
:1025D00043EA8453483464011E432E51D5F81C3815
:1025E0001F43C5F81C78BDE8F88305EB4917D7F8F9
:1025F000001B21F40041C7F8001BD5F81C1821EA84
:102600000303C0E704F13F0305EB83030A4A5A6062
:1026100028462146FFF7A2FE05EB4910D0F8003905
:1026200023F40043C0F80039D5F81C3823EA070723
:10263000D7E700BF0080001000040002826D12681E
:10264000C265FFF721BE00005831436D49015B5858
:1026500013F4004004D013F4001F0CBF022001202B
:10266000704700004831436D49015B5813F4004046
:1026700004D013F4001F0CBF02200120704700009B
:1026800000EB8101CB68196A0B6813604B685360DB
:102690007047000000EB810330B5DD68AA6913685C
:1026A000D36019B9402B84BF402313606B8A146830
:1026B000426D1C44013CB4FBF3F46343033323F049
:1026C000030302EB411043EAC44343F0C043C0F8A4
:1026D000103B2B6803F00303012B09B20ED1D2F893
:1026E000083802EB411013F4807FD0F8003B14BF90
:1026F00043F0805343F00053C0F8003B02EB41121B
:10270000D2F8003B43F00443C2F8003B30BD000068
:102710002DE9F041244D6E6D06EB40130446D3F8CD
:10272000087BC3F8087B38070AD5D6F81438190790
:1027300006D505EB84032146DB6828465B6898478D
:10274000FA071FD5D6F81438DB071BD505EB840331
:10275000D968CCB98B69488A5A68B2FBF0F600FB9D
:1027600016228AB91868DA6890420DD2121AC3E9A3
:102770000024202383F311880B482146FFF78AFFAA
:1027800084F31188BDE8F081012303FA04F26B8918
:1027900023EA02036B81CB68002BF3D02146024869
:1027A000BDE8F041184700BFB02C002000EB8103CA
:1027B00070B5DD68436D6C692668E6604A0156BBFA
:1027C0001A444FF40020C2F810092A6802F00302EC
:1027D000012A0AB20ED1D3F8080803EB421410F410
:1027E000807FD4F8000914BF40F0805040F00050C2
:1027F000C4F8000903EB4212D2F8000940F004408B
:10280000C2F80009D3F83408012202FA01F10143A9
:10281000C3F8341870BD19B9402E84BF4020206021
:1028200020682E8A8419013CB4FBF6F440EAC440C7
:1028300040F000501A44C6E7F8B504461E48456DFE
:1028400005EB4413D3F80869C3F80869F10717D5F5
:10285000D5F81038DA0713D500EB8403D9684B6933
:102860001F68DA68974218D2D21B00271A605F608F
:10287000202383F311882146FFF798FF87F31188FF
:10288000330617D5D5F834280123A340134211D0BD
:102890002046BDE8F840FFF723BD012303FA04F208
:1028A000038923EA020303818B68002BE8D02146C9
:1028B0009847E5E7F8BD00BFB02C00202DE9F74FA1
:1028C000984C666D7569B3691D4015F48058756143
:1028D00007D02046FEF70AFD03B0BDE8F04FFFF732
:1028E00085BC002D12DAD6F8003E8E489F071EBF29
:1028F000D6F8003E23F00303C6F8003ED6F80438AD
:1029000023F00103C6F80438FEF718FD280505D5A5
:102910008448FFF7B9FC8348FEF700FDA9040CD5F5
:10292000D6F8083813F0060FF36823F470530CBF81
:1029300043F4105343F4A053F3602A0704D56368AB
:10294000DB680BB177489847EB0274D4AF0227D508
:10295000D4F85490DFF8CCB100274FF0010A09EB0E
:102960004712D2F8003B03F44023B3F5802F11D176
:10297000D2F8003B002B0DDA62890AFA07F322EA4B
:102980000303638104EB8703DB68DB6813B139461B
:1029900058469847A36D01379B68FFB29F42DED926
:1029A000E80617D5676D3A6AC2F30A1002F00F0302
:1029B00002F4F012B2F5802F00F08880B2F5402FBB
:1029C00008D104EB83030022DB681B6A07F58057FC
:1029D00090426DD12903D6F8184813D5E20302D5E9
:1029E0000020FFF795FEA30302D50120FFF790FE1C
:1029F000670302D50220FFF78BFE260302D50320D2
:102A0000FFF786FE6D037FF567AFE00702D5002074
:102A1000FFF712FFA10702D50120FFF70DFF6207A4
:102A200002D50220FFF708FF23077FF555AF0320EB
:102A3000FFF702FF50E7636DDFF8E8B0019300276E
:102A40004FF0010AA36D9B685FFA87F999453FF63D
:102A50007DAF019B03EB4913D3F8002902F4402218
:102A6000B2F5802F22D1D3F80029002A1EDAD3F83C
:102A7000002942F09042C3F80029D3F80029002A27
:102A8000FBDB606D4946FFF769FC22890AFA09F30E
:102A900022EA0303238104EB8903DB689B6813B1FB
:102AA0004946584698474846FFF71AFC0137C9E798
:102AB000910708BFD7F80080072A98BF03F8018B59
:102AC00002F1010298BF4FEA182881E7023304EBB4
:102AD000830207F580575268D2F818C0DCF8082046
:102AE000DCE9001CA1EB0C0C002188420AD104EBAC
:102AF000830463689B699A6802449A605A68024436
:102B00005A6067E711F0030F08BFD7F800808C45C3
:102B100088BF02F8018B01F1010188BF4FEA182834
:102B2000E3E700BFB02C0020436D03EB4111D1F867
:102B3000003B43F40013C1F8003B7047436D03EBC7
:102B40004111D1F8003943F40013C1F8003970473E
:102B5000436D03EB4111D1F8003B23F40013C1F89E
:102B6000003B7047436D03EB4111D1F8003923F46A
:102B70000013C1F80039704700F1604303F5614369
:102B80000901C9B283F80013012200F01F039A4023
:102B900043099B0003F1604303F56143C3F88021BF
:102BA0001A60704730B5039C0172043304FB03259F
:102BB000C0E90653049B03630021059BC160C0E983
:102BC0000000C0E90422C0E90842C0E90A114363D9
:102BD00030BD0000416A0022C0E90411C0E90A22A8
:102BE000C2606FF00101FEF707BF0000D0E90432B8
:102BF000934201D1C2680AB9181D7047002070477E
:102C000003691960C2680132C260C26913448269F3
:102C10000361934224BF436A03610021FEF7E0BED3
:102C200038B504460D46E3683BB16269131D12686E
:102C3000A3621344E362002007E0237A33B92946F4
:102C40002046FEF7BDFE0028EDDA38BD6FF001002A
:102C5000FBE70000C368C269013BC36043691344DA
:102C600082694361934224BF436A436100238362C4
:102C7000036B03B11847704770B52023044683F3F4
:102C80001188866A3EB9FFF7CBFF054618B186F377
:102C90001188284670BDA36AE26A13F8015BA3623B
:102CA000934202D32046FFF7D5FF002383F3118818
:102CB000EFE700002DE9F84F04460E461746984608
:102CC0004FF0200989F311880025AA46D4F828B0CE
:102CD000BBF1000F09D141462046FFF7A1FF20B10B
:102CE0008BF311882846BDE8F88FD4E90A12A7EBC8
:102CF000050B521A934528BF9346BBF1400F1BD9D1
:102D0000334601F1400251F8040B43F8040B9142A1
:102D1000F9D1A36A40334036A3624035D4E90A238F
:102D20009A4202D32046FFF795FF8AF31188BD42ED
:102D3000D8D289F31188C9E730465A46FDF7D2FF49
:102D4000A36A5B445E44A3625D44E7E710B5029C5E
:102D50000172043304FB0321C0E906130023C0E918
:102D60000A33039B0363049BC460C0E90000C0E90D
:102D70000422C0E90842436310BD0000026AC26039
:102D8000426AC0E904220022C0E90A226FF0010170
:102D9000FEF732BED0E904239A4201D1C26822B9BB
:102DA000184650F8043B0B60704700207047000045
:102DB000C368C2690133C3604369134482694361D4
:102DC000934224BF436A43610021FEF709BE00001D
:102DD00038B504460D46E3683BB123691A1DA2626B
:102DE000E2691344E362002007E0237A33B92946FD
:102DF0002046FEF7E5FD0028EDDA38BD6FF0010052
:102E0000FBE7000003691960C268013AC260C26949
:102E1000134482690361934224BF436A0361002320
:102E20008362036B03B118477047000070B520231D
:102E30000D460446114683F31188866A2EB9FFF7C2
:102E4000C7FF10B186F3118870BDA36A1D70A36A15
:102E5000E26A01339342A36204D3E1692046043954
:102E6000FFF7D0FF002080F31188EDE72DE9F84F40
:102E700004460D46904699464FF0200A8AF3118881
:102E80000026B346A76A4FB949462046FFF7A0FF80
:102E900020B187F311883046BDE8F88FD4E90A07DE
:102EA0003A1AA8EB0607974228BF1746402F1BD9AE
:102EB00005F1400355F8042B40F8042B9D42F9D14D
:102EC000A36A4033A3624036D4E90A239A4204D36A
:102ED000E16920460439FFF795FF8BF311884645D9
:102EE000D9D28AF31188CDE729463A46FDF7FAFE92
:102EF000A36A3B443D44A3623E44E5E7D0E9042392
:102F00009A4217D1C3689BB1836A8BB1043B9B1A69
:102F10000ED01360C368013BC360C3691A44836960
:102F200002619A4224BF436A036100238362012342
:102F3000184670470023FBE700F088B84FF0804345
:102F4000002258631A610222DA6070474FF0804312
:102F50000022DA60704700004FF0804358637047EA
:102F60004FF08043586A70474B6843608B688360BA
:102F7000CB68C3600B6943614B6903628B69436231
:102F80000B6803607047000008B5264B26481A6995
:102F900040F2FF110A431A611A6922F4FF7222F00B
:102FA00001021A611A691A6B0A431A631A6D0A43FD
:102FB0001A651E4A1B6D1146FFF7D6FF02F11C0170
:102FC00000F58060FFF7D0FF02F1380100F5806066
:102FD000FFF7CAFF02F1540100F58060FFF7C4FF5C
:102FE00002F1700100F58060FFF7BEFF02F18C0175
:102FF00000F58060FFF7B8FF02F1A80100F58060DE
:10300000FFF7B2FF02F1C40100F58060FFF7ACFFEB
:1030100002F1E00100F58060FFF7A6FFBDE808407F
:1030200000F09AB80038024000000240BC360008A8
:1030300008B500F007FAFEF733FCFFF78DF8BDE89E
:103040000840FEF755BE000070470000104B1A6C98
:1030500042F001021A641A6E42F001021A660D4A29
:103060001B6E936843F0010393604FF0804353223B
:103070009A624FF0FF32DA6200229A615A63DA6094
:103080005A6001225A6108211A601C20FFF774BDA2
:1030900000380240002004E04FF0804208B511697A
:1030A000D3680B40D9B2C9439B07116107D52023D0
:1030B00083F31188FEF714FC002383F3118808BD05
:1030C00008B5FFF7E9FFBDE80840FFF78FB800003B
:1030D0001F4B1A696FEAC2526FEAD2521A611A691B
:1030E000C2F308021A614FF0FF301A695A69586139
:1030F00000215A6959615A691A6A62F080521A624B
:103100001A6A02F080521A621A6A5A6A58625A6A35
:1031100059625A6A1A6C42F080521A641A6E42F06E
:1031200080521A661A6E0B4A106840F48070106064
:10313000186F00F44070B0F5007F1EBF4FF4803070
:1031400018671967536823F40073536000F05AB985
:103150000038024000700040334B4FF080521A6438
:10316000324A4FF4404111601A6842F001021A607D
:103170001A689107FCD59A6822F003029A602A4BDC
:103180009A6812F00C02FBD1196801F0F90119607C
:103190009A601A6842F480321A601A689203FCD569
:1031A0005A6F42F001025A671F4B5A6F9007FCD5C5
:1031B0001F4A5A601A6842F080721A601B4A5368AC
:1031C0005904FCD5184B1A689201FCD5194A9A602B
:1031D000194B1A68194B9A42194B21D1194A116897
:1031E000194A91421CD140F205121A60144A136820
:1031F00003F00F03052BFAD10B4B9A6842F0020241
:103200009A609A6802F00C02082AFAD15A6C42F4C9
:1032100080425A645A6E42F480425A665B6E70472E
:1032200040F20572E1E700BF003802400070004044
:103230000854400700948838002004E011640020FE
:10324000003C024000ED00E041C20F41084A08B5D1
:10325000516913680B4003F00103536123B1054A20
:1032600013680BB150689847BDE80840FEF7BEBF31
:10327000003C0140282D0020084A08B55169136818
:103280000B4003F00203536123B1054A93680BB16D
:10329000D0689847BDE80840FEF7A8BF003C014051
:1032A000282D0020084A08B5516913680B4003F027
:1032B0000403536123B1054A13690BB15069984760
:1032C000BDE80840FEF792BF003C0140282D0020D9
:1032D000084A08B5516913680B4003F008035361AD
:1032E00023B1054A93690BB1D0699847BDE80840FE
:1032F000FEF77CBF003C0140282D0020084A08B59D
:10330000516913680B4003F01003536123B1054A60
:10331000136A0BB1506A9847BDE80840FEF766BFD4
:10332000003C0140282D0020174B10B55A691C683D
:10333000144004F478725A61A30604D5134A936AC0
:103340000BB1D06A9847600604D5104A136B0BB1D5
:10335000506B9847210604D50C4A936B0BB1D06B88
:103360009847E20504D5094A136C0BB1506C984795
:10337000A30504D5054A936C0BB1D06C9847BDE802
:103380001040FEF733BF00BF003C0140282D002055
:103390001A4B10B55A691C68144004F47C425A61F7
:1033A000620504D5164A136D0BB1506D984723057D
:1033B00004D5134A936D0BB1D06D9847E00404D542
:1033C0000F4A136E0BB1506E9847A10404D50C4AF6
:1033D000936E0BB1D06E9847620404D5084A136F00
:1033E0000BB1506F9847230404D5054A936F0BB176
:1033F000D06F9847BDE81040FEF7F8BE003C014092
:10340000282D0020062108B50846FFF7B5FB062148
:103410000720FFF7B1FB06210820FFF7ADFB0621CF
:103420000920FFF7A9FB06210A20FFF7A5FB0621CB
:103430001720FFF7A1FBBDE8084006212820FFF771
:103440009BBB000008B5FFF743FE00F00BF8FDF74B
:10345000E5FEFDF7BDFDFFF7F7FDBDE80840FFF70E
:103460006BBD00000023054A19460133102BC2E949
:10347000001102F10802F8D1704700BF282D00208A
:10348000034611F8012B03F8012B002AF9D17047EC
:1034900053544D3332463F3F3F00000053544D33A9
:1034A00032463430780053544D333246343278004B
:1034B00053544D333246343436585800000000001F
:1034C000903400083F000000130400009C34000802
:1034D0003F00000019040000A63400083F0000006F
:1034E00021040000B03400083F000000000000008C
:1034F0004D0F0008390F0008750F0008610F000814
:103500006D0F0008590F0008450F0008310F000823
:10351000810F000800000000010000000000000012
:103520006D61696E0000000069646C650000000058
:1035300028350008D8230020502500200100000075
:103540009D180008000000004172647550696C6F9E
:10355000740025424F415244252D424C00255345CD
:103560005249414C2500000002000000000000000C
:1035700069110008D511000840004000E82900202A
:10358000F8290020020000000000000003000000F5
:1035900000000000191200080000000010000000E8
:1035A000082A0020000000000100000000000000C8
:1035B000B02C0020010102008D1C00089D1B00089A
:1035C000391C00081D1C000843000000D03500080D
:1035D00009024300020100C0320904000001020296
:1035E0000100052400100105240100010424020249
:1035F0000524060001070582030800FF09040100F5
:10360000020A0000000705010240000007058102D0
:1036100040000000120000001C36000812011001DA
:10362000020000400912415700020102030100009C
:103630000403090425424F41524425004D6174653D
:103640006B463430352D53544400303132333435E9
:1036500036373839414243444546000000400000B7
:103660000040000000400000004000000000010099
:103670000000020000000200000002000000020042
:103680000000020000000200000002000000000034
:103690005113000809160008B51600084000400044
:1036A000102D0020102D002001000000202D0020F2
:1036B00080000000400100000300000000008012B4
:1036C00000000000AAAAAAAA00000000FFBF000094
:1036D0000000000000A00A0000001400000000002C
:1036E000AAAAAAAA00001000FFFD00000000000026
:1036F000000000001500000000000000AAAAAAAA0D
:1037000015000000FFFF00000000000000000000A6
:103710000000000000000000AAAAAAAA0000000001
:10372000FFFF00000000000000000000000000009B
:1037300000000000AAAAAAAA00000000FFFF0000E3
:103740000000000000000000000000000000000079
:10375000AAAAAAAA00000000FFFF000000000000C3
:10376000000000000000000000000000AAAAAAAAB1
:1037700000000000FFFF000000000000000000004B
:1037800000000000000000000A000000000000002F
:103790000300000000000000000000000000000026
:1037A0000000000000000000000000000000000019
:1037B00000000000000000007D000000000000008C
:1037C00000000F0000000000FF009600000000084D
:1037D00000960000000008000400000030360008D9
:1037E00000000000000000000000000000000000D9
:1037F0000000000000000000FFFFFFFFFFFFFFFFD1
:10380000FFFFFFFFFFFFFFFFFFFFFFFFFFFFFFFFC8
:10381000FFFFFFFFFFFFFFFFFFFFFFFFFFFFFFFFB8
:10382000FFFFFFFFFFFFFFFFFFFFFFFFFFFFFFFFA8
:10383000FFFFFFFFFFFFFFFFFFFFFFFFFFFFFFFF98
:020000040801F1
:100000000006002099120108014C08085D4B080801
:10001000C94B08085D4B0808954B08089B1201085E
:100020009B1201089B1201089B120108D5DF0A08E8
:100030009B1201089B1201089B1201089B120108E8
:100040009B1201089B1201089B1201089B120108D8
:100050009B1201089B1201086DEB0A0895EB0A0838
:10006000BDEB0A08E5EB0A080DEC0A0841900A0806
:1000700069900A0895900A08C1900A08ED900A084C
:1000800015910A0841910A08C58F0A089B120108B8
:100090009B1201089B1201089B12010835EC0A080B
:1000A0006DED0A0881ED0A0895ED0A0899ED0A0838
:1000B0009DED0A08B1ED0A08C5ED0A08CD960A08BB
:1000C00075980A089B1201089B1201089B120108EF
:1000D0009B12010809ED0A081DED0A0831ED0A0816
:1000E00099EC0A089B1201089B120108E9ED0A0825
:1000F000EDED0A0801EE0A0805EE0A086D910A08FE
:100100009B1201089B120108D9ED0A089B120108F5
:1001100045ED0A0859ED0A089B1201089B120108D7
:1001200099910A08C1910A08ED910A0819920A08E2
:1001300045920A089B1201089B1201089B120108B4
:100140009B1201089B1201089B12010801E70A0893
:100150006D920A0899920A08C5920A089B12010832
:100160009B1201089B1201089B1201089B120108B7
:100170009B1201089B1201089B1201089B120108A7
:100180009B1201089B1201089B1201089B12010897
:100190009B1201089B1201089B1201089B12010887
:1001A0009B1201089B1201089B1201089B12010877
:1001B0009B1201089B1201089B1201089B12010867
:1001C0009B1201089B1201089B1201089B12010857
:1001D0009B1201089B1201089B1201089B12010847
:1001E000FD3E01084D8B01087D340208315C030897
:1001F000C1F004081DF60408ED70050805D40508D3
:10020000DDDB050811DF0508395B060859E2060841
:1002100021000708510D0708993D08088D4208087C
:10022000DD75090851D2090845F609083D010A089B
:10023000F92E0A0825350A08000000000000000019
:1002400081F0004102E000BF83F0004330B54FEA87
:1002500041044FEA430594EA050F08BF90EA020FF4
:100260001FBF54EA000C55EA020C7FEA645C7FEA87
:10027000655C00F0E2804FEA5454D4EB5555B8BFAA
:100280006D420CDD2C4480EA020281EA030382EA1B
:10029000000083EA010180EA020281EA0303362DAD
:1002A00088BF30BD11F0004F4FEA01314FF4801C80
:1002B0004CEA113102D0404261EB410113F0004F92
:1002C0004FEA03334CEA133302D0524263EB430349
:1002D00094EA050F00F0A780A4F10104D5F1200EE7
:1002E0000DDB02FA0EFC22FA05F2801841F1000142
:1002F00003FA0EF2801843FA05F359410EE0A5F116
:1003000020050EF1200E012A03FA0EFC28BF4CF046
:10031000020C43FA05F3C01851EBE37101F00045FC
:1003200007D54FF0000EDCF1000C7EEB00006EEB09
:100330000101B1F5801F1BD3B1F5001F0CD3490893
:100340005FEA30004FEA3C0C04F101044FEA4452EA
:1003500012F5800F80F09A80BCF1004F08BF5FEA71
:10036000500C50F1000041EB045141EA050130BD51
:100370005FEA4C0C404141EB0101013C28BFB1F563
:10038000801FE9D291F0000F04BF01460020B1FAAE
:1003900081F308BF2033A3F10B03B3F120020CDA81
:1003A0000C3208DD02F1140CC2F10C0201FA0CF05F
:1003B00021FA02F10CE002F11402D8BFC2F1200CC4
:1003C00001FA02F120FA0CFCDCBF41EA0C0190407A
:1003D000E41AA2BF01EB0451294330BD6FEA0404C3
:1003E0001F3C1CDA0C340EDC04F11404C4F12002AE
:1003F00020FA04F001FA02F340EA030021FA04F3C0
:1004000045EA030130BDC4F10C04C4F1200220FA16
:1004100002F001FA04F340EA0300294630BD21FA54
:1004200004F0294630BD94F0000F83F4801306BF1A
:1004300081F480110134013D4EE77FEA645C18BF0E
:100440007FEA655C29D094EA050F08BF90EA020FA5
:1004500005D054EA000C04BF1946104630BD91EA9D
:10046000030F1EBF0021002030BD5FEA545C05D1A0
:100470004000494128BF41F0004130BD14F58004DF
:100480003CBF01F5801130BD01F0004545F0FE4153
:1004900041F470014FF0000030BD7FEA645C1ABF88
:1004A000194610467FEA655C1CBF0B46024650EABF
:1004B000013406BF52EA033591EA030F41F40021EB
:1004C00030BD00BF90F0000F04BF0021704730B571
:1004D0004FF4806404F132044FF000054FF0000146
:1004E00050E700BF90F0000F04BF0021704730B507
:1004F0004FF4806404F1320410F0004548BF4042DC
:100500004FF000013EE700BF42004FEAE2014FEA30
:1005100031014FEA02701FBF12F07F4393F07F4F0B
:1005200081F06051704732F07F4208BF704793F00E
:100530007F4F04BF41F40021704730B54FF4607421
:1005400001F0004521F000411CE700BF50EA010224
:1005500008BF704730B54FF000050AE050EA0102CD
:1005600008BF704730B511F0004502D5404261EB3D
:1005700041014FF4806404F132045FEA915C3FF47E
:10058000D8AE4FF003025FEADC0C18BF03325FEA1B
:10059000DC0C18BF033202EBDC02C2F1200300FACC
:1005A00003FC20FA02F001FA03FE40EA0E0021FAF1
:1005B00002F11444BDE600BF70B54FF0FF0C4CF4DF
:1005C000E06C1CEA11541DBF1CEA135594EA0C0F91
:1005D00095EA0C0F00F0DEF82C4481EA030621EACC
:1005E0004C5123EA4C5350EA013518BF52EA033507
:1005F00041F4801143F4801338D0A0FB02CE4FF0B9
:100600000005E1FB02E506F00042E0FB03E54FF0E8
:100610000006E1FB03569CF0000F18BF4EF0010EE0
:10062000A4F1FF04B6F5007F64F5407404D25FEADC
:100630004E0E6D4146EB060642EAC62141EA55518F
:100640004FEAC52040EA5E504FEACE2EB4F1FD0CD1
:1006500088BFBCF5E06F1ED8BEF1004F08BF5FEA4F
:10066000500E50F1000041EB045170BD06F0004601
:1006700046EA010140EA020081EA0301B4EB5C04AE
:10068000C2BFD4EB0C0541EA045170BD41F48011A6
:100690004FF0000E013C00F3AB8014F1360FDEBFCB
:1006A000002001F0004170BDC4F10004203C35DAA7
:1006B0000C341BDC04F11404C4F1200500FA05F32A
:1006C00020FA04F001FA05F240EA020001F00042CB
:1006D00021F0004110EBD37021FA04F642EB060141
:1006E0005EEA430E08BF20EAD37070BDC4F10C046B
:1006F000C4F1200500FA04F320FA05F001FA04F22F
:1007000040EA020001F0004110EBD37041F100011A
:100710005EEA430E08BF20EAD37070BDC4F1200525
:1007200000FA05F24EEA020E20FA04F301FA05F28D
:1007300043EA020321FA04F001F0004121FA04F235
:1007400020EA020000EBD3705EEA430E08BF20EA05
:10075000D37070BD94F0000F0FD101F0004640003F
:1007600041EB010111F4801F08BF013CF7D041EAC1
:10077000060195F0000F18BF704703F000465200C5
:1007800043EB030313F4801F08BF013DF7D043EA96
:100790000603704794EA0C0F0CEA135518BF95EA4C
:1007A0000C0F0CD050EA410618BF52EA4306D1D1D3
:1007B00081EA030101F000414FF0000070BD50EAF2
:1007C000410606BF1046194652EA430619D094EA7C
:1007D0000C0F02D150EA013613D195EA0C0F05D166
:1007E00052EA03361CBF104619460AD181EA0301BA
:1007F00001F0004141F0FE4141F470014FF0000072
:1008000070BD41F0FE4141F4780170BD70B54FF00C
:10081000FF0C4CF4E06C1CEA11541DBF1CEA13558C
:1008200094EA0C0F95EA0C0F00F0A7F8A4EB05046E
:1008300081EA030E52EA03354FEA013100F0888065
:100840004FEA03334FF0805545EA131343EA12632E
:100850004FEA022245EA111545EA10654FEA0026E3
:100860000EF000419D4208BF964244F1FD0404F59C
:10087000407402D25B084FEA3202B61A65EB0305F8
:100880005B084FEA32024FF480104FF4002CB6EBB5
:10089000020E75EB030E22BFB61A754640EA0C0035
:1008A0005B084FEA3202B6EB020E75EB030E22BF75
:1008B000B61A754640EA5C005B084FEA3202B6EBB6
:1008C000020E75EB030E22BFB61A754640EA9C0075
:1008D0005B084FEA3202B6EB020E75EB030E22BF45
:1008E000B61A754640EADC0055EA060E18D04FEA03
:1008F000051545EA16754FEA06164FEAC30343EAA3
:1009000052734FEAC2025FEA1C1CC0D111F4801F6F
:100910000BD141EA00014FF000004FF0004CB6E768
:1009200011F4801F04BF01430020B4F1FD0C88BF07
:10093000BCF5E06F3FF6AFAEB5EB030C04BFB6EB12
:10094000020C5FEA500C50F1000041EB045170BD05
:100950000EF0004E4EEA113114EB5C04C2BFD4EB32
:100960000C0541EA045170BD41F480114FF0000EB6
:10097000013C90E645EA060E8DE60CEA135594EA32
:100980000C0F08BF95EA0C0F3FF43BAF94EA0C0F35
:100990000AD150EA01347FF434AF95EA0C0F7FF4AA
:1009A00025AF104619462CE795EA0C0F06D152EAFE
:1009B00003353FF4FDAE1046194622E750EA4106E2
:1009C00018BF52EA43067FF4C5AE50EA41047FF4F3
:1009D0000DAF52EA43057FF4EBAE12E74FF0FF3C58
:1009E00006E000BF4FF0010C02E000BF4FF0010C29
:1009F0004DF804CD4FEA410C7FEA6C5C4FEA430CA2
:100A000018BF7FEA6C5C1BD001B050EA410C0CBFF0
:100A100052EA430C91EA030F02BF90EA020F002052
:100A2000704710F1000F91EA030F58BF994208BFB9
:100A300090422CBFD8176FEAE37040F00100704776
:100A40004FEA410C7FEA6C5C02D150EA013C07D1CD
:100A50004FEA430C7FEA6C5CD6D152EA033CD3D018
:100A60005DF8040B704700BF8446104662468C4612
:100A70001946634600E000BF01B5FFF7B7FF002845
:100A800048BF10F1000F01BD4DF808EDFFF7F4FF6E
:100A90000CBF012000205DF808FB00BF4DF808EDF9
:100AA000FFF7EAFF34BF012000205DF808FB00BF1C
:100AB0004DF808EDFFF7E0FF94BF012000205DF83E
:100AC00008FB00BF4DF808EDFFF7CEFF94BF0120F3
:100AD00000205DF808FB00BF4DF808EDFFF7C4FFEC
:100AE00034BF012000205DF808FB00BF4FEA410C35
:100AF0007FEA6C5C02D150EA013C0AD14FEA430C18
:100B00007FEA6C5C02D152EA033C02D14FF0000054
:100B100070474FF0010070474FEA410212F5001292
:100B200015D211D56FF47873B3EB625212D94FEA34
:100B3000C12343F0004343EA505311F0004F23FA1E
:100B400002F018BF404270474FF00000704750EA73
:100B5000013005D111F0004008BF6FF00040704730
:100B60004FF00000704700BF4A0011D212F500128A
:100B700011D20DD56FF47873B3EB62520ED44FEAF5
:100B8000C12343F0004343EA505323FA02F0704775
:100B90004FF00000704750EA013002D14FF0FF30B3
:100BA00070474FF0000070474FEA4102B2F1E04356
:100BB00024BFB3F5001CDCF1FE5C0DD901F0004C44
:100BC0004FEAC0024CEA5070B2F1004F40EB830094
:100BD00008BF20F00100704711F0804F21D113F1C0
:100BE0003872BCBF01F00040704741F480114FEAF9
:100BF0005252C2F11802C2F1200C10FA0CF320FA82
:100C000002F018BF40F001004FEAC1234FEAD3239E
:100C100003FA0CFC40EA0C0023FA02F34FEA430308
:100C2000CCE77FEA625307D150EA01331EBF4FF091
:100C3000FE4040F44000704701F0004040F0FE40AC
:100C400040F40000704700BF80F0004002E000BFA9
:100C500081F0004142001FBF5FEA410392EA030FA7
:100C60007FEA226C7FEA236C6AD04FEA1262D2EBF1
:100C70001363C1BFD218414048404140B8BF5B42F6
:100C8000192B88BF704710F0004F40F4000020F08F
:100C90007F4018BF404211F0004F41F4000121F0A5
:100CA0007F4118BF494292EA030F3FD0A2F10102EF
:100CB00041FA03FC10EB0C00C3F1200301FA03F12D
:100CC00000F0004302D5494260EB4000B0F5000F50
:100CD00013D3B0F1807F06D340084FEA310102F10F
:100CE0000102FE2A51D2B1F1004F40EBC25008BFC1
:100CF00020F0010040EA03007047490040EB00008B
:100D0000013A28BFB0F5000FEDD2B0FA80FCACF18B
:100D1000080CB2EB0C0200FA0CF0AABF00EBC250B8
:100D200052421843BCBFD0401843704792F0000FA6
:100D300081F4000106BF80F400000132013BB5E7F9
:100D40004FEA41037FEA226C18BF7FEA236C21D06F
:100D500092EA030F04D092F0000F08BF08467047D4
:100D600090EA010F1CBF0020704712F07F4F04D1A2
:100D7000400028BF40F00040704712F100723CBFB5
:100D800000F50000704700F0004343F0FE4040F4DF
:100D9000000070477FEA226216BF08467FEA23639D
:100DA0000146420206BF5FEA412390EA010F40F488
:100DB000800070474FF0000304E000BF10F00043D4
:100DC00048BF40425FEA000C08BF704743F09643BB
:100DD00001464FF000001CE050EA010208BF7047D6
:100DE0004FF000030AE000BF50EA010208BF70475D
:100DF00011F0004302D5404261EB41015FEA010C72
:100E000002BF84460146002043F0B64308BFA3F169
:100E10008053A3F50003BCFA8CF2083AA3EBC2534B
:100E200010DB01FA02FC634400FA02FCC2F120026A
:100E3000BCF1004F20FA02F243EB020008BF20F0A1
:100E40000100704702F1200201FA02FCC2F1200207
:100E500050EA4C0021FA02F243EB020008BF20EAFC
:100E6000DC7070477BB972B90029BEBF00204FF01B
:100E7000004106E008BF00281CBF6FF000414FF0A2
:100E8000FF3000F007BAADF1080C6DE904CE00297F
:100E900009DB002B1ADB00F095F8DDF804E0DDE952
:100EA000022304B07047404261EB4101002B1BDB81
:100EB00000F088F8DDF804E0DDE9022304B04042E8
:100EC00061EB4101524263EB43037047524263EBD3
:100ED000430300F077F8DDF804E0DDE9022304B015
:100EE000404261EB41017047524263EB430300F023
:100EF00069F8DDF804E0DDE9022304B0524263EB57
:100F00004303704753B94AB9002908BF00281CBFE2
:100F10004FF0FF314FF0FF3000F0BCB9ADF1080CDD
:100F20006DE904CE00F04EF8DDF804E0DDE90223BF
:100F300004B07047430803F05533C01A830803F028
:100F4000333300F03330184400EB101000F00F3052
:100F500000EB002000EB0040000E704707EE900A07
:100F6000F5EEC07AF1EE10FA01D400F00BB8F1EE14
:100F7000677A08B517EE900A00F004F8404261EB7A
:100F8000410108BDD0B5FFF7BFFA0C4B0022064661
:100F90000F46FFF711FBFFF7E7FD0446FFF792FA54
:100FA000074B0022FFF708FB02460B463046394646
:100FB000FFF74AF9FFF7D8FD2146D0BD0000F03D0C
:100FC0000000F0412DE9F047089D04468E46002BB5
:100FD0004DD18A42944669D9B2FA82F252B101FAED
:100FE00002F3C2F1200120FA01F10CFA02FC41EAFD
:100FF000030E94404FEA1C48210CBEFBF8F61FFA82
:101000008CF708FB16E341EA034306FB07F199421C
:101010000AD91CEB030306F1FF3080F01F819942CF
:1010200040F21C81023E63445B1AA4B2B3FBF8F0A9
:1010300008FB103344EA034400FB07F7A7420AD930
:101040001CEB040400F1FF3380F00A81A74240F258
:1010500007816444023840EA0640E41B00261DB1C3
:10106000D4400023C5E900433146BDE8F0878B42F8
:1010700009D9002D00F0EF800026C5E900013046B7
:101080003146BDE8F087B3FA83F6002E4AD18B4291
:1010900002D3824200F2F980841A61EB030301203B
:1010A0009E46002DE0D0C5E9004EDDE702B9FFDE27
:1010B000B2FA82F2002A40F09280A1EB0C014FEAD2
:1010C0001C471FFA8CFE0126200CB1FBF7F307FB2F
:1010D000131140EA01410EFB03F0884208D91CEBD2
:1010E000010103F1FF3802D2884200F2CB8043466F
:1010F000091AA4B2B1FBF7F007FB101144EA01444E
:101100000EFB00FEA64508D91CEB040400F1FF31DC
:1011100002D2A64500F2BB800846A4EB0E0440EACA
:1011200003409CE7C6F12007B34022FA07FC4CEAD3
:10113000030C20FA07F401FA06F31C43F9404FEAC6
:101140001C4900FA06F3B1FBF9F8200C1FFA8CFEDB
:1011500009FB181140EA014108FB0EF0884202FA2F
:1011600006F20BD91CEB010108F1FF3A80F08880F0
:10117000884240F28580A8F102086144091AA4B2AD
:10118000B1FBF9F009FB101144EA014100FB0EFE2E
:101190008E4508D91CEB010100F1FF346CD28E455D
:1011A0006AD90238614440EA0840A0FB0294A1EBEE
:1011B0000E01A142C846A64656D353D05DB1B3EB4B
:1011C000080261EB0E0101FA07F722FA06F3F1407B
:1011D0001F43C5E9007100263146BDE8F087C2F122
:1011E0002003D8400CFA02FC21FA03F3914001439A
:1011F0004FEA1C471FFA8CFEB3FBF7F007FB1036D3
:101200000B0C43EA064300FB0EF69E4204FA02F47E
:1012100008D91CEB030300F1FF382FD29E422DD9D1
:10122000023863449B1B89B2B3FBF7F607FB163306
:1012300041EA034106FB0EF38B4208D91CEB010186
:1012400006F1FF3816D28B4214D9023E6144C91A06
:1012500046EA004638E72E46284605E70646E3E616
:101260001846F8E64B45A9D2B9EB020864EB0C0E20
:101270000138A3E74646EAE7204694E74046D1E72F
:10128000D0467BE7023B614432E7304609E76444DD
:10129000023842E7704700BF02E000F000F8FEE7C6
:1012A00072B6374880F30888364880F30988364894
:1012B0003649086040F20000CCF200004EF634716E
:1012C000CEF200010860BFF34F8FBFF36F8F40F283
:1012D0000000C0F2F0004EF68851CEF20001086026
:1012E000BFF34F8FBFF36F8F4FF00000E1EE100A96
:1012F0004EF63C71CEF200010860062080F314889F
:10130000BFF36F8F9CF0C4FE9BF05EFF4FF0553033
:101310001F491B4A91423CBF41F8040BFAE71D49A3
:10132000184A91423CBF41F8040BFAE71A491B4A9C
:101330001B4B9A423EBF51F8040B42F8040BF8E7EE
:1013400000201849184A91423CBF41F8040BFAE7C3
:101350009CF0A2FE9BF08CFF144C154DAC4203DABE
:1013600054F8041B8847F9E700F0D4FB114C124DE8
:10137000AC4203DA54F8041B8847F9E79CF08ABEB4
:1013800000060020002200200000010808ED00E017
:101390000000002000060020001F0D080022002091
:1013A0009C250020A0250020C0410120E00101086B
:1013B0003802010838020108380201082DE9F04F0F
:1013C0002DED108AC1F80CD0C3689D46BDEC108A83
:1013D000BDE8F08F002383F311882846A047002042
:1013E0009BF078FCFEE79BF0FDFA00DFFEE70000D3
:1013F00001F0FF01102A2BDB10F0070F08D010F8C6
:10140000013B013A8B422DD010F0070F42B3F6D1C9
:10141000F0B441EA012141EA014122F007047FF0E2
:1014200000070023F0E80256083C85EA010586EA39
:10143000010685FA47F5A3FA87F586FA47F6A5FA75
:1014400087F68EB9EED1F0BC01F0FF0102F0070281
:1014500032B110F8013B013A83EA010313B1F8D12C
:101460000020704701387047002D06BF354603380D
:10147000073815F0010F07D1013015F4807F02BF46
:10148000013015F4C03F0130F0BC0138704700BF97
:1014900010F8012B11F8013B012A28BF9A42F7D01E
:1014A000D01A7047034613F8012B002AFBD1181AF3
:1014B0000138704738B50022002304460D46FFF777
:1014C000EDFA28B920462946BDE8384000F00AB8B0
:1014D000204605F1004100F005F8404261EB410172
:1014E00038BD00BFD0B50C4B002206460F46FFF7B3
:1014F00063F8FFF739FB0446FEF7E4FF074B0022D1
:10150000FFF75AF802460B4630463946FEF79CFE76
:10151000FFF72AFB2146D0BD0000F03D0000F0415E
:101520001FB5094BD3F8B0280092D3F8B428019224
:10153000D3F8B8280292D3F8BC3803936A4671F006
:1015400015FD05B05DF804FBB045002008B5064860
:10155000022104F093F928B9BDE8084002480421AB
:1015600004F08CB908BD00BFB025002037B5847FDA
:101570000191054644B9FFF7E9FF0199044630B9E6
:10158000064A284670F074FF204603B030BD284656
:1015900003B0BDE8304071F04FBD00BF5C630B0885
:1015A000F0B591B005460E4670F002FF0446D8B182
:1015B0001021284670F00CFDB0B100212E2204A8A5
:1015C00003AF0391A0F0CEFC0CF096F932233A461B
:1015D00000210BF059FD044630B9054B0097324607
:1015E0001021284670F0FCFC204611B0F0BD00BF71
:1015F00088630B08F8B5384F3B780646002B69D155
:1016000001253D7071F0D2FD044630B9334A38707F
:1016100013782B4313702046F8BD47F0F3FC29469E
:1016200046F0DCFC2E4803F0F3FA2E4B1D710B251F
:101630003AF03EFA013D3AF0D9F915F0FF05F7D13D
:101640000CF05AF9284BD0F8F821C3F8F42090F8A0
:101650007422D10706D5920704D42946A3F5405039
:1016600002F09AFD214B224D1B68D86A03680121C4
:101670001B6898471A4808F0B7FC01211D486EF016
:101680002FFE47F0BFFC2A7F95F8801D46F082FEB2
:10169000A5F5005003F0AEFA43F0D0FD43F022F977
:1016A0000023A5F500503B7000F0C6F90028B2D128
:1016B00050F09AFF0421104A4AF06CFD2021304678
:1016C00070F086FC0028A6D00C4B01222021304669
:1016D00070F086FC00249EE7A02500206C7B002093
:1016E000B02500204D7B0020B0550020A82500200B
:1016F000B04500205853002094630B08B1630B08D9
:10170000F0B5234B93F87B3E87B01BB900242046ED
:1017100007B0F0BD71F00EFE04460028F6D00CF0C4
:10172000EBF806460AF0B0FFD0B114F0D1FF90F903
:101730002430022B14D100250027E9B203AA304639
:1017400003970497059701910BF03AFB28B114F029
:10175000BFFF019903AA14F0C7FC0135032DECD19A
:1017600000210C486EF0BCFD0B4824F009F847F04E
:1017700049FC002146F032FC084B1B68D86A03681C
:1017800000211B689847064804F066F8BFE700BFD1
:10179000B04500205853002034500020A8250020D8
:1017A000B025002009F068B954F08CBC43F092BC1D
:1017B0001CF08EBF46F094BD0FF08CBC52F0AEB85A
:1017C00050F0ECB90EF082BB09F07AB908F02CBEEB
:1017D00018F07AB908F024BF02F00ABD04F0AEBFD9
:1017E00000F066BB03F040BE08F0FEBC1DF03ABA44
:1017F000034808601D21117008221A60704700BF5D
:101800009C660B0810B5044603F066FC204603F006
:1018100027FD204603F0C0FB204603F069FB52F091
:10182000A5FB52F0B7FA04F521502430BDE8104072
:1018300002F086BBFFF7E6BF38B5044600F544501A
:1018400008300FF017F814F043FF90F92130F3B18E
:1018500090F84033DBB104F537502C304AF016F8DD
:10186000034693ED000ADFED0A0A9E20B7EE001A48
:101870001EF0FAFE94F9C83504F29455012B08BF06
:1018800085ED0E0A2846BDE8384014F031BE38BD5B
:1018900000000000FFF7D0BF13B50121044609F096
:1018A000D3F8A8B3204601F0BFFC04F56C5304F54F
:1018B0005C5204F5365104F5595028312C302C3344
:1018C00028320AF0A3F94FF48051204609F0BCF801
:1018D000F0B104F5235004F5635208303432652129
:1018E000019046F0CBF904F5675201982032662149
:1018F00046F0C4F904F56B5201980C32672146F0AA
:10190000BDF904F5775201982032682146F0B6F906
:101910008021204609F098F860B14FF4002120465C
:1019200009F092F830B91EF0BDF902B0BDE81040E0
:101930001CF0A0BB02B010BDFFF7AEBF10B504464F
:1019400000F5275018306DF09BFC204603F0F8F9A5
:10195000204603F063F9204603F0A8F9204603F07F
:1019600009FC204603F028FD204603F05DFD04F548
:101970008C500430BDE8104056F0B4BBFFF7DEBF1A
:1019800010B5044600F58F50083001210BF04AFFD6
:1019900004F559502C30BDE810400AF03DBA000063
:1019A000FFF7EEBF10B5044608F0F4FC1021204606
:1019B00009F04AF840B1204601F086FB1EF072F9AA
:1019C000BDE810401CF048BC10BD0000FFF7EABFA6
:1019D00010B500F5005292F87D3D13F0010408D1D6
:1019E000084A00F52D50383004214AF0D3FB00207E
:1019F00010BD92F8A13DDB0701D5034AF1E70120B4
:101A0000F6E700BF1C640B083B640B0800230B6067
:101A10000120704710B500F5005300F50454183448
:101A2000204693F87B1E61F0ABFC2046BDE81040D9
:101A300061F046BCFFF7EEBF70B505468AB005F50C
:101A40008F5602A8083611F011FA02A930460BF0A1
:101A50008DFD044688BB05F5887016F045F960BB1E
:101A6000254ADFED267AD2ED006A12ED017A9FED6C
:101A7000246A66EEA76A52ED027A009427EE067A8F
:101A800067EE867AFDEEE66ABDEEC77AFDEEE77A8E
:101A900016EE903A17EE102A17EE901A06A811F0DB
:101AA00005FA089805F52D55383508B1099939B961
:101AB000144A042128464AF06DFB20460AB070BD46
:101AC0001FF00CF8044608B90F4AF2E706A93046A1
:101AD0000AF048FE044608B90C4AEAE70C4A062117
:101AE00028464AF057FB30460CF0E6F842212846DB
:101AF00051F028F9E1E700BF104E00200000C84275
:101B00008096184B50640B087F640B08A8640B0880
:101B1000D7640B0838B5054B1C6823680A461D6856
:101B2000034B01462046A847002038BDA8250020C9
:101B3000B025002010B5044643F080FB04F50051A9
:101B400001F6A853426FDA6004F5405303F5E560EF
:101B500003F62C334264C3F8082391F8803D133B0D
:101B6000012B06D904F55C502830BDE8104068F020
:101B70001BBC10BDFFF7DEBF37B50221044608F0DD
:101B800063FFD0B30121204608F05EFFA8BB2046CA
:101B900001F04AFB04F56C5304F55C5204F5365130
:101BA00004F5595028312C302C3328320AF02EF805
:101BB0004FF48051204608F047FFF0B104F5235060
:101BC00004F56352083034326521019046F056F82E
:101BD00004F5675201982032662146F04FF804F56B
:101BE0006B5201980C32672146F048F804F57752A1
:101BF00001982032682146F041F84FF40031204628
:101C000008F022FF20B104F5365028306FF0B2FB07
:101C10004021204608F018FF20B104F52350083079
:101C200045F0FEFC4FF48061204608F00DFF20B126
:101C300004F52350083045F08DFD2021204608F0A2
:101C400003FF58B11D4DD5F8B00103689B68984754
:101C5000D0B104F56C502C306BF026F88021204672
:101C600008F0F2FEC0B11EF01DF81CF027FA10219A
:101C7000204608F0E9FEF0B104F55C50283003B0CE
:101C8000BDE8304068F090BCD5F8B0010368DB686F
:101C900098470028DDD0E1E74FF48021204608F086
:101CA000D3FE0028DFD14FF40021204608F0CCFEFF
:101CB0000028D8D1DBE703B030BD00BFB0750020ED
:101CC000FFF75ABF70B5044600F55750002104F5E0
:101CD00000550830FFF74AFC95F87C3D224E60F332
:101CE000000385F87C3DB071204608F097FE95F81A
:101CF0007B3EF0714FF6FF712046737108F0A4FE31
:101D000028B1D5F87C2D0721204601F0BBFA95F8C3
:101D10007B3E23B904F5365028306FF003FD53F0B5
:101D2000A5FC204608F0BEFE104B1B68DB6A93F84A
:101D30009C6026B1AB7F13B972F098FF2862AE7732
:101D400043F07CFA42F0F6FE04F55C50283068F06F
:101D500097F843F073FA42F0EDFE04F57550083041
:101D6000BDE8704060F0E4BB4D7B0020A82500205A
:101D7000FFF7A8BF10B506480C466CF0ADF8DFEDD4
:101D8000057A20EE270A012084ED000A10BD00BF6D
:101D90008C6400200AD7233C10B508480C466CF030
:101DA000AFF807EE900A9FED067AF8EEE77A012089
:101DB00067EE877AC4ED007A10BD00BF8C64002006
:101DC0000AD7233C70B52DED048B00F5005482B08A
:101DD0000E4615464FF47A714FF4FA52B4F95C008E
:101DE0008DED011AF0EE408AB0EE608A1EF07AFCAA
:101DF000034607EE903ADFED240AA4F85C00B8EE43
:101E0000E71A0B209DED010ADFED209A1EF02CFC55
:101E1000B4F95C30DFED1E6A07EE103AB8EEC77A0F
:101E2000B0EE409AC7EE267A67EEA88A27EE888A37
:101E300028EEA80AA8EE080A9DF0C6FFB4EEC09AE4
:101E4000F1EE10FA42BFC9EE007A28EE278A68EE5A
:101E5000A78A28EE290A9DF04BFCB0EE409A28EEA6
:101E6000A90A9DF0D5FD29EE000A9DF021FBDFEDCA
:101E7000097A20EE270A86ED000A85ED008A02B075
:101E8000BDEC048B70BD00BF00007A44D40237392A
:101E900000A08C459F0CB34507EE901A00F500504A
:101EA000F8EEE77A90ED3F0A27EE800A70470000CF
:101EB00073B5044600F58F5001A9083004F50056AB
:101EC0000BF040F9D6F8743B8342054606D004F582
:101ED0005C50283069F0ACFBC6F8745B02B070BD92
:101EE00038B5104A13780133DBB2032B044600F5F2
:101EF000405505D8137005F2346595ED000A38BDDC
:101F000000F559500023103013706DF049F904F5B5
:101F1000585128311EF060FD05F2346383ED000A4C
:101F2000E9E700BFA125002038B5044600F5595067
:101F30002DED028B10306DF039F905461FF022FFB0
:101F40002046B0EE408A08F069FD04F54054C0B167
:101F5000DFED0F7AB4EEE78AF1EE10FA11DDD5ED80
:101F6000000A95ED010A9DF0E5FDDFED0A7A20EE0D
:101F7000270ADFED097A20EE270A04F2446383ED95
:101F8000000ABDEC028B04F2446494ED000A38BDF3
:101F900000401C46E02E65420000C84200F580501B
:101FA00000F5866300F23C40D3ED005AD2ED007A92
:101FB000D0ED006A91ED006A26EEE77A67EEA57A29
:101FC000A6EE257AE6EE267A81ED007AC2ED007A59
:101FD0007047000000F50050B0F98A3033B9B0F90D
:101FE00088000028B8BF404280B2704783EAE3709F
:101FF000A0EBE370F8E7000070B52DED068B00F55F
:10200000005482B094F8A01D8DED010A11F0010179
:102010000546009162D1D4F8B8089FED329A51F08C
:10202000FFFFB4F98E30DFED300A9DED010A07EEB7
:10203000900A08EE103A05F5405606F20C63F8EEE9
:10204000E79AB8EEC88AD3ED007A6720B0EE491A55
:1020500028EE278A1EF008FB39EEC8AA0099B4F9C9
:102060008E004FF4C872F0EE408A1EF03BFBB4EED7
:10207000E8AAF1EE10FAA4F88E0016DD2846FFF764
:10208000A9FF07EE900A78EECA8AB8EEE70A60EE7A
:10209000288A88EE8A0AFDEEC07A17EE903AA6F8F2
:1020A000F83002B0BDEC068B70BD78EE297AF4EE04
:1020B000E87AF1EE10FA49BFB4F988309FED0A0AC8
:1020C00000EE103A78EEE78A41BFB8EEC00A79EE2A
:1020D000677A60EE288A88EEA70ADCE79FED020A9D
:1020E000DFE700BF00007A440000000000207047D6
:1020F00070470000704700007047000000207047E4
:102100000020704700207047012070477047000092
:102110007047000070470000002070470C4991F89C
:10212000803D102B0FD801229A400A4B1340002B00
:102130000CBF1020182091F87B3E33B940F04000CE
:1021400040F0010070471020F5E740F0C000F7E7CD
:10215000B045002098000100014B93F864007047DF
:10216000B04500207047000010B504464DF07CF9E2
:1021700005486EF093F9054A034606212046BDE85E
:1021800010404DF059B900BF58530020E8680B08C3
:1021900000B513EE103A8DB06222CDF8253013EE63
:1021A000903ACDF829302123CDE900328DF8241062
:1021B000192303AAC2218DED030ACDED040A8DED8A
:1021C000051ACDED061A8DED072ACDED082A4AF045
:1021D000DDFF0DB05DF804FB08B50B4849F056FB78
:1021E0000346DFED0A0A93ED000A9E20B7EE001ABF
:1021F0001EF03AFADFED067A20EE270ABDEEC00A9D
:1022000010EE103A18B208BD9C53002000000000E8
:102210000000C8424DF0E6BEF8B5704E04460BF023
:102220006BFBB6F89C300546D80736D56C4BDFED16
:102230006D7AD3ED002A13ED012A9FED6B7AD5ED6F
:10224000C30A207C06F5C853D3ED001A93ED031A98
:1022500013ED030AD3ED053A93ED063A62EEA72A91
:1022600022EE272A61EEA71A21EE271A60EE870ACE
:1022700020EE270A0121FFF78BFF207C4AF01CFF8C
:102280000746207C4BF024FE00F121039F4204D23C
:10229000207CBDE8F8404AF065B9B6F89C30990753
:1022A0002FD5524BDFED4F7A53ED032A13ED042A5D
:1022B00053ED051A13ED021A13ED080A9FED4A7A41
:1022C000D5EDC40AD3ED003A93ED013A207C62EEDD
:1022D000A72A22EE272A61EEA71A21EE271A60EE1E
:1022E000870A20EE270A0221FFF752FF207C4AF0DE
:1022F000E3FE0746207C4BF0EBFD00F121039F42FB
:10230000C6D3B6F89C305A072FD5394BDFED357A56
:1023100053ED032A13ED042A53ED051A13ED021AA7
:1023200013ED080A9FED307AD5EDC50AD3ED003ADA
:1023300093ED013A207C62EEA72A22EE272A61EE75
:10234000A71A21EE271A60EE870A20EE270A03213A
:10235000FFF71EFF207C4AF0AFFE0746207C4BF0C3
:10236000B7FD00F121039F4292D3B6F89C301B07C2
:1023700032D5204B9FED207AD5EDD40ADFED197AC6
:1023800053ED032A13ED042A53ED051A13ED021A37
:1023900013ED080AD3ED003A93ED013A207C70EE7C
:1023A000870A62EEA72A22EE272A61EEA71A21EEFB
:1023B000271A20EE270AF1EE600A0421FFF7E8FE53
:1023C000207C4AF079FE0546207C4BF081FD00F12F
:1023D00021039D42FFF45CAFF8BD00BFB045002073
:1023E000B85E00200AD7233CE02E6542B05F002093
:1023F0009C600020B06300200AE81C41014802F004
:1024000043BA00BFB025002007B50846019110F07F
:1024100021FE38B10448019905F05AF8002003B0B4
:102420005DF804FB0420FAE754780020014801F02D
:10243000B3BE00BFB0250020014801F067BE00BF59
:10244000B025002038B5C5780B46352D044628BF89
:1024500035253522002118469FF084FD2A4604F1D7
:102460000C01BDE838409FF033BD00002DE9F04776
:102470002DED028B8A7A4B7A43EA0223CA7A43EA29
:102480000243522BA2B005460C4600F0568111D8EB
:10249000452B00F0E680462B00F03C81012B00F03C
:1024A00066822146284622B0BDEC028BBDE8F0478B
:1024B00050F012BD562B00F0DE8100F2C080542B8C
:1024C000EFD114A92046FFF7BDFFAE4B93F8802D46
:1024D000042A09D0032A40F0188103F5405393F8E9
:1024E0005434032B40F011819DF884200C2A00F213
:1024F0000C8141F28234D440E44314F0010440F0F2
:102500000481BDF88030002613F0070703F0380A75
:1025100003F4E07903F4806803F400650D960E96E9
:102520000F962CD19FED986A9DED167ADDED177A06
:10253000DDED156A27EE067A67EEC67A66EE866AE4
:10254000A2F10803012BCDED0D6A8DED0E7ACDEDD4
:102550000F7A01D90C2A04D18C480EAA0DA9FFF7D5
:102560001DFD9DF88430DA1F022A01D90C2B06D1FB
:1025700087486CF013FE01460DA820F0E1FB109691
:1025800011961296BAF1000F20D19FED7F6A9DED52
:10259000197ADDED1A7ADDED186A9DF8843027EEA0
:1025A000067A67EEC67A66EE866AA3F10802012A09
:1025B000CDED106A8DED117ACDED127A01D90C2B8B
:1025C00004D1724811AA10A9FFF7E8FCB8F1000F76
:1025D00040F02781DFED6F7A9DED1E0A9DF8844063
:1025E00020EE270ADFED687AA4F10906744220EE96
:1025F000270A7441002D40F01781DFED667ADDED8A
:102600001F0A60EEA70ADFED607A60EEA70A002FCE
:1026100040F00D81BAF1000F40F01D81B9F1000FBB
:1026200073D0B5FA85F56D09B8FA88F30194009571
:102630005B0910AA0DA9584805F05EFE65E003F19C
:102640008073863B23F07F43012B3FF62AAF0A4677
:10265000017C524822B0BDEC028BBDE8F04743F04C
:102660001BBB484DCA79B5F964309A424DD1CE783A
:102670001E2E28BF1E261E22002114A89FF072FCC9
:10268000324604F10C0114A89FF022FC9DF85A2058
:10269000B5F962309A4238D1BDF96C300B93BDF96F
:1026A0006A300A93BDF968300993BDF96630089322
:1026B000BDF964300793BDF962300693BDF960300F
:1026C0000593BDF95E3004939DF85D300393BDF82A
:1026D0005B300293BDF858300193BDF95630BDF917
:1026E0005220BDF950100093A5F50050BDF95430AB
:1026F00003F0DEFD72F0BAFAC5F88C0D4FF074FFEE
:10270000044672F0B3FAC4F8940122B0BDEC028B17
:10271000BDE8F0871B4ECA79B6F964309A42F4D10D
:1027200072F0A4FA2146C6F88C0D284622B0BDEC02
:10273000028BBDE8F0474EF019BCCD78272D28BF9D
:1027400027252722002114A89FF00CFC2A4604F11B
:102750000C0114A89FF0BCFB9DF876305F0623D5D2
:1027600072F084FA0E4D14ACC5F86C010FCC05F56F
:10277000B8750FC50FCC0FC594E8030085E80300BA
:10278000C3E700BFB04500200000C842B0250020CC
:10279000005C0020E02E654290780020806E0020D2
:1027A000B07500200000000013F0C00FADD15FED48
:1027B000030A9DED1C0A40F28A20B7EE001A1DF0B4
:1027C00053FFF6EE000AB0EE408A1DF073FE28BB00
:1027D000B6EE007A854BB4EEC78AF1EE10FA78EEC9
:1027E000477ADABF03F6FC6393ED000A03F6F86359
:1027F00077EEA77ACCBF93ED000AB0EEC00A20EEC8
:10280000270A159B1093169B1193179B12937848D8
:10281000189B139310A905F037FE76E79FED750A14
:10282000EFE79FED740AE5E6DFED720AEFE6BAF135
:10283000000F7FF46AAFB9F1000F3FF466AFB5FA4D
:1028400085F3B8FA88F26A4800945B09520910A926
:1028500005F082FC59E7B9F1000F3FF456AFB5FA25
:1028600085F3B8FA88F200945B0952090DA9604813
:1028700006F040FA49E714A92046FFF7E3FD5E4A57
:1028800092F8803D042B08D0032B1CD102F5405256
:1028900092F85424032A7FF438AFBDF88020500703
:1028A00002F0070102F0380602F4E0740DD4022BA6
:1028B0000BD1DDED177A9FED517A514B67EE877A98
:1028C000C3ED007A21E7022BE5E700230D930E9379
:1028D0000F9300296AD1DDE915011EF0FFF80028E9
:1028E0003FF413AF9DF884100CAA28464FF004FA69
:1028F00000283FF40AAFDDED177A9FED408A0C9B6C
:10290000009367EE887ADDE91512FDEEE77A10A8EC
:1029100017EE903A10F0CAFA0DA910A810F028FC92
:1029200000283FF4F2AED6B9002C3FF4EEAEDDED58
:10293000186A9DED197ADDED1A7A2D4866EE886ADF
:1029400027EE087A27EEC88A10AA0DA9CDED106AE5
:102950008DED117A8DED128A05F062FCD5E6002C22
:102960003FF4D3AE0DA9224806F08EF9CDE6CD781E
:102970001F2D28BF1F251F22002114A89FF0F2FA47
:102980002A4604F10C0114A89FF0A2FA159B9A00A4
:102990007FF5BBAE169B9B003FF5B7AE194822B042
:1029A000BDEC028BBDE8F0476CF088BC002E7FF4D4
:1029B000ACAE002C3FF4A9AE9FED106ADDED186AB5
:1029C0009DED197ADDED1A7A094866EE866A27EEE2
:1029D000067A67EEC67A10A9CDED106A8DED117AF0
:1029E000CDED127A05F09EFB8FE600BFB0550020BA
:1029F0009078002000000000B04500200000C84290
:102A000028640020884F002010B5074B93F9D02888
:102A100040F6C53440F6C513002A08BF1C464BF0EB
:102A200025FE204310BD00BFB0650020044B93F885
:102A30007D3D13F0010301D04BF084BC1846704774
:102A4000B0450020044B93F87D3D13F0010301D005
:102A50004BF0F6BF18467047B045002010B504464D
:102A600010F018FD204610BD08B54B69012B03D0AE
:102A7000BDE808404BF0E0BE4FF0B6FD024A06212B
:102A800049F088FB032008BDF4680B0810B50C481A
:102A900090F87B4E3CB14FF0A7FD0A4A062149F061
:102AA00079FB04200BE0A0F50050FEF791FF002811
:102AB000F7D00DF059FA01210DF0FCF8204610BDB9
:102AC000B04500201C690B08094B93F8C52562B975
:102AD000A3F5805393F8A02D120706D193F87B3EFF
:102AE000002B0CBF0320042070470520704700BF57
:102AF000B05500200C207047014B93F8800D7047B3
:102B0000B045002038B512212DED028B044649F066
:102B10003BFD20B90025BDEC028B284638BD0720BF
:102B200052F062FEB6EE008AF0EE487AE0EE087AE5
:102B30004B49F7EE008A204638EEE70A4DF098FC44
:102B40001221204649F020FD0028E3D0062052F053
:102B50004BFEF0EE487AE0EE087A4249204638EE25
:102B6000E70A4DF085FC1221204649F00DFD0028B2
:102B7000D0D03D4D3D49D5F80436002BB8BF0333C6
:102B80009B1000EE103A2046B8EEC00A4DF070FCE3
:102B90001221204649F0F8FC0028BBD0B52052F0A5
:102BA00023FEF0EE487AE0EE087A31492046B0EE96
:102BB000670A4DF05DFC1221204649F0E5FC002833
:102BC000A8D03C2052F010FEA0EE088A29492046E9
:102BD000B0EE480A4DF04CFC1221204649F0D4FCDE
:102BE000002897D005F20C63234993ED000A204694
:102BF0004DF03EFC1221204649F0C6FC002889D049
:102C000095F810361D4900EE103A2046B8EE400AFD
:102C10004DF02EFC1221204649F0B6FC00283FF46E
:102C200079AF95F81136164900EE103A2046B8EE05
:102C3000400A4DF01DFC1221204649F0A5FC054636
:102C400000283FF467AF0F4BDFED0F7A93ED000ADA
:102C50000E4980EE270A20464DF00AFC5BE700BFD4
:102C600038690B0840690B08B055002047690B080C
:102C700051690B0859690B0861690B086B690B08EE
:102C800075690B08F87900200000C8427F690B08BD
:102C9000272938B5054606D044290FD1FFF732FF62
:102CA0000124204638BD122149F06EFC044600285C
:102CB000F7D0297C034842F0F5FEF2E7BDE8384042
:102CC0004FF0ECB9806E0020024B93F87C0DC0F3FE
:102CD00000107047B045002008B5022210210448BA
:102CE00003F054FD00280CBF0420002008BD00BFE5
:102CF000B025002008B502220921044803F046FD52
:102D000000280CBF0420002008BD00BFB025002013
:102D100013B5D1ED007AF5EEC07AF1EE10FA0C465B
:102D200002DA022002B010BD9FED187AF4EEC77AE5
:102D3000F1EE10FAF5D891ED030ADFED157AB0EE59
:102D4000C07AB4EEE77AF1EE10FA18D5D4ED037A32
:102D50001048D4ED010A94ED000AFCEEE77ACDEDBF
:102D6000007AD4ED027A9DF80020FDEEE77ACDEDF1
:102D7000017A9DF9041004F037FB0020D2E7F7EE4A
:102D8000000A1DF097FB0028CBD0DFE70000B4431A
:102D9000000000345478002008B5D1ED017AF5EE3A
:102DA000C07AF1EE10FA08DD9FED050A054827EE1E
:102DB000800A6BF0D7F9002008BD0420FCE700BFB3
:102DC0000000C8428C64002008B5084890F87B3E9B
:102DD0000BB9042008BD02220321A0F5005003F026
:102DE000D5FC0028F5D00020F4E700BFB045002056
:102DF00070B501F10C050E460FCD86B06C460FC4C0
:102E000095E8030084E8030096E80E00044807F004
:102E100035F900280CBF0420002006B070BD00BFAB
:102E2000B025002030B48B8BB22B05460C4616D053
:102E30000AD8152B1CD0732B0ED0112B15D0214680
:102E4000284630BC50F094BAD12B0BD0B3F5967F06
:102E5000F5D130BCFFF7B8BF30BCFFF759BF30BC6D
:102E6000FFF79ABF30BCFFF7C3BF30BCFFF734BFDA
:102E700030BCFFF73FBF000070B52DED068B9FED16
:102E80002F0ADFED2F8A8CB004462E481FF038FF42
:102E900021EE281A2C48267CBDEEC11A60EEA89AB5
:102EA00011EE103A20EE28AA1DB26BF029F807EEB9
:102EB000900AF8EEE77A244867EEA87AFDEEE77A02
:102EC00017EE903A1CB26BF007F8DFED207A204B3A
:102ED00020EE288A03F67862B4EEE78AF1EE10FA63
:102EE000D3F8340B92ED009A58BFB0EE678A6CF0BD
:102EF00059F9BCEEC88A002339EE400A08930993B9
:102F000018EE103A60EE288AADF82C30B7221A235A
:102F1000CDE900323E2105AA30468DED05AACDED62
:102F2000069ACDED078AADF82850ADF82A404AF050
:102F30002DF90CB0BDEC068B70BD00BF9F0CB345E6
:102F40000AD7233C205D00208C64002000FF7F47CF
:102F5000B055002008B591ED007AF6EE007AB4EE97
:102F6000E77AF1EE10FA06DD044801220521FEF7AA
:102F7000C7FB002008BD0420FCE700BF785B0020F1
:102F800000207047002070470020704701207047E4
:102F900090F878308B4286BF00EB8100C06F002034
:102FA0007047000090F878308B4286BF00EB8100BC
:102FB000C06F002070470000FA207047014B93F863
:102FC00062007047B045002038B50446D0E90230B1
:102FD000216940F4E052E26041F4E052226143F49E
:102FE000F842A2602B4A92F8805D023D0E2D0FD868
:102FF000DFE805F00808080E0E080E080E0E0E0E8B
:103000000E0E080040F4F84041F4F841E060216100
:1030100092F87D1DC80708D543F4F84343F0080330
:10302000A360E36843F00803E360236923F0080327
:10303000236192F8A41DC90744BF43F0080323612C
:10304000154B93F86831013B012B0BD8A36843F46F
:103050008003A360E36843F48003E360236943F4DF
:103060008003236192F8FC39DB0712D50B4B1868FB
:10307000A36843F48073A360E36843F48073E36060
:1030800038B119213CF062FD18B1236943F4807313
:10309000236138BDB0450020B0750020F07B0020D2
:1030A00013B54FF45070CDE9002110F0EDF904464E
:1030B00028B1DDE900214FF0A9FA024B2360204638
:1030C00002B010BD006B0B08F0B52DED028B8FB078
:1030D0000023009300F580439FED508A93F9D03888
:1030E000044600F50056002B00F08F8000F591405B
:1030F00001226946503043F043FB3322002101A8EE
:103100009EF030FFA3238DF8043095238DF8053011
:1031100071F0B4FD04F5405505F5E563CDF8070001
:1031200004F53750D3F8B820D3F8BC30CDF80B10E5
:103130002C30CDF80F20CDF8133048F0A7FB034614
:10314000DFED370A93ED000A9E20B7EE001A1DF05E
:103150008BFA10EE103ACDF8173006F6D463B6EEBF
:10316000061AF4EE000A05F62C3793ED000A30201B
:103170001DF07AFA97EDD37ADFED2A7AC7EE277A37
:1031800004F55950103010EE103ACDF81B3017EE00
:10319000903ACDF81F306CF005F820EE080A94F84C
:1031A000792410EE103A2421CDF8233004F58D63F4
:1031B00001FB023304F52350DB6ACDF8273004F518
:1031C000A843D3ED127AFDEEE77A332217EE903A58
:1031D000D7EDD97AADF82B30FDEEE77AB6F8FE39A7
:1031E000ADF82D30009BCDF82F3017EE903A01A9A5
:1031F000ADF833300830B5F80036ADF8353044F06E
:1032000009FF0FB0BDEC028BF0BD06F60C23D3ED29
:10321000007A67EE887ACDED007A6EE70AD7233C14
:10322000000000000000C84230B5044600F55D50C3
:103230008BB09FED130A30301FF062FD0AAACDED6E
:10324000080A8DED091A8DED070A12E9070001AD94
:1032500085E8070004AB9DED030A83E807001DF035
:1032600097F904F58F50294608308DED030A08F0D0
:10327000DDFB0AF041FB0AF015F90BB030BD00BFD1
:103280009F0CB3457FB50E464FF6FF7104461546B9
:1032900007F0DAFBE8B11022002168469EF062FEDA
:1032A000A3238DF8003095238DF8013004238DF889
:1032B000023071F0E3FCCDF8030004F52350CDF8A3
:1032C00007101022694608308DF80B60039544F012
:1032D00021FF04B070BD0000F0B58BB01546064666
:1032E0000F462422002101A81C469EF03BFEA3238A
:1032F0008DF8043095238DF8053006238DF80630BF
:1033000071F0BCFC2B6804936B680593AB68069363
:103310002368CDF80700079306F523506368CDF8BE
:103320000B1008932422A3688DF80F7001A90830B0
:10333000099344F06FFE0BB0F0BD000010B500F52E
:103340000053044600F523501A7F93F8801D08307F
:1033500045F020F804F58F5008300AF0ADFC04F574
:103360008870BDE8104015F0FBB8000000F5235050
:1033700002499422083045F02FBB00BF0C8E0B0889
:103380007047000000207047002070470020704701
:1033900000207047002070470020704770470000F1
:1033A0000120704700F5005090F8800D7047000034
:1033B00000B52DED028B08EE101A87B00346074AC0
:1033C000142101A870F006FDB8EEC80A01A83BF070
:1033D000E1FC07B0BDEC028B5DF804FBC4A00B0858
:1033E00070B504465FF0E8FE04F1580050F09CFC14
:1033F0000C4E0D4BA3657825601950F0EBFD66511E
:103400002C35B5F54E7FF7D104F54E7052F06AFABF
:1034100004F24C7000F08AFD204604493BF07AF833
:10342000204670BD00A20B081CAE0B0814A30B08AD
:1034300030B50A4D0FCD8DB06C460FC40FCD0FC403
:1034400095E80F0084E80F000022032168463AF057
:103450001FFE52F093F80DB030BD00BF48610B085D
:103460002DE9F0413C4B1E680446F06A036804F500
:10347000015586B01B6800212035984728463BF04F
:103480001FF928B104F50053B3F96030012B15D0B2
:10349000B069324903681B68984752F059FB39F00C
:1034A0003FFD012302A92846ADF808303BF0F2FEAB
:1034B000B0692B4A03682B491B68984702A9284624
:1034C0000127ADF808703BF0C1FE71F0C3FB054663
:1034D0003AF080FCB6693368D3F8008071F0BAFB2B
:1034E0002149421B3046C0470521204800223AF0BE
:1034F000CFFD3BF015FA1E4A1388204643F008031F
:103500001380FFF795FF17211A483BF0D5FB1A48A7
:10351000B6EE000A3BF0E6FB04F5045002A91830B1
:103520003AF006FBA8B1002540F6D373CDE900358B
:10353000124ABDF80800132304F5F0513AF0ACFD2F
:10354000CDE900570E4A2B4604F5FB5139203AF0DD
:10355000A3FD06B0BDE8F081A8250020D8A00B0887
:10356000FCA00B0836420C0802A10B08C4A20B08F1
:10357000D47B00200CA20B0816A10B0808BB0B087B
:10358000B0AE0C082DE9F347DFF85880144EDFF891
:103590005890092538F9027B0DF10701384652F0A1
:1035A0000BF978B9681EC0B251F0B0FE50B9B246FE
:1035B00004461AF8011B484602F060F958B9013474
:1035C000092CF6D10135EDB20C2D06F10906E1D139
:1035D00002B0BDE8F08739462846FFF7E9FEF1E77B
:1035E00078AC0B0894AC0B08B02500202DE9F04F07
:1035F00085B0B523ADF80830B623ADF80A303B23CB
:10360000ADF80C301A4EDFF86CA03C23ADF80E304C
:1036100002AF00250DF10C0937F9028B0DF10701FE
:10362000404652F0C9F830B939F915000DF10701DB
:1036300052F0C2F818B90336B5B90125ECE7B34624
:1036400003241BF8011B504602F018F938B19DF80D
:10365000070001304146C0B2FFF7AAFEEBE7013C8C
:1036600014F0FF04EDD1E6E705B0BDE8F08F00BF30
:1036700070AC0B08B0250020F0B500F5275600F51A
:103680002D541C4F85B033360125383416F9011BF3
:10369000002924DD3B68D86903680DF10F02DB695E
:1036A000C9B29847D8B19DF80F0052F013FAB0B9DB
:1036B0009DF80F0051F02AFE9DF80F300133009362
:1036C0002B4688B9062120460B4A48F063FD9DF839
:1036D0000F0001304FF0FF31C0B2FFF769FE013536
:1036E000042DD3D105B0F0BD044A0421204648F092
:1036F00051FDF4E7A825002028A10B0859A10B08CB
:103700002DE9FF4700F58B56264FDFF8A0800546D0
:10371000002302364FF0060909FB03F25FFA83FA31
:10372000B15EB256002A03F101042EDD3B68D86970
:1037300003680DF10F02DB69C9B2984728B35146FF
:1037400005F58B5054F036FCF8B19DF80F0052F09F
:10375000C1F9D0B99DF80F0051F0D8FD9DF80F3098
:1037600005F52D5C013300930CF1380C234690B91C
:10377000494660460C4A48F00DFD9DF80F000130A7
:103780004FF0FF31C0B2FFF713FE062C2346C1D124
:1037900004B0BDE8F08742460421604648F0FAFCD8
:1037A000F3E700BFA825002098A10B08C1A10B08D2
:1037B00000207047002070470069C0F34010704738
:1037C0000F299DBF2C2303FB0100203000207047F0
:1037D000002070470120704701F0B0B801F0F2B945
:1037E00000F036BD01F05ABC70B51F4B036000F508
:1037F00000530446D3F8100D1C4AC3F8782B08B1C7
:103800000FF04EFE1A4B236004F5805393F8AC2D55
:1038100042B9D3F8A85D2DB1284619F0A5FD284678
:103820000FF038FE04F58750103065F0E9FE04F61D
:10383000F87052F087FE04F6FC4504F69C46B5424B
:1038400004D0183D284619F0D5FAF8E7094BC4F81A
:10385000D83804F6CC1047F02DFD04F5146047F07D
:1038600029FD204670BD00BF20AC0B0868590C082C
:103870008C380C08E4010C0838B5414B044640F87C
:10388000043B52F0D7FF04F110000DF0F9F804F1F9
:10389000600041F0BDF904F5887014F081F904F579
:1038A0008D600BF021FF04F2945012F0A7F904F69A
:1038B000D8001AF0B1FD04F6784052F043FF04F648
:1038C00048503CF01BF804F6F87052F023FE04F563
:1038D000815014300EF046FC04F58750103065F02E
:1038E0007BFE04F588500C3041F040FD04F58B5010
:1038F00054F07CF904F580530025224A83F8845162
:1039000004F58C5004F58C5304331430136037F0F5
:10391000E1FE04F58F502946083008F0A5FB04F5B8
:10392000C15018305FF03AF804F5E1501C3062F0F5
:1039300051FF04F5EA50143065F008F804F5ED5035
:10394000183065F033FC04F5F05007F007F904F582
:10395000FB5058F0CDFF04F5005318461D770A4D73
:10396000343066F08FF92B6813B1084871F04CF9C8
:10397000204607493AF0CEFD2C60204638BD00BFF6
:103980008C380C08C4850020287C002038AE0B0839
:10399000F4370C0810B5044656306BF00FFC04F1F8
:1039A00058006BF00BFC04F15A006BF007FC04F1BB
:1039B0005C006BF003FC04F15E006BF0FFFB04F1B4
:1039C00060006BF0FBFB04F162006BF0F7FB04F1AD
:1039D00064006BF0F3FB04F166006BF0EFFB04F1A5
:1039E00068006BF0EBFB04F16A006BF0E7FB04F19D
:1039F0006C006BF0E3FB04F16E006BF0DFFB04F195
:103A000070006BF0DBFB04F172006BF0D7FB04F18C
:103A100074006BF0D3FB04F176006BF0CFFB04F184
:103A200078006BF0CBFB04F17A006BF0C7FB04F17C
:103A30007C006BF0C3FB04F17E006BF0BFFB04F174
:103A400080006BF0BBFB04F182006BF0B7FB04F16C
:103A500084006BF0B3FB04F186006BF0AFFB04F164
:103A600088006BF0ABFB04F18A006BF0A7FB04F15C
:103A70008C006BF0A3FB04F18E006BF09FFB04F154
:103A800090006BF09BFB04F192006BF097FB04F14C
:103A900094006BF093FB204610BD00002DE9F04F21
:103AA000044685B0FFF7E8FEB94B236004F50150EA
:103AB0002030FFF76FFF04F504501830FFF790FC3B
:103AC00004F5025104F523501031083004F5005577
:103AD00044F0B6F904F5275018306BF091FB95F8D7
:103AE000FC3923F0030385F8FC3905F608234FF071
:103AF00000080026A5F8FE89C5F8008AC5F8048AE2
:103B00001E6005F60C2304F528501E60103047F0A7
:103B100047FE04F52850203052F010F99D4BC5F8AF
:103B2000A03A9D4BC5F8A83A04F52B509B4BC5F81D
:103B3000B03AC5F89C4AC5F8A44AC5F8AC4A043066
:103B40000FF094F904F52B5020300FF08FF904F5A5
:103B50002B503C300FF08AF94FF6FF79904BC5F8A7
:103B6000103B04F52A5707F19800A5F8149B0FF0B5
:103B70007DF904378B4B8C491F6038463AF0CAFCFC
:103B800004F5015B894BC5F8748B04F52E5704F5D9
:103B90002F580BF11C0BA5F8BC9AA5F8D89AC5F8BC
:103BA000783B0C3708F13008384614374CF05CFA93
:103BB0004745F9D10723C5F8143D0023A5F8183D62
:103BC0004FF4CB700FF06AFCC5F8100D04F53450BB
:103BD0001C306FF07BFF04F5355020306FF076FF1E
:103BE000734A13681BB904F52D5338331360714BB6
:103BF000C5F8783B04F53659132309F1280985F8EF
:103C0000803D4FF4C87148466DF066FC6A4BC5F8BC
:103C1000A83D6A4B04F54058C8E91C33684B1F683F
:103C200017B1684870F0F0FFC3F80090664BC5F814
:103C3000A83D05F6A8534FF07E52C3F84023C3F8C1
:103C40004463624948463AF065FC614B0393614B1B
:103C50000093029404AB04F5445013E90C004FF4B4
:103C6000007108300CF070FA04F5575008306EF00F
:103C700063F9594BC8F8C83504F5585088F81176DF
:103C800014300FF0F3F8012388F8243608F5C563E3
:103C900004F58F511E605E609E6008F5CA630831AE
:103CA0001E605E609E6008F25C639FED4C0A1E60C1
:103CB0005E609E6004F559562C36C8F868163A4680
:103CC000304604F55C5808F05BF908F128085A46BC
:103CD00004F5595A04F56C5B0AF1100A0BF12C0B30
:103CE00031464B46404666F08BF931464B465246CC
:103CF000CDF80080584668F0FBFA04F57B50324658
:103D00005B465146CDF800801C306AF01DF904F581
:103D10008F4032465B465146CDF8008014306AF041
:103D2000C1FF04F58F405B4632465146643069F06E
:103D3000B5FD04F590404FF400413C300CF0A2FF7B
:103D400004F591403C303BF05BFB04F59140503072
:103D500004F5A04642F0C8FB2C22394606F5B670A1
:103D60009EF000F91E4A1F49116004F5A343183361
:103D70004FF0140CB8B20CFB00120137127C002A71
:103D8000F8D1194A1080194A17689FB3184849E7B3
:103D900020AC0B08D9370108DD370108E1370108ED
:103DA0000000FFFF207B0020D40E0C0868590C088F
:103DB0002C7F0020D86B0B0840CD0C08776A0C08CC
:103DC0003C8C00204CAE0B08D8CB0C08E0CA0C0889
:103DD000E5370108E0680B08E8630B080000000005
:103DE000E47B002094A30B08E07B0020A47B002050
:103DF0006EAE0B0804F5A3403430C6E96A77C6F806
:103E0000B001136002F028FC304BC6F8B43104F561
:103E1000A340703002F020FC2D4BC6F8F03104F5C1
:103E2000A4402C3002F018FC2A4BC6F82C3204F5C2
:103E3000A440683002F010FC274BC6F8683204F545
:103E4000A540243002F008FC244BC6F8A43204F547
:103E5000A540603002F000FC214BC6F8E03204F5CA
:103E6000A6401C3002F0F8FB1E4BC6F81C3304F5CC
:103E7000A640583002F0F0FB1B4BC6F8583304F54F
:103E8000A740143002F0E8FB184BC6F8943304F551
:103E9000A740503002F0E0FB154BC6F8D03304F5D4
:103EA000A8400C3005F0CAFDA6F8547495F8A03D62
:103EB00043F0010385F8A03D0E4B1A680AB10E4885
:103EC000B0E620461C6005B0BDE8F08FD4B40B0806
:103ED00090B60B087CB20B08D0B20B08E4B30B0809
:103EE00084B40B083CB60B0834B40B08E0B60B08DE
:103EF000ECB50B08A425002089AE0B0810B570F0B6
:103F0000C1F9064C064B18602046FFF7C7FD204656
:103F1000044A0549BDE810409BF0C4BAB025002012
:103F2000A8250020A4D80020E937010810B50349CE
:103F300004463AF0EFFA204610BD00BF48AF0B0828
:103F400073B51B4D00F13006B8240DF1070120B206
:103F500051F032FC08B39DF807300F2B25D82A68A2
:103F6000D6ED006A03EB830302EB830032F82330C3
:103F70004288D21A92B207EE902AB8EEE77A07EE9C
:103F8000903AF8EEE77A0022E7EE267AFCEEE77A3E
:103F900017EE903A99B251F067F80134A4B2BE2CF2
:103FA00006F10406D1D102B070BD00231B88FFDEEC
:103FB000A07F0020F7B51B4F054600F13006B8245E
:103FC0000DF1070120B251F0F7FBD8B19DF8073091
:103FD0000F2B23D83A6803EB830302EB830032F8FC
:103FE000231082884388521A07EE902A5B1A9BB2EC
:103FF000B8EEE77A07EE903AF8EE677AC7EE276AEE
:10400000C6ED006A0134A4B2BE2C06F10406D7D175
:10401000284603B0BDE8F040FFF792BF00231B889D
:10402000FFDE00BFA07F0020052910B510D800EBEF
:10403000810494ED0C0AD4ED007ADFED060A30EE2F
:10404000270A6020B7EE001A1CF00EFB84ED0C0A64
:1040500010BD00BF00000000052910B510D800EB0E
:10406000810494ED0C0AD4ED007ADFED060A30EEFF
:10407000670A6720B7EE001A1CF0F6FA84ED0C0A06
:1040800010BD00BF0000000005299EBF00EB8100AD
:10409000002303637047000005299EBF00EB8100E9
:1040A0004FF07E530363704705290ED800EB810162
:1040B00091ED0C7ADFED057AB4EEE77AF1EE10FAC5
:1040C0004CBF4FF07C5300230B637047CDCCCC3EEC
:1040D00005290FD800EB810191ED0C7ADFED067A0E
:1040E000B4EEE77AF1EE10FAACBF4FF07C534FF02C
:1040F0007E530B63704700BF9A99193F05299EBFF5
:1041000000EB81004FF07C5303637047F0B5044629
:1041100085B004F58F56684608360F4615460EF0F2
:10412000A5FE6946304609F021FA10B9002005B015
:10413000F0BD3946304609F0B9F80028F6D0002D18
:10414000F5D004F58054284694F85C3443F002031B
:1041500084F85C34EBE7000030B5044689B068466B
:1041600004F58F550EF082FE083504A80EF07EFE91
:104170006946284609F0B6F958B104A9284609F05D
:10418000F5F930B1059B0193002269462046FFF7FF
:10419000BDFF09B030BD000010B586B0044602A8CE
:1041A00001910EF063FE04F58F5002A9083009F06A
:1041B00099F9019AC0B194F87914DDED037A9FED75
:1041C0000B7A242004F58D6300FB0133D3ED0B6AD9
:1041D000F8EEE77A02A9E6EEC77A2046FDEEE77A26
:1041E000CDED037AFFF792FF06B010BD0000C84284
:1041F00000F5805292F85C24D20708D400F50053F1
:1042000093F87B1E09B1FFF7A7BFFFF7C5BF704743
:1042100030B585B0054668460C460EF027FE05F51C
:104220008F506946083009F0A1F960B1684621460F
:104230000FF05AF8DFED057AB4EEE70AF1EE10FA66
:10424000CCBF0120002005B030BD00BF0050434767
:1042500010B50A4A1378044600F5A54043F08003E0
:104260002430137003F0A8FA30B920460822BDE8C4
:104270001040022102F08ABA10BD00BF6C7B002002
:104280002DE9F04101F1080305460F460FCB88B038
:1042900004AC84E80F0005F54056134301BFD6F87F
:1042A0001C360693D6F820360793059BB3B92046F3
:1042B0000EF00CFE05F5585808F11408014603AA43
:1042C00040460EF00FFEC0B10399019120460EF05A
:1042D000FDFD0199024620460EF0CEFD0023C6F8F2
:1042E000FC30BB88A6F8FA3005F5A54021462430FD
:1042F00002F04EFF08B0BDE8F081D6F81816019123
:104300004046E4E770B58CB00D4604AC0646204646
:104310000EF0ACFD2B691F490BB96B693BB3002351
:104320000B7005F108010FC984E80F0006F558501D
:1043300003AA032114300EF0D5FD90B108AA032181
:1043400020460EF0CFFD60B10399032220460EF007
:1043500093FD06F5A5402146243002F019FF0CB06C
:1043600070BD06F540530122D3F81816EEE701227E
:104370000A7006F54051009208ADD1F82026D1F818
:104380001C1628460EF092FD95E80F0084E80F00F9
:10439000DFE700BF087A002000F5A25100F5A54034
:1043A0000C31243002F0F4BE70B5083105460FC957
:1043B0008EB006AC84E80F00134312D105F57B5094
:1043C000002303A91C3003930493059369F036FE80
:1043D000022203A90AA80EF0FDFF0C9B08930D9B77
:1043E0000993079BABB920460EF070FD05F55856B2
:1043F000143601460AAA30460EF074FD88B10A99B7
:10440000019120460EF062FD0199024620460EF011
:1044100033FD05F5A5402146243002F0B9FE0EB06B
:1044200070BD05F540533046D3F818160191E9E701
:10443000F0B501F1080305460E460FCB89B004AC78
:1044400084E80F00134307D105F54053D3F81C2629
:10445000D3F8203606920793059BABB920460EF0A1
:1044600035FD05F558571437014603AA38460EF0B6
:1044700039FD08B30399019120460EF027FD0199FB
:10448000024620460EF0F8FC327EB388D2074FEA8F
:10449000132344BF03EB83035B00327A07EE903AA9
:1044A00005F5A540B8EE670AC2F340022146243064
:1044B00002F0B2FE09B0F0BD05F540533846D3F81E
:1044C000181601910EF002FD0199024620460EF0E9
:1044D000D3FC44F097FD0222152144F04BFBD3E7B7
:1044E00038B504460D46FFF75FFF04F54050002342
:1044F000C0F8FC30AB88A0F8FA3038BD10B58B8816
:1045000053B100F5A5442434204604F0B5FA204602
:10451000BDE8104003F0C0BA10BD000073B50546F9
:104520000C4670F0A3FB05F54056C6F80401D4ED27
:10453000027AF5EEC07AF1EE10FA17DD9FED137AEC
:1045400067EE877AFCEEE77AC6ED407AD6F800216E
:1045500005F52D504FF47A73B2FBF3F30C4A0621A4
:10456000383002B0BDE8704047F014BE58F06AF928
:104570000023009394F90D2094F90E3094F90C1057
:1045800058F0FCF8C6F80001E0E700BF00007A44EC
:10459000B8AF0B08DFED0B7A91ED041AD1ED030AE9
:1045A00091ED020A8B8800F5A5404FF47A7121EE57
:1045B000271A60EEA70A20EE270A5943603004F05C
:1045C0004FBA00BF0000C842F8B500F54055064696
:1045D00095F8E04E14F001040F4602D10024204665
:1045E000F8BD114A537843F001035370D5F8FC30FD
:1045F0001BB970F03BFBC5F8FC0070F037FBD5F839
:10460000FC30B5F8FA20C31A4FF47A70B3FBF0F31C
:104610009342E3D306F52D503B88044A06213830F7
:1046200047F0B8FDDBE700BF6C7B0020C8AF0B088C
:10463000F0B5144E357887B0044625B1012D1AD057
:10464000012007B0F0BD00F5405393F8E02E12F0C2
:104650000100F6D001270097D1E904122B4602A8E9
:104660000EF024FC04F5A540243002A902F090FDD0
:1046700037702846E5E700F5405494F8E00E00F066
:104680000100DEE7087A002010B500F5405494F8E8
:10469000E03E13F0010015D0D4F8FC301BB970F0E7
:1046A000E5FAC4F8FC0070F0E1FAD4F8FC30C01A66
:1046B0004FF47A73B0FBF3F3B4F8FA00834234BFDB
:1046C0000020012010BD00007FB500F5A043054685
:1046D00093F85434012B0C4636D100F5405393F82F
:1046E000E00E10F001002DD001AE0023314604F1A0
:1046F00008000193029303930EF03AFDDDED037A77
:104700009FED207AF0EEE77AF4EEC77AF1EE10FA38
:1047100006D505F5595010306AF044FD8DED030AB9
:1047200023694BB963693BB905F5595010306AF0FC
:1047300037FD03C886E8030005F5A540243002F0E4
:1047400055FD002004B070BD0B79DFED0F6A07EE58
:10475000903A0B7E9B070D4B48BF9FED0D7A93ED72
:10476000006AF8EE677A48BF67EE877A86EE267AA7
:10477000B0EEC77AB4EEE77AF1EE10FAACBF0120E2
:104780000020DFE700000034DB0FC940CC6D0020C3
:104790000000803B8B8823B100F5A540243004F055
:1047A0007DB901207047000010B5044670F05EFA34
:1047B00004F54053D3F80421801AD3F80021904225
:1047C0004FF0000084BFC3F80001012010BD0000BD
:1047D00038B504460D4670F049FA04F540539FED94
:1047E000077AC3F84C06D5ED027A67EE877AFDEEBC
:1047F000E77A17EE902AC3F8482638BD00007A44BD
:104800000B464A7CD3ED030A91F9101093ED020A8E
:10481000014802F0E9BD00BF5478002010B50446FD
:1048200070F024FA04F54053D3F84C26801AD3F8DC
:10483000482622EAE27290424FF0000084BFC3F89B
:104840004806012010BD000038B500F5405504466B
:1048500095F82436032B03D00A48032103F098FB74
:1048600004F58054D5F83C36D4F8E003C01A1BF0A8
:10487000C3FE0028B8BF4042C828CCBF002001209A
:1048800038BD00BF5478002008B500F5005393F8F8
:10489000803D042B07D0032B0AD100F5A04393F8E9
:1048A0005434032B04D14B88102B03D0732B07D027
:1048B000002008E0BDE808400348083104F09CB936
:1048C000FFF79EFF012008BD90780020D1F8093045
:1048D00007EE903AF5EEC07AF1EE10FA08DD9FEDA2
:1048E000050A00F57B5027EE800A1C3069F03ABCBF
:1048F000704700BF0000C84213B58B88012B0446E7
:1049000005D00B6953B94B6943B9CB6833B9002162
:10491000204602B0BDE81040FFF73EBC08312046FB
:104920000191FFF775FC0199024628B9204602B0B3
:10493000BDE81040FFF7EABB02B010BD37B50D4629
:104940004FF48071044606F07FF840B104F52A5117
:1049500004F523502A460431083043F04FFD05F199
:104960000801084601910EF0B1FA012801990CD115
:10497000EB68002B12DD494A04F52D500421383034
:1049800047F008FC002003B030BD032804D1EB68D9
:10499000002B03DA424AEFE7424AEDE76B88702BBF
:1049A00062D017D8152B09D80F2B0BD9113B042B2C
:1049B00032D8DFE803F040454A3C37005C2B49D051
:1049C0005D2B4CD004F52D50374A0421383047F088
:1049D000E1FBD7E7B32B56D014D8732B49D0B22BB9
:1049E0004CD0722BEED1D5ED027A9FED307A67EE86
:1049F000877A04F54054FDEEE77A17EE903AC4F852
:104A000048360DE0CD2B0BD0DE2B41D0C92BD9D1B0
:104A1000274802F05DFD03E029462046FFF730FC01
:104A20000120B0E729462046FFF76CFCF8E7204656
:104A3000FFF7B2FCF4E729462046FFF7B5FCEFE7A5
:104A400029462046FFF7F4FCEAE729462046FFF70F
:104A500047FDE5E729462046FFF750FDE0E72946F8
:104A60002046FFF75BFDDBE729462046FFF7B0FE57
:104A7000D6E729462046FFF7C3FED1E72946204660
:104A8000FFF724FFCCE729462046FFF735FFC7E7AD
:104A900029462046FFF77EFDC2E700BFDCAF0B08CA
:104AA000FCAF0B081FB00B082DB00B080000C8426C
:104AB0005478002010B5044604F5405400F57B50AE
:104AC0001C3069F009FAD4F8483623EAE37307EE9C
:104AD000903AF8EEE77A0020B4EEE70AF1EE10FA29
:104AE00044BFC4F84806012010BD000010B54B8833
:104AF000152B04460A4609D80F2B0ED9113B042B5F
:104B00002FD8DFE803F0583F44383300702B4AD0E9
:104B10000BD85C2B3FD05D2B41D004F52D50274A9C
:104B20000421383047F036FB19E0732B3FD005D80D
:104B3000722BF2D1BDE81040FFF7BCBFB32B02D8F7
:104B4000B12BEAD90BE0A3F1C90189B21529E4D848
:104B50001B48012202FA01F108400028DDD00120A3
:104B60000FE0BDE810401146FFF72EBDBDE8104034
:104B70001146FFF75DBD00F5405494F8E00E00F0DB
:104B8000010010BDBDE810401146FFF79DBDBDE816
:104B90001040FFF779BDBDE81040FFF7FBBDBDE851
:104BA0001040FFF701BEBDE81040FFF737BEBDE87B
:104BB0001040FFF749BE0020E3E700BF44B00B08F8
:104BC0003100200070B500F50053054693F8803D94
:104BD000032B0E4602D00024204670BDFFF786FF4F
:104BE00004460028F7D005F52D50318838304EF0B6
:104BF00003F9F1E708B5044B01221A7070F02AF8A6
:104C0000024B186008BD00BF0A7A0020107A00200D
:104C1000014B00221A7070470A7A002038B500F55F
:104C20000054054694F97630C3B170F01FF8D4ED06
:104C30001E7A05F58D6393ED097A194BF8EEE77A44
:104C4000F4EEC77AF1EE10FA09DD1860154B186022
:104C500094F8A03D6FF3451384F8A03D38BD1B6860
:104C600003F5FA6383423EBF94F8A03D43F020036E
:104C700084F8A03D94F8A03D9B06EFD5094A13683F
:104C800003F5EA4330338342E8D2106005F52D5036
:104C9000054ABDE838400421383047F07BBA00BFF0
:104CA0001C7A0020207A002060B00B0838B500F58F
:104CB0000054054694F97730D3B16FF0D7FF94F9DB
:104CC0007C3007EE903A05F58D6393ED0A7A194B27
:104CD000F8EEE77AF4EEC77AF1EE10FA09DD186023
:104CE000154B186094F8A03D6FF3861384F8A03D2F
:104CF00038BD1B6803F5FA6383423EBF94F8A03DBC
:104D000043F0400384F8A03D94F8A03D5B06EFD546
:104D1000094A136803F5EA4330338342E8D210604E
:104D200005F52D50054ABDE838400421383047F0DC
:104D300031BA00BF247A0020287A00207CB00B080A
:104D400070B500F50054284E94F8EA39054613B1C1
:104D500094F9743093B994F8A03DD90605D544F080
:104D600051F900221B2143F005FF94F8A03D0022D9
:104D700062F30413F27484F8A03D70BD0123F37450
:104D80006FF074FFD4F8843D03F59C4320338342D5
:104D900008D2C4F8840D05F52D50144A022138308C
:104DA00047F0F8F994F8A03DDA06E6D443F0100392
:104DB00084F8A03D44F026F901221B2143F0DAFEDD
:104DC00094F8A03DDB06D8D594F97430022BD4D1E9
:104DD00094F87B3E002BD0D028461D22BDE87040C1
:104DE000092101F0D3BC00BF4D7B00209CB00B0813
:104DF00038B504460D466FF039FF04F500533DB950
:104E0000D3F8902DC3F8940D0AB9C3F8900D38BDAE
:104E1000D3F8942D801A642882BF0022C3F8942D01
:104E2000C3F8902DF3E70000F8B504466FF012FFC9
:104E3000294BB4F8B6201988284E914205460ED069
:104E40001A80274B18603378A3B10024347044F0E3
:104E5000D9F822461321BDE8F84043F08BBE3378E1
:104E6000204FD3B93B782BB11D4B1F4A1B68C31A87
:104E7000934200D8F8BD0123337004F5005393F832
:104E80007B3E23B104F5365028306AF0C5FA44F071
:104E9000B9F80122132143F06DFE3B78002BE9D0D5
:104EA0003378002BE6D00E4A10491368EB1A8B4278
:104EB000E0D904F50053156093F87B3E002BD9D060
:104EC00004F536542834204600216BF009FA2046B8
:104ED000BDE8F8406CF0FEBD0C7A0020097A002095
:104EE000107A00200A7A002080841E0040420F00C1
:104EF00038B500F50054054694F87D3DD80714D523
:104F000094F8A41D94F8A13DC90703F001020DD542
:104F10005AB144F077F800221A2143F02BFE94F89E
:104F2000A13D6FF3000384F8A13D38BD002AFCD1F8
:104F300043F0010305F52D5084F8A13D144A0221E8
:104F4000383047F027F944F05DF803221A2143F086
:104F500011FE94F8803D022B0FD11C22132128460C
:104F600001F014FC0028E0D105F557500122BDE8FE
:104F7000384017210830FCF7C3BB092BEDD0054B97
:104F8000D3F8B00103689B6898470028E5D1CCE7C7
:104F9000ACB00B08B0750020F0B500F500543C4EE5
:104FA00094F994708BB0054667B96FF05FFE94F882
:104FB000A03D306067F3820384F8A03D354BDF737A
:104FC0000BB0F0BD002307930893099307AF05AB1F
:104FD00000F58F50019303AA04AB06A9009708308F
:104FE00008F0EAF938461EF089FAD4ED267AF4EE94
:104FF000C07AF1EE10FA13DD9DED067AF4EEC77A71
:10500000F1EE10FA0CDD6FF031FE94F8A03D306047
:105010006FF3820384F8A03D1E4B0022DA73CFE7C2
:105020006FF024FE336803F5FA63984294F8A03DCC
:10503000EED35A07C4D443F0040384F8A03D154BC3
:105040000122DA7343F0DEFF0222102143F092FDC9
:105050006FF00CFED4F89C3D03F59C43203398423E
:105060000AD96FF003FEC4F89C0D05F52D500A4ACD
:105070000421383047F08EF894F99430022B9FD1F8
:1050800005F55750012218210830FCF739FB97E746
:10509000147A00204D7B0020C0B00B0838B51546AF
:1050A000044643F0AFFF0122062143F063FD022DC9
:1050B00008D0032D0FD120460422BDE83840092135
:1050C00001F064BB04F557500122BDE838400721C8
:1050D0000830FCF715BB38BD38B500F5005405465F
:1050E00094F97E3033B994F8A03D6FF3000384F84F
:1050F000A03D38BD6FF0BAFDD4F88C3D9FED1B7A12
:10510000D4ED206A07EE903AF8EE677AE6EE877AF9
:1051100007EE100AB8EE477AB4EEE77AF1EE10FA2D
:10512000E1D494F8A03DDA07E3D443F0010384F816
:10513000A03D43F067FF01221C2143F01BFD05F554
:105140002D500B4A0221383047F024F8284600F051
:105150006BFB94F97E30022BCBD105F55750012221
:10516000BDE838401D210830FCF7CABA00007A4477
:10517000C8B00B0870B500F50054054694F97530B9
:10518000CBB1D4F80C6DB6B16FF070FD40F6C3131F
:10519000861B9E4210D894F8A03D990705D543F090
:1051A00031FF0022082143F0E5FC94F8A03D6FF3A5
:1051B000410384F8A03D70BDD4F8883D47F23052D9
:1051C000C31A93420AD9C4F8880D05F52D50B4F9D5
:1051D0006430224A0421383046F0DCFF94F8A03DC8
:1051E0009A07E8D494F87B2E002AE4D043F0020317
:1051F00084F8A03D43F006FF0122082143F0BAFCE9
:1052000094F97530022B08D10122122105F557506F
:105210000830BDE87040FCF773BA032B0DD194F849
:105220007B3E002BC7D005220221284601F0AEFAB2
:105230000028C0D101221A21E8E7042BBBD194F841
:105240007B3E002BB7D005220921284601F09EFAAB
:105250000028B0D101221921D8E700BFDCB00B082B
:1052600038B5054605F500546FF000FD94F87B2E27
:10527000294B12B194F995203AB9186094F8A03DE1
:105280006FF3C71384F8A03D38BD94F8802D012A30
:10529000F3D0132AF1D005F55C529FED207AD2EDC0
:1052A000377A67EE877AB3EE0E7AF4EEC77AF1EECC
:1052B00010FAE2D91B6803F5FA638342E4D8D4F804
:1052C000983D03F59C432033834208D2C4F8980DDF
:1052D00005F52D50124A0421383046F05BFF94F951
:1052E000A03D002BD0DB94F8A03D43F0800384F870
:1052F000A03D43F087FE01220C2143F03BFC94F9D2
:105300009530022BC0D105F557500122BDE8384039
:105310000C210830FCF7F4B9187A0020E02E654221
:10532000F8B00B0810B500F50053044693F97D3032
:10533000012B0AD0022B18D000F55750BDE81040C1
:10534000012215210830FCF7DBB90B22102101F0F6
:105350001DFA20B90B220221204601F017FA044A57
:10536000137843F00803137010BD0B220921F4E7F2
:105370006C7B002038B500F50055044695F8A03D3B
:1053800043F0080385F8A03D43F03CFE01221721BD
:1053900043F0F0FB95F8FC39DB0704D42046BDE868
:1053A0003840FFF7BFBF034802F0AEF80028F5D041
:1053B00038BD00BF5478002070B500F50055064692
:1053C00095F8803DD5F8944DD5F8902D033B012BF1
:1053D00018D8A41AB4F57A7F94BF0024012495F854
:1053E000A03DC3F3C003A3421AD06CB106F52D5003
:1053F00038300C4A022146F0CDFE3046BDE8704000
:10540000FFF7B8BF0024EAE743F0FCFD224617216E
:1054100043F0B0FB95F8A03D64F3C30385F8A03DCD
:1054200070BD00BF08B10B0813B500F5005393F829
:105430007B3EA3B100F5805090F8A04F094857F08B
:1054400029FD024648B1019243F0DCFD019A092191
:1054500002B0BDE8104043F08DBB002CF3D102B088
:1054600010BD00BF1045002030B500F5595510356E
:1054700087B004460021284669F034FE02A80DF0EA
:10548000F5FC04F58F5002A904F54054083008F0EB
:1054900029F8049BC4F81C36059BC4F8203628461E
:1054A00069F072FE830611D5284669F07BFEBDEED9
:1054B000C00A284610EE103AC4F8183669F07AFE91
:1054C000BDEEC00A10EE103AA4F8003607B030BDA9
:1054D000012252F029BD0000002252F025BD00003B
:1054E0001F2900F28D80DFE801F08B1014181C20BA
:1054F00023272B2F33373B3F43474B4F53575B5F9C
:1055000063676B6F73777B7F838700F5025038305A
:10551000704700F502503A30704700F502503C30B9
:10552000704700F502503E30704700F50350704759
:1055300000F503500230704700F503500430704707
:1055400000F503500630704700F5035008307047EF
:1055500000F503500A30704700F503500C307047D7
:1055600000F503500E30704700F5035010307047BF
:1055700000F503501230704700F5035014307047A7
:1055800000F503501630704700F50350183070478F
:1055900000F503501A30704700F503501C30704777
:1055A00000F503501E30704700F50350203070475F
:1055B00000F503502230704700F503502430704747
:1055C00000F503502630704700F50350283070472F
:1055D00000F503502A30704700F503502C30704717
:1055E00000F503502E30704700F5035030307047FF
:1055F00000F503503230704700F5035034307047E7
:1056000000F502503630704710B50446FFF768FFCA
:10561000114669F0DDFD030648D4672808D85128F3
:105620003ED84F285AD84C38C0B2012850D910BDA6
:10563000A0F16803172BFAD801A252F823F000BF9B
:10564000B9560108C5560108C9560108CD560108CA
:105650002F5601082F5601082F5601082F56010812
:105660002F5601082F5601082F5601082F56010802
:105670002F560108E1560108E15601082F5601088E
:105680002F5601082F5601082F5601082F560108E2
:105690002F5601082F560108E5560108E556010866
:1056A0005438C0B20128C2D8022112E07930C0B209
:1056B0000128BCD805210CE0002104F58B50FFF730
:1056C0000BFFB4E70121F8E70221F6E70321F4E735
:1056D0000021BDE810400448FEF710BD0121F8E7A5
:1056E0000321F6E70421F4E7144E0020F0B50F4B38
:1056F00089B06A46064603F12007144618685968BF
:10570000154603C50833BB422A46F7D10025E9B246
:105710003046FFF7E5FE0135627814F8021B69F0A8
:105720005DFD102DF3D109B0F0BD00BF78610B080D
:1057300037B5044604F50055FFF7D8FF01221321C1
:10574000204601F023F895F9AC30002B09DC04F574
:10575000025001230DF107012C308DF8073039F08C
:1057600047FD95F9AC2095ED280A95ED291AD5ED60
:105770002A0A012A04F540540FD0DFED287A31EED1
:10578000277AB4EEC07AF1EE10FA2CDD70EEE77AEB
:10579000F4EEC07AF1EE10FA25D523201AF064FF5A
:1057A00004F20C6383ED000A04F20C64DFED1C0AC2
:1057B00094ED000AB7EE001A29201AF055FFB52023
:1057C00084ED000A9FED170A4FF088FE9FED150A41
:1057D000B6204FF083FE9FED130AB72003B0BDE85B
:1057E00030404FF07BBE02EBD2735B10013B5BB2EB
:1057F00007EE903A013A31EE601AF8EEE77A07EEDA
:10580000102A67EE817AB8EEC77A04F20C61C7EE0F
:10581000876A76EEA00AC1ED000AC5E70AD7233CE5
:10582000CDCCCC3D0000000038B56FF01FFA00244D
:105830000546E0B22A4640F2DC5101344EF012FB3C
:10584000062CF6D1024A00231380024A138038BD89
:10585000467A0020447A0020054A00231380054A36
:1058600000F540501380044A80F8103613807047CA
:10587000307A0020327A0020347A00202DE9F84373
:105880000025814688462F462C46E9B24846FFF758
:1058900027FE0646B0B1002169F09AFC404503D1CD
:1058A00001242046BDE8F8830021304669F090FCD1
:1058B00001210128304608BF012469F089FC4045D8
:1058C00008BF01270135202DDFD1002CE9D0002FA2
:1058D000E6D13C46E5E7000070B52DED028B84B0C3
:1058E0001D460446FFF7FCFD114669F071FC0238C5
:1058F000882800F2D680DFE810F089009A00A60020
:10590000AC00B600B900C800BC00C200BF00C500B2
:10591000CB00D400D400D400D400D400D400D400F0
:10592000D400CE00D100D400D800F900FB00D40090
:10593000D400D400FD00450169018E01D301F901B5
:10594000D400D400D400D4001F026902DE02340364
:105950004A0353035C036503C104D400CB03B503BE
:10596000BB03DB03D103D303E703DD03DF03D40071
:10597000F50308041B045304AE04FE0311042404BD
:105980005C04B7040004130426045E04B9041B0479
:1059900053042E04890424045C043A049504260468
:1059A0005E043F049A04D400D400D400D400D40090
:1059B000D400D400D400D400D400D400D400D40047
:1059C000F303E903EB03C803D803E403F003D400B3
:1059D000D400D400D40028046004BB0402041504DD
:1059E0002804600444049F042A046204BD040404DF
:1059F00017042A0462044904A4042C04D400BF043C
:105A0000060419042C04D4004E04A90404F55750CC
:105A100004F50054012294F87B3E083011465BB136
:105A200004B0BDEC028BBDE87040FBF769BE0122FB
:105A300004F557501146083004B0BDEC028BBDE8A8
:105A40007040FBF7D7BD012204F5575011460830CE
:105A5000E6E701221321204604B0BDEC028BBDE82D
:105A6000704000F093BE01220021F4E701220221E0
:105A7000F1E701220321EEE701220421EBE70122F5
:105A80000721E8E701221146E5E701221021E2E7BC
:105A900001221521DFE7BB4BBB4A01E0B94BBB4AF2
:105AA0001A6004B0BDEC028B70BD002DF9D1B84A6C
:105AB000137804F52D5483F001031370383473B157
:105AC0009FEDB40AB7204FF009FDB34A06212046E6
:105AD00004B0BDEC028BBDE8704046F05BBB9FEDAF
:105AE000AF0AB7204FF0FAFCAD4AEFE7AD4BD3E772
:105AF000AC4BD4E7002DD4D104F500549FEDA58A1A
:105B0000B4F9B430A84CA94D07EE103AB8EEC77AF4
:105B100095ED000AC8EE077AFCEEE77A17EE903AA8
:105B20009BB207EE903A2378F8EEE77A13B3DFEDF5
:105B30009B0A37EE800AE420B0EE481A1AF094FD72
:105B400085ED000A95ED000AB4EEC80AF1EE10FAF0
:105B500004DAB5EEC00AF1EE10FA03D8237883F028
:105B600001032370B52004B0BDEC028BBDE870408A
:105B70004FF0B4BCDFED890A30EE670AE620B0EEE4
:105B8000481ADBE7002D8CD104F500549FED811AF3
:105B9000B4F9B430854CDFED810A94ED000A07EECC
:105BA000103AB8EEC77AF120C1EE077AFCEEE77A38
:105BB00017EE903A9BB207EE903AF8EEE77A37EE9E
:105BC000800A1AF051FD84ED000ACBE7002D7FF426
:105BD00068AF04F500549FED6F1AB4F9B430734DFB
:105BE000DFED6E0A95ED000A07EE103AB8EEC77ABF
:105BF000F820C1EE077AFCEEE77A17EE903A9BB2F6
:105C000007EE903AF8EEE77A30EE670A1AF02CFDCC
:105C100085ED000AA6E7002D7FF443AF04F500549C
:105C20009FED5C8AB4F9B430614C624D07EE103AD6
:105C3000B8EEC77A95ED000AC8EE077AFCEEE77A6F
:105C400017EE903A9BB207EE903A2378F8EEE77A97
:105C5000EBB1DFED520A37EE800A40F20110B0EEF0
:105C6000481A1AF001FD85ED000A95ED000AB4EE20
:105C7000C80AF1EE10FA04DAB5EEC00AF1EE10FA35
:105C800003D8237883F001032370B6206BE7DFEDA0
:105C9000430A30EE670A40F20310B0EE481AE0E71C
:105CA000002D7FF4FEAE04F500549FED3A1AB4F9CE
:105CB000B430404CDFED390A94ED000A07EE103A9B
:105CC000B8EEC77A4FF48770C1EE077AFCEEE77A38
:105CD00017EE903A9BB207EE903AF8EEE77A37EE7D
:105CE000800A1AF0C1FC84ED000ACEE7002D7FF493
:105CF000D8AE04F500549FED271AB4F9B4302D4DF9
:105D0000DFED260A95ED000A07EE103AB8EEC77AE5
:105D100040F21510C1EE077AFCEEE77A17EE903AE2
:105D20009BB207EE903AF8EEE77A30EE670A1AF087
:105D30009BFC85ED000AA8E7002D7FF4B2AE1E4A59
:105D4000137883F00103002BF6EE007AB7EE007AA9
:105D50000CBF17EE100A17EE900A137004F5585393
:105D600004F52D54D860FAF7CFFB0022134BFAF755
:105D700023FCCDE90001124A38340621204646F0C2
:105D800009FA8EE6082200200080ED440080894454
:105D9000487A002000007A4424B10B08000000007B
:105DA0003BB10B08042200200C2200203C7A00208A
:105DB0000D220020407A0020497A0020000059403E
:105DC00052B10B08CDCC4C3FCDCCCC3D002D7FF457
:105DD00068AE04F500551FED051A5FED050A95ED57
:105DE0002A0A4FF494701AF03FFC04F5025003A9FC
:105DF00028308DED030A39F0A1F9D5ED2A0A95ED89
:105E0000290AB7EE001A40F229101AF02DFC04F509
:105E1000025003A924308DED030A39F08FF90A22CC
:105E2000012195F9AC001AF05DFC8DF80C0004F529
:105E3000025003A92C3039F0DBF995F9AC30012B75
:105E400004F540560ED140F22D1095ED291AD5EDEE
:105E50002A0A95ED280A1AF007FC06F20C6383ED76
:105E6000000A18E0013B95ED291AD5ED2A0A07EE44
:105E7000903A31EE607AF8EEE77A06F20C6587EE3A
:105E8000270A40F22F10D5ED007A30EE270A1AF0DB
:105E9000EBFB85ED000A06F20C6604F52D54306824
:105EA000FAF732FB0022C74BFAF786FB3834CDE90C
:105EB0000001C54A61E7002D7FF4F3AD04F50055FC
:105EC0009FEDC21ADFEDC20A95ED2A0A4FF49C70CD
:105ED0001AF0CAFB04F5025003A928308DED030A1D
:105EE00039F02CF9D5ED2A0A95ED290AB7EE001AFA
:105EF00040F239101AF0B8FB04F5025003A924301F
:105F00008DED030A39F01AF90A22012195F9AC0046
:105F10001AF0E8FB8DF80C0004F5025003A92C30B0
:105F200039F066F995F9AC30012B04F5405602D1F1
:105F300040F23D1089E7013B95ED291AD5ED2A0A7B
:105F400007EE903A71EE606AF8EEE77A06F20C65B9
:105F500086EEA77A40F23F1095ED000A30EE470A30
:105F600095E79C4CB4F900300A3300EE103A4FF438
:105F7000A3709FED991ADFED990AB8EEC00A1AF0E6
:105F800073FBBDEEC00A10EE103A238089E5914CF8
:105F9000B4F900300A3B00EE103A40F24910E8E74D
:105FA0008F4CB4F900300A3300EE103A4FF4A6706B
:105FB000DFE78B4CB4F900300A3B00EE103A40F2B8
:105FC0004F10D6E704F5005393F87B3E002B3FF4C7
:105FD00068AD002D7FF465AD824BB3F90030A3F5B9
:105FE000FA7383EAE372A2EBE372322AC8BF1DB2EE
:105FF0007D4B1D807D4BB3F9002082EAE273A3EB59
:10600000E2739BB2322B7A4B98BF00221A80794BF5
:10601000B3F9003083EAE371A1EBE37189B232296D
:1060200098BF0023744915431D430B8004F5405667
:1060300010D00123714A86F8103604F52D50062140
:10604000383046F0A7F896F810366D4A83F0010311
:10605000137026E596F8103686F81056002BF2D00D
:10606000684AEAE7002104F58B50FFF735FA18E596
:10607000002D7FF416AD294604F58B5004B0BDEC1D
:10608000028BBDE8704051F05DBF002D7FF409AD7B
:10609000002104F58B50FFF71BFA02E50121E2E72E
:1060A000002D7FF4FEAC0121E6E7002D7FF4F9AC72
:1060B0000121EEE70221D6E7002D7FF4F2AC0221A8
:1060C000DAE7002D7FF4EDAC0221E2E70321CAE715
:1060D000002D7FF4E6AC0321CEE7002D7FF4E1AC88
:1060E0000321D6E70021484804B0BDEC028BBDE88F
:1060F0007040FDF799BF0121F5E70221F3E7032185
:10610000F1E70421EFE70521EDE700213E4804B067
:10611000BDEC028BBDE87040FDF79EBF0121F5E7A5
:106120000221F3E70321F1E70421EFE70521EDE781
:106130000021354804B0BDEC028BBDE87040FDF78E
:10614000A3BF0121F5E70221F3E70321F1E70421D1
:10615000EFE70521EDE7002D7FF4A3AC29462A489F
:1061600004B0BDEC028BBDE87040FDF79DBF002D73
:106170007FF497AC0121F2E7002D7FF492AC02216D
:10618000EDE7002D7FF48DAC0321E8E7002D7FF4CF
:1061900088AC0421E3E7002D7FF483AC0521DEE722
:1061A0000021194804B0BDEC028BBDE87040FDF73A
:1061B00073BF0121F5E70221F3E70321F1E7042191
:1061C000EFE700BF0000594061B10B08CDCC4C3F58
:1061D000CDCCCC3D447A002000004843000048C3A9
:1061E000467A00203A7A0020347A0020367A00205D
:1061F000307A0020387A0020327A002072B10B0801
:106200000022002082B10B08144E0020002D7FF4E4
:1062100048AC2946234804B0BDEC028BBDE8704071
:10622000FDF756BF002D7FF43CAC0121F2E7002DB5
:106230007FF437AC0221EDE7002D7FF432AC03216F
:10624000E8E7002D7FF42DAC0421E3E7002D7FF477
:1062500028AC0521DEE70021124804B0BDEC028B1A
:10626000BDE87040FDF74ABF0121F5E70221F3E7E1
:106270000321F1E70421EFE70521EDE7002D7FF48D
:1062800010AC04F5405204F52D5092F8113683F00D
:10629000010382F81136383013B1034A062117E49E
:1062A000024AFBE7144E002097B10B08A9B10B0876
:1062B0002DE9F84F2DED068B994600F55853D3ED97
:1062C00003AADFEDCB7A9FEDCB9A9FEDCB8ABDF889
:1062D000447000F500532AEE899A6AEEA7AAD3ED1E
:1062E0002C7A6AEEA7AADFEDC57AF0EE488AEAEECC
:1062F000E78A4FF0000804460E46FDEEE88A154690
:1063000018EE903A1BB208EE903ABD4B83ED008A2E
:10631000BC4B83ED008ABDF84830C34647EA0347CB
:106320004FF0010A0AFA08F33B425FFA88F109D0FC
:106330002046FFF7D5F8002168F04AFF012808BF82
:106340004FF0010B08F10108B8F1200FEAD1DFF896
:10635000D4A24FF00008012303FA08F0DAF8003065
:1063600038425FFA88F103EA000300F00981003B3C
:1063700018BF01235A462046FFF7AEFA08F101087C
:10638000B8F1200FE7D104F54053CAF8007093F834
:1063900011269D4BBAB1724207EE902AF8EEE77AC9
:1063A00067EE897AFDEEE77A17EE902A07EE905AAB
:1063B000F8EEE77A1A8067EE897A944AFDEEE77A7A
:1063C00017EE901A11806EF051FC914ADFF8588256
:1063D0001278DFF858A28C4B07461FFA89F18D48D6
:1063E000002A40F0D5800088B8F900B000F5FA70B6
:1063F00000B20AEE100ABAF9000009EE900A6FF432
:10640000E170014462290FD885EAE570A0EBE570E0
:1064100080B2312808D886EAE672A2EBE67292B220
:10642000312A8CBF00220122794802701888BDF9F8
:10643000503000F2DC50184440F26C7240F24C4193
:1064400000B21AF04FF93A46014600204DF00AFD1D
:106450006E4B1888BDF9543000F2DC50184440F2FD
:106460006C7240F24C4100B21AF03CF93A460146D7
:1064700001204DF0F7FCB8EECAAAF8EEE88A40F227
:106480006C72EAEE2A8A40F24C4104F54054FDEE6B
:10649000E88A18EE903A18B21AF024F93A46014602
:1064A00002204DF0DFFCBDF9403007EE103AB8EEA7
:1064B000C77AF0EE487AE7EE097A40F26C7240F261
:1064C0004C41FDEEE77A17EE903A18B21AF00AF94D
:1064D0003A46014603204DF0C5FC94F81136002BD6
:1064E00067D1F8EEE99AF0EE487AE9EE897A40F25F
:1064F0006C7240F24C41FDEEE77A17EE903A18B21A
:106500001AF0F0F83A46014604204DF0ABFC07EED5
:1065100090BAF8EEE77A40F26C72A7EE898A40F200
:106520004C41BDEEC88A18EE103A18B21AF0DAF8EB
:106530003A46014605204DF095FC324BD3ED007AEA
:10654000FDEEE77A3A4617EE903A062019B24DF082
:1065500089FC2B4BD3ED007AFDEEE77A3A4617EE35
:10656000903A072019B24DF07DFC2B4B1E802B4B2F
:106570001D802B4BA3F80090BDEC068BBDE8F88F77
:10658000002B3FF4FBAE5A462046FFF73DF8F5E6F8
:106590000288B8F800B011440AB20AEE102ABAF81C
:1065A00000203244AB4412B209EE902A0FFA8BFB62
:1065B0003CE7BAF9003007EE103AB8EEC77AF0EED1
:1065C000487AE7EE097A40F26C7240F24C41FDEEF7
:1065D000E77A17EE903A18B21AF084F83A46014674
:1065E00004204DF03FFCB8F9003007EE903A90E7F8
:1065F000CDCC4C3FCDCCCC3E0080BB440000FA4318
:106600000822002004220020467A0020447A00203C
:1066100000220020347A0020367A0020387A0020C8
:106620003A7A00202C7A0020327A0020307A00203A
:1066300001207047002070470020704700207047FD
:1066400000207047002070479FED010A704700BF8F
:106650000000000070470000144A0260144A4260C3
:1066600002F1B80181601349C160A2F6786101614D
:1066700002F64851416102F50561816102F654015B
:10668000C16102F65801016202F65C01416202F545
:10669000066102F66402C262074A0263A2F2044281
:1066A0004263064A81628263704700BF34B20B08BE
:1066B00010460020005C0020DC600020B82600208E
:1066C000152938D8DFE801F00F1317232737372BA8
:1066D000372F3737373737371F37370B331B00F52F
:1066E000A3403430704700F5A3407030704700F588
:1066F000A4402C30704700F5A4406830704700F586
:10670000A8400C30704700F5A6401C30704700F5DB
:10671000A5402430704700F5A5406030704700F573
:10672000A6405830704700F5A7401430704700F578
:10673000A7405030704700207047000000F5A0408F
:10674000D0F8B00103685B681847000038B500F561
:10675000A0450446D5F8B00103685B6998470A4B29
:1067600004F50052187492F8802DD5F8B001DA7053
:1067700003681B6A9847014604F58C501430BDE845
:10678000384035F07DB900BF4D7B00202DE9F04742
:1067900000F50059064699F8803D8B420F46924617
:1067A00005D189F81C2001252846BDE8F087FFF7B0
:1067B00087FF044620B9304640F0EAFB2546F3E760
:1067C00003689B68984706F52D5808F13808A8B16A
:1067D0002C4804F023F9054680B923682046DB697C
:1067E0009847294A03460421404645F0D3FC42F02D
:1067F00009FC3A460A2142F0BDF9D5E72148FBF7EA
:10680000E7F808B3236800211B682046984705462F
:1068100088B399F8803D89F8813D06F5A04306F5D7
:106820002350C3F8B0415246394689F8807D89F833
:106830001CA0083041F0AEFD404600214CF082FA29
:106840003046FFF783FFAFE706F5A043D3F8B0016A
:106850000368DB6898470028D4D023682046DB68AB
:10686000984705460028CDD123682046DB69984724
:10687000064A0346B7E723682046DB699847044A7F
:106880000346B0E7B0250020BCB10B08E5B10B080A
:106890000EB20B080148FFF779BF00BFB0250020FA
:1068A0002DE9F04F07EE902A2DED048BF8EEE78AE4
:1068B00007EE901AB8EEE78A91B028EE080A4FF07A
:1068C000000BA8EEA80A0646884615461F46CDF8D6
:1068D00004B0CDF808B0CDF80CB0CDF810B0CDF8BC
:1068E00014B0CDF818B099F06FFADFEDC89AB4EE95
:1068F000E90AF1EE10FA10DDC9EE807A27EE888AF7
:1069000067EEA87ABDEEC88AFDEEE77A18EE103A77
:106910000FFA83F817EE903A1DB2736807EE908A6B
:1069200093ED2B7AB8EEE79AB5EEC07A07EE905A5F
:10693000F1EE10FAF8EEE75A00F2B18093ED268AF4
:1069400028EE099A28EE258A736807EE907A93ED6F
:10695000270A93F9A830F8EEE78A68EE808A002BC0
:1069600000F08F803369D3F8F00119F045FEA84993
:1069700040F6B832814619F0A5FE434207EE903A40
:106980007368F8EEE77A93ED287A336967EE877AD1
:10699000D3F8F401CDED017A19F02EFE40F6B832AD
:1069A0009B49824619F08EFE42427368CDF80CB0C6
:1069B00007EE102AD3ED296A93F9A820B8EEC77A1A
:1069C000022A27EE267A8DED027A20D1914AB2F979
:1069D0005C404C4580F29080A9EB040907EE909A48
:1069E000D3ED285AB8EEE76ADDED017AE5EEC67A16
:1069F000CDED017A544580F29180AAEB040407EEB4
:106A0000904AF8EEE77AA6EEE77A8DED027AD6F8AC
:106A100034A09FED810A0AF148001CF071F910AB17
:106A20008DED0D0ACDED0E0A8DED0F1A13E907005D
:106A30000DF1280907AC89E8070084E807009FEDFD
:106A4000770A20461CF05CF904AB01AA494650467F
:106A50008DED0A0ACDED0B0A8DED0C1A64F02CFABF
:106A6000736893F9A830022B5ED1DDED047A39EE1C
:106A7000279ADDED057A38EE278ADDED067A78EE85
:106A8000A78A1E9B83ED009A1F9B83ED008A209BA3
:106A9000C3ED008A11B0BDEC048BBDE8F08FF7EEBA
:106AA000007AB4EEE77A89EE297A85EEA98AF1EECA
:106AB00010FAC8BFC3ED2B7A7368D3ED2B6A93ED40
:106AC000260A77EEE67A27EE076A27EE879A26EE01
:106AD000076A28EE087A67EE887A27EE087AA6EE2B
:106AE000869AE6EE877A29EE299A27EEA98A29EE78
:106AF000009A28EE008A27E762424A457FF77AAF7C
:106B0000A14407EE909A9DED016AD3ED285AF8EE64
:106B1000E77AA5EEE76A8DED016A6BE763425345BC
:106B20007FF775AF54446AE7002D88EAE871B8BF73
:106B30006D42A1EBE87189B2ADB2A942D4BF224641
:106B40006A460091002F0795B8BF7F421368DFEDBA
:106B5000340ABFB29F42A8BF4A460A97D2ED007AD4
:106B6000F8EEE77AB7EE001A87EEA90A4FF48270C2
:106B700031EE400A19F078FD3369D3ED917A04A81B
:106B800020EE270A1CF0BCF8F0EEC07A8DED061A54
:106B9000B0EEC91A31EE671A8DED040AB0EEC11AD3
:106BA00030EE090ACDED050A4FF48670F1EE410A88
:106BB00019F05AFDB0EE409A9DED050AB0EEC81AE4
:106BC000F0EEC07A31EE671A30EE080AB0EEC11A64
:106BD000F1EE410A40F2111019F046FDB0EE408A84
:106BE0009DED060AB0EEE81AF0EEC07A31EE671AB3
:106BF00038EE800AB0EEC11A4FF48B70F1EE410A04
:106C000019F032FDF0EE408A3BE700BF00A08C4552
:106C100048F4FFFFB04500209F0CB345D30237393D
:106C2000000000000148FFF7B1BD00BFB025002003
:106C3000004870472851002000207047012070470D
:106C40000120704700207047004870476CB20B0865
:106C5000004870476CB20B0808B5036B034800226C
:106C6000C3F84C23FEF7E0FD012008BDB02500204D
:106C700070B50446406990F8D33088B093B90121CB
:106C800069F03EFB606B62680368D2ED020A9B6D9F
:106C90009FED240A01219847606B08B0BDE8704061
:106CA00064F0EABC022169F02BFB636AE269A16926
:106CB0001B6812680968B2F90820B1F90810B3F925
:106CC000083007A8029006A8019005A80090204669
:106CD000FFF7E6FD606B9DED071A0368DDED060A20
:106CE0009DED050A9B6B9847656B2B689E6D236A2B
:106CF00018684DF019FA63680021D3ED020A28469E
:106D0000B047A36A656918684DF00EFA85ED0E0A62
:106D1000E36A656918684DF007FA85ED0F0A08B057
:106D200070BD00BF000000000020704700207047C9
:106D3000012070470020704700487047B4B20B082C
:106D400000487047C0B20B0870B504462148FAF7F6
:106D50003FFE054600283AD01E48266BFBF73AF95D
:106D60006368B3F92C20B3F9283000EE903A43421F
:106D700001EE102A00EE103AB8EEC11AF8EEE00A61
:106D8000B8EEC00A304665F083FC1248266BFBF76C
:106D900021F96368B3F92C20B3F9283000EE903A5A
:106DA000434201EE102A00EE103AB8EEC11AF8EE96
:106DB000E00AB8EEC00A304665F0E4FC206B66F0ED
:106DC000CBFB2369D3F8F821034BC3F89C21284659
:106DD00070BD00BFB0250020B075002070B52DED4E
:106DE000028B8AB004466DF041FF06467348256B5E
:106DF000FBF7F0F86368B3F92C20B3F9283000EE04
:106E0000903A434200EE103A01EE102A2846B8EEBE
:106E1000C11AF8EEE00AB8EEC00A65F039FC606904
:106E2000674D90F8D330EBB9012169F069FA606BD6
:106E300062680368D2ED020A9B6D0121B6EE000A7A
:106E40009847606B64F018FC6069266B0368DB6828
:106E50009847304666F0E8FB2369D3F8F831C5F867
:106E60009C3190E0022169F04BFAD5F86C3141F287
:106E70008732F31A934233D8D5F874310693D5F894
:106E800078310793D5F87C310893D5F88031099390
:106E900003A905AB06A804AA1BF080FC9FED497A64
:106EA000DDED037ADDED040A9DED051A606B9FEDC3
:106EB000460A67EE877A60EE870A21EE071ACDED63
:106EC000040A8DED051ACDED037A036821EE001A50
:106ED00060EE800ADB6A27EE800A0121984752E0C3
:106EE000A369606B1B68B3F9083008EE103AE369D8
:106EF0001B68B3F9083000EE903A0368F8EEE00A38
:106F0000DB6DCDED010A9847B8EEC88AB0EE401AA5
:106F1000DDED010AB0EE480A04AA03A9A5F5A040D8
:106F2000FAF750FF636A1868438A828907EE903A3D
:106F3000264BF8EEE77A93ED007A67EE877AFCEE5F
:106F4000E77A17EE903A99B24DF084F80146A5F52C
:106F5000A040FAF7A1FFDFED1E7A606BB0EEC07AB9
:106F6000B4EEE77AF1EE10FAB0EE401A0FD40368EF
:106F7000DDED040A9B6A9DED030A98472369D3F867
:106F8000F831C5E967360AB0BDEC028B70BDD5F8A3
:106F9000A03102689DED030ADDED040AFA33B34225
:106FA00004D9936A9FED0B1A984755E795ED671A38
:106FB000D36AB8EE411A012190E700BFB025002046
:106FC000B0750020E02E65420000C842BC5B002086
:106FD000000000340000000038B5836A45690446AB
:106FE00018684DF0A1F885ED0E0AE36A6569186826
:106FF0004DF09AF885ED0F0A38BD000030B52DED43
:10700000028B036A1B68B3F9083000EE103A83B0B4
:107010000446B8EEC00A2F48FAF7EEFF2D488DED72
:10702000010AFAF7D7FF63689DED010AB3F928302A
:1070300001EE103A434200EE903AB8EEC11AF8EE73
:10704000E00A6C2019F010FBDFED237AB0EEC07A75
:10705000B4EEE77AF1EE10FAB0EE408A19D51F4B84
:10706000256B93F87C2D93F97C3D002B1EDA636829
:1070700095EDD37AD3ED2C7AF1EE046A77EEE67AC9
:10708000F4EE477AF1EE10FAC8BFF0EE477AC5ED9C
:10709000D37A206BB0EE480A65F0C4FB206B03B0D6
:1070A000BDEC028BBDE8304066F014BB5306F0D552
:1070B000E06868F077F8236BF2EE047A30EE270A86
:1070C000D3EDD37AB4EE670AF1EE10FAC8BFF0EE52
:1070D000407ADCE7B0250020CDCC4C3DB045002007
:1070E00010B50446FFF77AFE2046FFF787FF2046DB
:1070F000BDE81040FFF770BF0120704700207047C7
:1071000001207047012070470048704708B30B0802
:107110000048704708B30B0830B5054685B01748DE
:1071200003F07CFC044620B3154BB3F8B42A012AC3
:1071300022D903F5405203F58053042193F82436F5
:1071400082F85414022B03D10021284600F020FFBE
:10715000DFED0C0A0C48B0EE601AF0EE601AB0EEEB
:10716000600A67F0D3FB284600F008FF07481EF0CE
:107170003FFD204605B030BD0024FAE7B0250020D1
:10718000B0450020000000008C6400203450002036
:1071900070B5134D04460026124885F8546467F014
:1071A0001BFB60B92046FFF743FD0F4A042144F062
:1071B000F1FFA5F5A040BDE87040FEF7DBB8A5F5EE
:1071C000005595F82436022B09D03146204600F0B0
:1071D0002BFE01462046BDE8704000F0D9BE70BDD0
:1071E000B07500208C64002010B30B08094901F52C
:1071F000A043022283F8542401F5804303F5016281
:1072000001F5904192ED000A93F83428A1F11C0099
:1072100066F0D2BCB025002070B52DED028B04467F
:10722000B0EE408A4948DFED4A8A8EB00D461646D8
:1072300066F050FBF0EEC87AF4EEE87AF1EE10FA60
:1072400006D49FED440A414828EE000A66F0A8FBE8
:10725000414B93ED000AB0EEC00A0EB1B1EE400A08
:107260003A4866F08DFB002307A938480793089336
:10727000099366F0A5FBE06867F090FF07A91BF093
:1072800029FD0AA88DED0A0ACDED0B0A8DED0C1A29
:107290001CF034F9DFED317AB4EEE70AF1EE10FAC2
:1072A00050DD2F4E0123022207A90AA886F8543484
:1072B0000CF090F86968019128460BF007FE0199DF
:1072C00002460AA80BF0D8FD26480AA967F084FAFE
:1072D00018B9A6F5A040FEF74DF8E068224D67F01A
:1072E0005FFF03A9026843680392284604931AF0DB
:1072F00085FC05A88DED050ACDED060A1AF04CFDBA
:10730000D5ED037AF4EEE87AF1EE10FAB8BF55ED58
:10731000037AF4EEC07AF1EE10FA4FF00001204645
:107320000AD5DFED127AB4EEE70AF1EE10FA03DDCA
:1073300000F07AFD0146204600F02AFE0EB0BDECBA
:10734000028B70BD2046FFF751FFF7E7946D0020D8
:10735000000000340000C842C06D002000009643C9
:10736000B07500208C640020B06D00200000FA434E
:1073700037B59FED1A0A1A4D04461A4866F0B6FC56
:1073800001462846FDF734FD694601AA284602F069
:10739000A1FD6369009ADA636369019A9A63206BBD
:1073A00066F098F9E369606B1B68B3F9083000EE8A
:1073B000903AA3691B68B3F9083000EE103A0368ED
:1073C00005F59045DB6A95ED051AF8EEE00AB8EE92
:1073D000C00A0121984703B030BD00BF0000000083
:1073E000B0250020946D0020F0B52DED028B0446F1
:1073F000406B264D85B0F0EE408A48309FED240A60
:10740000B0EE608A0E4617461BF07AFCDFED217A5B
:107410008DED031AF7B928EEA70A19F0B9F89FED18
:107420001E7ABDEEC00AF0EEC87A10EE103AF4EE05
:10743000C77AF1EE10FAC5F83C3618D53C23032183
:107440002046A5F8403605B0BDEC028BBDE8F04003
:1074500000F09EBD9DED030ABDEEC00A002EB8EE01
:10746000C00AB8BFF1EE688AA8EEA70AD5E7DFED3B
:107470000B7AB4EEE78AF1EE10FA58BFB0EE678AE5
:10748000BDEEC88A18EE103AD9E700BFB05500200B
:107490009F0CB3450000C842000000340000704259
:1074A000DFED097A094BB4EEE70AF1EE10FA58BFA6
:1074B000B0EE670ABDEEC00A072110EE102AA3F84D
:1074C000402600F065BD00BF00007042B0550020AE
:1074D00010B54A6804460B465AB98A684AB9C96861
:1074E00039B900F0A1FC01462046BDE8104000F08B
:1074F0004FBD044918460BF03BFE08B10221F3E7EB
:1075000010BD00BFD85B0020F8B5192105462648FC
:1075100038F0C4FA0238022844D8244C052384F8F1
:1075200054346DF0A3FBC4F8A40121481CF04CF8BE
:10753000A4F5046200231360A4F64402A4F66C00D0
:10754000136067F03BFC68692E6B0368A4F5005478
:10755000DB68984704F60C77304604F6F86604F6C4
:10756000FC6466F061F894ED000A97ED001AD6ED20
:10757000000A286BB0EEC00A65F08AF894ED000AA4
:1075800097ED001AD6ED000A286BB0EEC00A65F040
:10759000F9F82846FFF74CFB064A042144F0FAFDAF
:1075A0000120F8BD0020FCE7F8320020B075002073
:1075B000345000203CB30B0870B52DED028B04460F
:1075C000406990F8D33084B0FBB9012168F098FE8F
:1075D000606B62680368D2ED020A9B6D9FED6C0AD6
:1075E00001219847606B64F047F86A4867F0E6FB52
:1075F0006069256B0368DB689847284604B0BDECDA
:10760000028BBDE8704066F00FB86348634D1921E6
:1076100038F044FA032865D004286DD00228604E63
:1076200040F0A58005F57B55002395ED0E8A33606B
:107630005C4D6DF01BFBD5F8A43103F51C531033E2
:1076400098420AD92046FFF7F3FA574A022144F03C
:10765000A1FDA5F5A040FDF765FE4E48012167F0AC
:1076600037FD694601AA4D4802F0EEFB6369009AB6
:10767000DA636369019A9A63B0EE480A206B9FED62
:10768000448A65F0CFF8206B66F024F847488DED0A
:10769000028AB0F95C308DED038A01EE103AE3699D
:1076A0001B68B3F9083000EE903AA3691B68B3F980
:1076B000083000EE103AB8EEC11AF8EEE00AB8EE63
:1076C000C00A03AA02A9A0F50050FAF77BFB606B81
:1076D000DDED030A03689DED020A9B6AB0EE481ACD
:1076E000984750E005F57B5595ED0F8A2C4B00220D
:1076F000B0EEC88A1A609BE705F5005595F8FC398D
:107700009B0731D5264D2B6853B96DF0AFFA286031
:107710006069266B0368DB689847304665F084FF34
:107720006DF0A4FA2B6803F2DC5398421CD9204672
:10773000FFF77EFA1E4A062144F02CFD174801216E
:10774000FDF756FB194890F8A03D6FF3C30380F88E
:10775000A03D00F54053042200F6842083F8542411
:107760001EF0D8F900232B609FED098A60E72046C0
:10777000FFF75EFA0F4A022144F00CFD2846FDF7A0
:10778000D1FD0023336004B0BDEC028B70BD00BF9F
:1077900000000000446D0020F8320020B0250020D9
:1077A0004C7A0020B0750020B9B30B08B04500201A
:1077B00060B30B0886B30B0830B5054685B00F489B
:1077C00003F02CF90446A8B10D4B0E48042283F8AF
:1077D00054240DEB0201002301930293039366F0FE
:1077E0003DFC01A90748002267F070F900212846F6
:1077F00000F0CEFB204605B030BD00BFB025002014
:10780000B07500208C64002070B52DED028B04460D
:10781000406990F8D33088B03BBB012168F070FD1F
:10782000606B9FED508A62680368D2ED020A9B6D1F
:10783000B0EE480A01219847606B63F01DFF4A488B
:107840008DED058AF0EE480AB0EE481AF0EE481ABF
:10785000B0EE480A8DED068A8DED078A08B0BDECC2
:10786000028BBDE8704067F051B8404E96F8A01DFD
:1078700011F001055DD1636A1B68A6F50050B3F9EC
:107880000810FAF709FBDFED3A7AB0EEC07AB4EEF1
:10789000E77AF1EE10FAB0EE408A03D4294620468A
:1078A00000F076FB0221606968F02AFD2E4866F040
:1078B00013FF01462F48FDF79BFA02A92D4803AAA2
:1078C00002F0C2FA6369029ADA636369039A9A63FF
:1078D000206B65F0FFFEB6F95C30264801EE103AE9
:1078E000E3691B68B3F9083000EE903AA3691B689E
:1078F000B3F9083000EE103AB8EEC11AF8EEE00A1B
:10790000B8EEC00A05AA04A9FAF75CFA1A4B656B2F
:1079100093F8243683B92B68DDED050A9B6A9DED4B
:10792000040AB0EE481A2846984708B0BDEC028B0E
:1079300070BD9FED0C8AB5E72B68DDED050A9DED66
:10794000048ACDED010A2046DE6A00F0E1FDDDED9E
:10795000010AB0EE401A0121B0EE480A2846B047AD
:10796000E3E700BF000000008C640020B045002069
:1079700000000034B0250020B055002030B52DEDBA
:10798000028B0446406990F8D33087B03BBB01219D
:1079900068F0B6FC606B9FED3C8A62680368D2EDCC
:1079A000020A9B6DB0EE480A01219847606B63F0B4
:1079B00063FE36488DED038AF0EE480AB0EE481AB1
:1079C000F0EE481AB0EE480A8DED048A8DED058A76
:1079D00007B0BDEC028BBDE8304066F097BF2C4D80
:1079E00095F8A03DDB074BD4636A1B68A5F50050F2
:1079F000B3F90810FAF750FAB0EE408A6069022134
:107A000068F07EFC214866F067FE01462148FDF7DC
:107A1000EFF9694601AA1F4802F016FA6369009A55
:107A2000DA636369019A9A63206B65F053FEB5F9D6
:107A30005C30184801EE103AE3691B68B3F908306E
:107A400000EE903AA3691B68B3F9083000EE103AD3
:107A500003AA02A9B8EEC11AF8EEE00AB8EEC00A0D
:107A6000FAF7B0F9606BDDED030A03689DED020AD9
:107A70009B6AB0EE481A984707B0BDEC028B30BD48
:107A80009FED018ABAE700BF000000008C6400206F
:107A9000B0450020B025002008B50748012101F0BD
:107AA0009BF8064B032283F8542403F52970BDE8A4
:107AB000084000F0E1BF00BF90780020B0750020C2
:107AC00010B5044613481DF02FFF134B93F85434A0
:107AD000052B1DD8DFE803F00303080D121720461D
:107AE000BDE81040FFF790BE2046BDE81040FFF70C
:107AF0003FBCBDE81040094801F03CBA2046BDE853
:107B00001040FFF73BBF2046BDE81040FFF754BDD3
:107B100010BD00BF34500020B075002090780020C8
:107B200001207047002070470120704701207047F6
:107B3000004870471CB40B080048704724B40B0879
:107B4000F0B55C4DDFED5C0AD5ED047A95ED000AE9
:107B50002DED028BDFED598AF4EEE87AF1EE10FAA2
:107B60000446A8BFF0EE670A83B0006BA5F6F46682
:107B700064F0AEFCA6F54050276BFAF72BFA636869
:107B8000B3F92C20B3F9283000EE903A434200EECE
:107B9000103A01EE102A3846B8EEC11AF8EEE00AA3
:107BA000B8EEC00A64F074FD606990F8D330C3B9D0
:107BB000012168F0A5FB606B62680368D2ED020AE0
:107BC0009B6D9FED3F0A01219847606B63F054FD68
:107BD00005F50F6003B0BDEC028BBDE8F04066F028
:107BE00007B8636A37481B68B3F90810FAF754F905
:107BF000F0EEC07AF4EEE87AF1EE10FA5CBF012301
:107C000086F8F030236A2F481B68B3F90830B0EECD
:107C1000408A00EE103AB8EEC00AFAF7EDF90221F8
:107C20006069F0EE408A68F06BFB9FED250A2648FC
:107C300066F05CF801462348FDF7DAF8214801AA0E
:107C4000694602F047F96369009ADA636369019A49
:107C50009A63D4E9063212681B68606BB3F9083086
:107C6000B2F9082096F8F01000EE103A00EE902AD3
:107C7000036899B19B6AF8EEE00AB8EEC00AB0EE6C
:107C8000481A9847206BB0EE680A64F0CBFD206B71
:107C900065F020FD03B0BDEC028BF0BD0B4ADB6A42
:107CA00092ED001AF8EEE00AB8EEC00A01219847FA
:107CB000E8E700BFA464002000007A43000000341D
:107CC00000000000B0250020946D0020C46D00204D
:107CD0002DE9F04104462DED028B354802F09EFE61
:107CE000064600285FD0334DDFED338A9FED338A9F
:107CF00005F60478D8ED000A0023F4EEE80A85F8CA
:107D0000F030F1EE10FA05F6F46797ED000A206BFB
:107D1000B8BFF0EE480A64F0DBFBD8ED000A97ED3F
:107D2000000A206BF4EEE80AF1EE10FAB8BFF0EEAC
:107D3000480A64F045FCA5F54050276BFAF74AF96C
:107D40006368B3F92C20B3F9283000EE903A43422F
:107D500001EE102A00EE103AB8EEC11AF8EEE00A71
:107D6000B8EEC00A384664F093FCA5F54050276B86
:107D7000FAF730F96368B3F92C20B3F9283000EE34
:107D8000903A434201EE102A00EE103A3846B8EE1F
:107D9000C11AF8EEE00AB8EEC00A64F0F3FC08F588
:107DA0000E6065F025FFBDEC028B3046BDE8F0812A
:107DB000B0250020B05500200000003400007A43B8
:107DC0000120704700207047012070470120704754
:107DD000004870476CB40B080048704774B40B0837
:107DE00090ED007ADFED0F7AB0EEC77AB4EEE77A65
:107DF000F1EE10FA14D590ED017AB0EEC77AB4EE38
:107E0000E77AF1EE10FA0BD590ED027AB0EEC77A70
:107E1000B4EEE77AF1EE10FA4CBF01200020704773
:107E20000020704700000034436893F92530042B8C
:107E30000BD8DFE803F00C0A0503080004207047A4
:107E400081F0010070470620704701207047002034
:107E50007047000038B52DED048B0446406990F85A
:107E6000D330B3B9012168F04BFA606B62680368E4
:107E7000D2ED020A9B6D9FED3D0A01219847606B90
:107E800063F0FAFBBDEC048B206BBDE8384065F075
:107E900063BB374D95ED028AD5ED018A28EE080ABD
:107EA000A8EEA80A97F090FF606B0368DB6DB0EE58
:107EB000409A98472F4BB3F95C3007EE903AF8EEB2
:107EC000E77AB4EEE70AF1EE10FA58BFB0EE670AAF
:107ED000B4EEC90AF1EE10FA48BFC0EE097A95ED8A
:107EE000030A44BF28EE278A68EEA78A18F066FBCB
:107EF000214BD3ED010A93ED001AF0EEE00AF1EE0A
:107F0000600AF0EE409A4FF42F7095ED040A18F0D5
:107F1000ABFBB0EE409A6CF0A9FE2B68C01AB0F52E
:107F20007A7F88BF9FED118A60694FF0020184BF9C
:107F3000B0EE489AF0EE488A68F0E2F9606B0368A8
:107F4000B0EE691ADB6AF0EE480AB0EE680A012169
:107F50009847206BB0EE490A64F064FCBDEC048BDA
:107F6000206BBDE8384065F0B5BB00BF00000000E5
:107F7000547A0020B0450020A8640020034B002262
:107F80001A6000225A609A60DA607047807A002096
:107F90000C4B93F824268A420FD0022983F824162A
:107FA00002D004290AD0704703F234630269D2ED8B
:107FB0007E7AF8EEE77AC3ED007A704703F2446305
:107FC000F4E700BFB05500202DE9F0412DED048B02
:107FD00082B088461446F0EE608A0193B0EE408A83
:107FE000074605F089FC9FED279A90ED810A264D02
:107FF00018F010FB28EE098AF0EE409AB0EE480A1D
:1080000018F008FB30EE690A18F01AFBB5EEC00A4A
:10801000F1EE10FA4CBF4FF0FF360126B8F1000F19
:1080200016D0019A71B26CB9DFED180A85F82546B1
:108030001748B0EE480A02B0BDEC048BBDE8F04131
:10804000FFF7D2B9002368EE890A85F82536EFE7F5
:1080500064B128EE890A0E48012385F8253602B05E
:10806000BDEC048BBDE8F041FFF71ABA2146384653
:1080700085F8254602B0BDEC048BBDE8F041FFF762
:1080800087BF00BF0AD7233CB05500200000000086
:108090005478002070B5224D05F5A0430122044616
:1080A00083F85524066B2846F9F794FF6368B3F903
:1080B0002C20B3F9283000EE903A434201EE102A0A
:1080C00000EE103AB8EEC11AF8EEE00AB8EEC00AB7
:1080D000304664F0DDFA2846266BF9F77BFF6368CB
:1080E000B3F92C20B3F9283000EE903A434201EE68
:1080F000102A00EE103AB8EEC11AF8EEE00AB8EE17
:10810000C00A304664F03EFB206B65F025FA206B18
:1081100065F03AF820460021BDE87040FFF738BF0F
:10812000B025002038B50A4B93F85534012B05468D
:108130000C4601D0FFF7AEFF6CF098FD054B1860C0
:1081400094E807002B6B03F5547383E8070038BDF0
:10815000B0750020507A002030B50C4611461A4602
:10816000134B93F85534012B85B005460DD0CDED5A
:10817000030A02928DED010A0091FFF78BFFDDEDFE
:10818000030A029A9DED010A00999DF820302846C5
:10819000FFF71AFF6CF06AFD064B186094E80700C1
:1081A0002B6B03F5547383E8070005B030BD00BFA7
:1081B000B0750020507A0020F8B5184B03F5A042A6
:1081C00003F5405303F6FC64022194ED000A82F8A3
:1081D000551403F60C7703F6F866054697ED001A7A
:1081E000D6ED000A006BB0EEC00A64F051FA94EDCF
:1081F000000A97ED001AD6ED000A286BB0EEC00A0F
:1082000064F0C0FA286B65F0A7F9286B64F0BCFF36
:1082100028460021BDE8F840FFF7BABEB02500208F
:108220002DE9F0472DED028B2D4B93F85534022BA1
:1082300088B081460C46154601D0FFF7BDFF0222EB
:10824000214604A80BF0C6F8264804A954F092FC75
:10825000804658B940F0D6FE0522162140F08AFC2F
:10826000404608B0BDEC028BBDE8F0876CF0FEFC28
:108270001D4B1E4E216862681860A368B3603160B0
:10828000726095E807001A4F9FED1A8A4FF0010AB5
:1082900087E8070002ABD9F83000CDF800A03A46D5
:1082A00031468DED028A8DED038A64F091F9B36851
:1082B000D9F83000029307F10802534602A9B0EE44
:1082C000480A64F0D5FE0648029B90F85514B36046
:1082D00022462B46A0F5A040FAF7FEFFC0E700BFFC
:1082E000B075002010450020507A0020687A0020E8
:1082F000747A0020000000002DE9F0472DED028B7C
:108300001E46354B93F85534022B88B007460C4671
:108310001546B0EE408AF0EE608A01D0FFF74CFFC0
:108320000222214604A80BF055F82C4804A954F069
:1083300021FC814658B940F065FE0522162140F027
:1083400019FC484608B0BDEC028BBDE8F087F0EEA2
:10835000680AB0EE480A9DF84C309DF84820DFF8D6
:108360008C809FED1F8A31463846FFF72DFE6CF05A
:108370007DFC1C4B1C4E216862681860A368B360CA
:108380003160726095E807004FF0010A88E8070045
:1083900002AB386BCDF800A0424631468DED028A23
:1083A0008DED038A64F014F9B368386B029308F119
:1083B0000802534602A9B0EE480A64F059FE064886
:1083C000029B90F85514B36022462B46A0F5A040BE
:1083D000FAF782FFB5E700BFB07500201045002016
:1083E00000000000507A0020687A0020747A002093
:1083F000F8B5234B03F5A04203F5405303F6FC64A4
:10840000032194ED000A82F8551403F60C7703F665
:10841000F866054697ED001AD6ED000A006BB0EE3F
:10842000C00A64F035F994ED000A97ED001AD6ED14
:10843000000A286BB0EEC00A64F0A4F9286B65F05E
:108440008BF86CF013FC2A690E4BD2ED7C7A186025
:10845000F8EEE77A2846C3ED017AD2ED7D7AF8EEA0
:10846000E77A0021C3ED027AD2ED7E7AF8EEE77A60
:108470000022C3ED037A1A61BDE8F840FFF788BD1A
:10848000B0250020547A002038B52DED028B1C4B0E
:1084900093F85534032B0D46B0EE408A01D0FFF718
:1084A000A7FF184C284604F10C0304F10802211D13
:1084B0001AF074F9DFED146AD4ED017A9FED137AA6
:1084C00094ED030A67EEA67A20EE260A67EE877A15
:1084D00020EE070AC4ED017AD4ED027A67EEA67A9F
:1084E00067EE877AC4ED027A18F068F884ED048AA2
:1084F00084ED030A6CF0BAFBBDEC028B206038BD42
:10850000B0750020547A0020E02E65420000C84279
:1085100010B52DED028B3C4B93F82426023A82B025
:108520000446042A6BD8DFE802F0030B151D200077
:10853000364802B0BDEC028BBDE81040F9F7D0BC64
:1085400003F23C6393ED000AB8EEC00A02B0BDEC42
:10855000028B10BD2D4802B0BDEC028BBDE810406F
:10856000F9F7E2BC93ED3D0AEEE72949DFED298AF0
:10857000A1F10C0018F030FA236B6846D3F85C23A5
:10858000D3F860330193B0EE408A009219F004FCF6
:10859000236B9FED217AD3EDC57A67EE877AB4EE2F
:1085A000E70AF1EE10FA27DB684619F0ABFBDFEDC6
:1085B0001B7A20EE270AF0EE487AD0EE287AB0EE49
:1085C000670A17F0FBFF636893F9243007EE903ACF
:1085D0005B4200EE903AB8EEE71AF8EEE00A21EEC0
:1085E000281A60EEA80A4FF44C7018F03DF838EEE7
:1085F000000A17F0CDFFA9E79FED090AE3E7D3F8DA
:10860000EC3E93EDCF0AA1E7B0550020B025002045
:10861000146D00200000C842CDCCCC3DE02E654258
:108620000000000070B52DED028B0446406990F803
:10863000D33084B0D3B9012167F062FE606B626809
:108640000368D2ED020A9B6D9FED6C0A01219847E9
:10865000606B63F011F8206B64F07EFF206B04B058
:10866000BDEC028BBDE8704064F08EBD644890F8AC
:10867000A01D11F0010500F580566BD1636A1B68DF
:10868000A0F50050B3F90810F9F706FCDFED5D7AAC
:10869000B0EEC07AB4EEE77AF1EE10FAB0EE408AAE
:1086A00051D429462046FFF773FC6069022167F028
:1086B00027FE6CF0DBFA544B1B68C01A40F6B83347
:1086C00098420CD9256B05F55470FFF789FB30B93A
:1086D0000023C5F85033C5F85433C5F85833206B20
:1086E00063F0BCFF206B64F039FE206B90EDD60A7E
:1086F00064F098F8206B64F0EDFF03AA02A94348E8
:1087000001F02EFC6369029ADA636369039A9A6343
:1087100096F82436656BD4E90612F3B91368B3F9F9
:10872000083000EE903A0B68B3F9083000EE103ACA
:108730002B68F8EEE00A9B6AB8EEC00AB0EE481A61
:108740002846984735E096F825360BB10721A9E76A
:108750000321A7E79FED298AA7E709681268B1F905
:108760000810B2F9082008EE101A00EE902A032B28
:10877000B8EEC88AF8EEE00A1FD1B6F94036DFED50
:10878000247ACDED010A01EE903AF8EEE11A204686
:1087900061EEA71ACDED001AFFF7BAFEDDED001A63
:1087A000DDED010AB0EE401A2846B0EE480A61F04D
:1087B0004FFE04B0BDEC028B70BD072B2A680DD1B3
:1087C000B6F940369FED121A07EE903AF8EEE77AC6
:1087D000936A27EE811AB0EE480AB1E72046CDED44
:1087E000000AD66AFFF794FEDDED000AB0EE401AEB
:1087F0000121B0EE480A2846B047DAE70000000041
:10880000B045002000000034507A0020B025002040
:108810000000C842F0B52DED028B0446406990F887
:10882000D3308DB0D3B9012167F06AFD606B626807
:108830000368D2ED020A9B6D9FED800A01219847E3
:10884000606B62F019FF206B64F086FE206B0DB048
:10885000BDEC028BBDE8F04064F096BC78489FED1B
:10886000778A90F8A01D11F0010500F5805640F0C0
:108870009180636A1B68A0F50050B3F90810F9F7FE
:108880000BFBDFED707AB0EEC07AB4EEE77AF1EE72
:1088900010FAF0EE408A76D429462046FFF778FB9E
:1088A0006069022167F02CFD6CF0E0F9664B1B68F3
:1088B000C01A40F6B83398420AD9644D2846FFF7EB
:1088C0008FFA28B985ED028A85ED018A85ED008A47
:1088D000236B5E4893EDC20A5D4D1AF011FA012731
:1088E00009A92846CDED070A8DED081ACDED0A0A33
:1088F0008DED0B1A8DED060A8DED090A1AF020FA9E
:108900002946524A206B009709AB8DED098A8DEDFF
:108910000A8A63F05DFEAB689FED480A4D4A206B02
:10892000059305A93B4664F0A3FB059B206BAB6058
:1089300064F014FD206B64F0CDFE09AA06A9464838
:1089400001F00EFB6369069ADA636369099A9A6318
:1089500096F82436656BD4E90612F3B91368B3F9B7
:10896000083000EE903A0B68B3F9083000EE103A88
:108970002B68F8EEE00A9B6AB8EEC00AB0EE681AFF
:108980002846984735E096F825360BB1072184E74D
:10899000032182E7F0EE488A82E709681268B1F99C
:1089A0000810B2F9082008EE101A00EE902A032BE6
:1089B000B8EEC88AF8EEE00A1FD1B6F94036DFED0E
:1089C000277ACDED030A01EE903AF8EEE11A20463F
:1089D00061EEA71ACDED021AFFF79AFDDDED021A3E
:1089E000DDED030AB0EE401A2846B0EE480A61F009
:1089F0002FFD0DB0BDEC028BF0BD072B2A680DD109
:108A0000B6F940369FED151A07EE903AF8EEE77A80
:108A1000936A27EE811AB0EE480AB1E72046CDED01
:108A2000020AD66AFFF774FDDDED020AB0EE401AC5
:108A30003946B0EE480A2846B047DAE700000000A1
:108A4000B045002000000034507A0020747A0020E5
:108A5000687A00207C7A0020B02500200000C842FF
:108A6000044B196083ED010AC3ED020A83ED031A7A
:108A7000704700BF807A002038B505466CF0F6F8E4
:108A8000054C2061E86866F089FB07C804F114030F
:108A900083E8070038BD00BF807A002037B5284C36
:108AA00023680546002B3FD1E86866F077FBD4EDDC
:108AB000017A9FED247AF0EEE76AF4EEC76AF1EEF0
:108AC00010FA06D4D0ED026AF4EEE67AF1EE10FA6E
:108AD00031DCD4ED027AF0EEE76AF4EEC76AF1EE2B
:108AE00010FA06D490ED027AF4EEC77AF1EE10FA9D
:108AF00021D4D4ED037AF5EEC07AF1EE10FA1DDD43
:108B0000114919F07BF868468DED000ACDED010A98
:108B100019F042F9D4ED037AF4EEC07AF1EE10FACE
:108B20004CBF0120002007E06CF0A0F82369226808
:108B3000C31A9342B8D3012003B030BD0020FBE735
:108B4000807A002000000034947A0020024B00223A
:108B50005A619A61DA617047807A002030B52DED54
:108B6000028B9FED1A8A1A4B85B004460025F0EE61
:108B7000480AB0EE481AF0EE481AB0EE480A154816
:108B800083F855548DED018A8DED028A8DED038AAF
:108B900065F0BCFE01A90F488DED018A8DED028ABA
:108BA0008DED038A65F05AFA2A4601A9094865F055
:108BB0008DFF29462046FFF737F901462046FFF78B
:108BC000E7F905B0BDEC028B30BD00BF000000002E
:108BD000B07500208C64002038B5054605480C4669
:108BE00001F01CFF00B91CB12846FFF7B7FF0124B4
:108BF000204638BDB025002030B5204B93F85534C1
:108C000087B00D460BB1FFF7A9FF1D48294653F069
:108C1000B1FF044640B940F0F5F9052216213FF0B6
:108C2000A9FF204607B030BD1648294665F0D4FD9F
:108C3000044618B940F0E6F90222EFE7D5ED027AD2
:108C40000E48F8EEE76AD5ED037A90F85514CDEDAD
:108C5000006AB8EEE77AD5ED017A8DED017A00234E
:108C6000F8EEE77A0393049305936A4603ABA0F505
:108C7000A040CDED027AFAF72FFBD2E7B0750020C5
:108C8000104500208C64002030B5174B93F8553404
:108C900089B00C460BB1FFF761FF0222214604A800
:108CA0000AF098FB114804A953F064FF054640B947
:108CB00040F0A8F9052216213FF05CFF284609B0D4
:108CC00030BD214600220A4865F000FF0648002317
:108CD00090F85514019302930393224601ABA0F53B
:108CE000A040FAF7F9FAE9E7B07500201045002036
:108CF0008C6400202DE9F0412DED028B9846234B2A
:108D000093F8553488B006460C461746B0EE408AB4
:108D1000F0EE608A0BB1FFF721FF0222214604A882
:108D20000AF058FB1A4804A953F024FF054658B925
:108D300040F068F9052216213FF01CFF284608B0D4
:108D4000BDEC028BBDE8F0819DF84030F0EE680A82
:108D50004246B0EE480A39463046FFF735F96BF027
:108D600085FF0C4B2146186000220B4865F0AEFED3
:108D70000648002390F8551401930293039322466A
:108D800001ABA0F5A040FAF7A7FAD7E7B07500202D
:108D900010450020507A00208C64002070B52DED25
:108DA000028B0446406990F8D33086B03BBB01216A
:108DB00067F0A6FA606B9FED698A62680368D2ED7E
:108DC000020A9B6DB0EE480A01219847606B62F081
:108DD00053FC63488DED038AF0EE480AB0EE481A62
:108DE000F0EE481AB0EE480A8DED048A8DED058A42
:108DF00006B0BDEC028BBDE8704065F087BD5948F8
:108E000090F8A01D11F0010500F5805651D1636A5C
:108E10001B68A0F50050B3F90810F9F73DF8DFED35
:108E2000527AB0EEC07AB4EEE77AF1EE10FAB0EE14
:108E3000408A37D429462046FFF7AAF80221606904
:108E400067F05EFA464865F047FC01464748FBF785
:108E5000CFFF02A9454803AA00F0F6FF6369029A12
:108E6000DA636369039A9A63206B64F033FC96F8C3
:108E70002436656BD4E90612F3B91368B3F90830E8
:108E800000EE903A0B68B3F9083000EE103A2B6808
:108E9000F8EEE00A9B6AB8EEC00AB0EE481A28461F
:108EA000984735E096F825360BB10721C3E7032133
:108EB000C1E79FED2A8AC1E709681268B1F9081075
:108EC000B2F9082008EE101A00EE902A032BB8EE33
:108ED000C88AF8EEE00A1FD1B6F94036DFED247AF1
:108EE000CDED010A01EE903AF8EEE11A204661EE6E
:108EF000A71ACDED001AFFF70BFBDDED001ADDED33
:108F0000010AB0EE401A2846B0EE480A61F0A0FA15
:108F100006B0BDEC028B70BD072B2A680DD1B6F9E7
:108F200040369FED131A07EE903AF8EEE77A936A0F
:108F300027EE811AB0EE480AB1E72046CDED000ACF
:108F4000D66AFFF7E5FADDED000AB0EE401A01211E
:108F5000B0EE480A2846B047DAE700BF000000003C
:108F60008C640020B045002000000034B0250020B3
:108F70000000C842084B93F85534032B0BD8DFE8A8
:108F800003F002040608FFF709BFFFF74BBBFFF72A
:108F900041BCFEF75FBF7047B075002000207047EE
:108FA000012070470120704700207047004870473B
:108FB000BCB40B0800487047C4B40B0808B5036B79
:108FC00003480022C3F84C23FCF72EFC012008BD07
:108FD000B025002038B52C4D95F87B3E04469BB952
:108FE00005F6A850012167F08BF9606B6268036891
:108FF000D2ED020A9B6D9FED250A01219847606B17
:10900000BDE8384062F038BB022105F6A85067F091
:1090100077F9A36918684BF087F805F6BC5383ED20
:10902000000AE36918684BF07FF805F6C45383ED36
:10903000000A636A18684BF077F86268D2ED277A05
:1090400020EE270AB0EE0B7AC0EE077A05F6CC5375
:10905000C3ED007A236A18684BF066F805F6D4531E
:1090600083ED000AA36A18684BF05EF805F55E63AD
:1090700083ED000AE36A18684BF056F805F6E455EC
:1090800085ED000A38BD00BFB0450020000000009B
:109090000020704700207047012070470120704772
:1090A000004870470CB50B080048704718B50B080E
:1090B000044A00231370044A1370044B01201880E3
:1090C000704700BFA07A0020AE7A0020AC7A002062
:1090D000F0B50446406990F8D3508BB0B5B9012182
:1090E00067F00EF960692946EEB267F021F828B101
:1090F000606940F2DC52314667F010FD01350C2DFD
:10910000F0D19E4B00221A700BB0F0BD9B4D2B7816
:10911000042BF9D8DFE813F00500110040005E00D1
:109120002201974B01241C80964B00221A706BF091
:109130009DFD954B2C701860E6E70026606931466E
:10914000F7B266F0F5FF28B1606940F2DC523946AB
:1091500067F0E4FC01360C2EF0D121698A4C01F550
:109160004371084619F048FEDFED887AB4EEE70A4D
:10917000F1EE10FA02DD6BF079FD20606BF076FD08
:10918000236803F5FA739842BED902232B706BF063
:109190006DFD7F4B1860B7E76BF068FD7C4B1B687B
:1091A00003F5FA73984212D2754B60691A88754BB1
:1091B00002EB8202C2EB0212920002F2DC52197838
:1091C00012B267F0ABFC00289ED1042300E0032319
:1091D0002B7099E72369DFED6F5AD3EDC37ADFED8A
:1091E0006E6A674F93EDC46A93EDC57AB7F90010C4
:1091F000644EF4EEE57AF1EE10FAF4EEE67ACCBFC6
:1092000001220022F1EE10FA4CBF01230023D21AF2
:10921000B4EEE56A4A43F1EE10FAB4EEE66A07EE00
:10922000902ACCBF01220022F1EE10FA4CBF01239C
:109230000023D21AF8EEE77A4A43CDED017A07EE21
:10924000902AF8EEE77ACDED027AF6EE007AB4EEE7
:10925000E77AFEEE007AF1EE10FAB4EEE77ACCBFD0
:1092600001230023F1EE10FA4CBF012200229B1AC9
:109270004B4307EE903AF8EEE77A3178CDED037A7A
:1092800066F03CFF07A901A88DED070ACDED080A9D
:109290008DED091A19F0BEFCF8B12046FDF7C8FCA7
:1092A00033783E4A0133062142F074FF3178606919
:1092B00001231944C9B22B7031703B8066F038FF2E
:1092C00000287FF421AF042620462E70FDF7B0FC65
:1092D000334A314642F05EFF16E701A819F0D4FC8C
:1092E000317860698DED040ACDED050A8DED061A21
:1092F00066F004FF07A904A88DED070ACDED080A62
:109300008DED091A19F086FC70B12046FDF790FC2E
:109310003378244A0133062142F03CFF31786069FA
:10932000012266F00DFFC1E72046FDF781FC1E4AD1
:10933000062142F02FFFB7F90030013309D1204652
:10934000FDF776FC3378194A0133042142F022FFFD
:109350003BE74FF6FF733B80012339E7144B0822AC
:1093600093F8811D2046FDF75DFC1248012216216D
:109370000BB0BDE8F040F8F7C3B900BFAE7A0020EB
:10938000AC7A0020A07A0020A47A00200AD7233CDF
:10939000A87A0020CDCCCC3ECDCCCCBE20B50B08DD
:1093A000BAB50B0833B50B0857B50B0888B50B08D1
:1093B000B0450020785B00200020704700207047F7
:1093C00001207047012070470048704724B60B0801
:1093D000004870472CB60B0870B52DED028B84B099
:1093E00004466BF043FC064660696C4D90F8D33040
:1093F00003BB012166F084FF606B62680368D2EDF5
:10940000020A9B6D0121B6EE000A9847606B62F07C
:1094100033F9206B63F042FF206BB6EE000A64F074
:1094200003F92369D3F8F831C5F89C3104B0BDECD9
:10943000028B70BD022166F063FFE36A18684AF090
:1094400073FEA36A1868B0EE408A4AF06DFE0023EE
:10945000A5F5A040F0EE408A0093019301F0DEFAFA
:1094600000287AD09FED4E7AF0EEC87AF4EEC77AF3
:10947000F1EE10FA06DCF0EEE87AF4EEC77AF1EEDF
:1094800010FA02DD206B63F009FF464801AA694625
:1094900000F066FD206B63F061FF9DED010A6369DA
:1094A00070EE288A9DED000AC3ED0E8A30EE088A20
:1094B000636983ED0F8A636A1868438A828907EEBD
:1094C000903A394BF8EEE77A93ED007A67EE877AB7
:1094D000FCEEE77A17EE903A99B24AF0BBFD0146EE
:1094E0003048F8F7D9FC314B2E48B3F95C3001EE27
:1094F000103AE3691B68B3F9083000EE903AA369AB
:109500001B68B3F90830B0EE408A00EE103AB8EEAE
:10951000C11AF8EEE00AB8EEC00A03AA02A9F8F7E9
:1095200051FCDFED237A606BB0EEC87AB4EEE77AD7
:10953000F1EE10FA15D40368DDED030A9B6A9DED88
:10954000020AB0EE481A98472369D3F8F831C5E902
:1095500067362046FDF752FD68E7206B63F09EFEFC
:109560009BE7D5F8A03102689DED020ADDED030A04
:10957000FA33B34209D9936A9FED0E1A98472369CB
:10958000D3F8F831C5F89C31E3E795ED671AD36A53
:10959000B8EE411A01219847DBE700BFB075002003
:1095A000CDCCCC3DB0250020BC5B0020B0450020D8
:1095B00000000034000000002DE9F04104462DEDCC
:1095C000028B414801F02AFA0646002877D03F4D29
:1095D000DFED3F8A9FED3F8A206B05F60478D8EDDA
:1095E000000AF4EEE80A05F6F467F1EE10FA97EDDA
:1095F000000AB8BFF0EE480A62F06AFFD8ED000A30
:1096000097ED000A206BF4EEE80AF1EE10FAB8BF0D
:10961000F0EE480A62F0D4FFA5F54050276BF8F74A
:10962000D9FC6368B3F92C20B3F9283000EE903AE6
:10963000434201EE102A00EE103AB8EEC11AF8EEDD
:10964000E00AB8EEC00A384663F022F8A5F54050AB
:10965000276BF8F7BFFC6368B3F92C20B3F9283007
:1096600000EE903A434201EE102A00EE103AB8EEB6
:10967000C11AF8EEE00AB8EEC00A384663F082F884
:10968000206B63F00BFE206B63F066FF606B62681B
:109690000368D2ED020A9B6D0121B6EE000A9847DD
:1096A000606B61F0E9FF206BB6EE000A63F0BCFF6F
:1096B000236905F50055D3F8F831C5F89C31BDECA8
:1096C000028B3046BDE8F081B0250020B055002067
:1096D0000000003400007A430020704701207047EA
:1096E00001207047002070470048704774B60B088F
:1096F0000048704780B60B08036B0022C3F84C2368
:109700000369D3F8F821024B0120C3F89C2170476C
:10971000B075002073B504466BF0A8FA0646606980
:10972000524D90F8D330B3B9012166F0E9FD606B7A
:1097300062680368D2ED020A9B6D9FED4D0A01211C
:109740009847606B61F098FF2369D3F8F831C5F84A
:109750009C3102B070BD022166F0D2FDA5F54053E8
:1097600001AAB3F95C3001EE103AE3691B68B3F962
:10977000083000EE903AA3691B68B3F9083000EE98
:10978000103AB8EEC11AF8EEE00AB8EEC00A69461F
:10979000A5F5A040F8F716FB636A1868438A82892A
:1097A00007EE903AA5F5CF5313ED057AF8EEE77A78
:1097B00067EE877AFCEEE77A17EE903A99B24AF0B4
:1097C00049FC0146A5F5A040F8F766FBDFED297AD4
:1097D000606BB0EEC07AB4EEE77AF1EE10FAB0EE5C
:1097E000401A27D40368DDED010A9B6A9DED000A4B
:1097F00098472369D3F8F831C5E96736656B2B685C
:109800009E6D236A18684AF08FFC63680021D3EDCF
:10981000020A2846B047A36A656918684AF084FCC2
:1098200085ED0E0AE36A656918684AF07DFC85EDEE
:109830000F0A8EE7D5F8A03102689DED000ADDED34
:10984000010AFA33B34209D9936A9FED091A98477E
:109850002369D3F8F831C5F89C31CFE795ED671A45
:10986000D36AB8EE411A01219847C7E7B0750020C6
:109870000000000000000034012070470020704705
:10988000012070470120704700487047C8B60B0898
:1098900000487047D0B60B0837B5436993F8D3201A
:1098A0000446D2B91A681846526A90476069012185
:1098B00066F026FD606B62680368D2ED020A9B6D5C
:1098C0009FED360A01219847606B61F0D5FE206B51
:1098D00003B0BDE8304063F03FBE314D95F97C3DAB
:1098E000002B03DA1B220221FDF79CF9B5F95C304D
:1098F0002C482D4D01EE103AE3691B68B3F908308E
:1099000000EE903AA3691B68B3F9083000EE103AF4
:1099100001AAB8EEC11AF8EEE00A6946B8EEC00A2C
:10992000F8F750FA636A1F481B68B3F90810F8F794
:10993000B3FA606BDDED010A0368B0EE401A9B6A72
:109940009DED000A984705F6F86292ED000A236B38
:10995000F7EE000A93EDC61A3320B0EEC00A16F0F7
:1099600083FEFDEEC07A17EE903AA5F8F830206B32
:1099700062F058FF206B63F0ADFEA36A656918685A
:109980004AF0D2FB85ED0E0AE36A656918684AF071
:10999000CBFB85ED0F0A03B030BD00BF0000000017
:1099A000B0450020B0250020B055002070B5044619
:1099B0001D48F8F70DF80546A0B31B48266BF8F7CD
:1099C00009FB6368B3F92C20B3F9283000EE903A14
:1099D000434201EE102A00EE103AB8EEC11AF8EE3A
:1099E000E00AB8EEC00A304662F052FE0E48266B1E
:1099F000F8F7F0FA6368B3F92C20B3F9283000EED9
:109A0000903A434201EE102A00EE103A3046B8EE8A
:109A1000C11AF8EEE00AB8EEC00A62F0B3FE206B9D
:109A200063F09AFD284670BDB025002000487047BD
:109A300018B70B080048704724B70B0810B5044648
:109A4000FCF70AFE054B2360054BE363002384F813
:109A5000403000236364204610BD00BF4CB80B08A3
:109A6000000080BF054BC363054B03F57B5103F535
:109A70007A5300220A60DA63704700BF000080BF9B
:109A8000B025002037B50546FDF75EF9044660B104
:109A90002846FFF7E7FF154800F068FD054638B98E
:109AA000134A1448062142F075FB204603B030BD2E
:109AB0001148124C65F076FBD4ED1C7AB4EEE70A3F
:109AC000F1EE10FA0FDB9FED0E7A67EE877A17EE54
:109AD000900AF6F719FD0B4ACDE90001042104F6BE
:109AE000783042F057FB2C46DFE700BFB02500205E
:109AF0002CB70B0828510020005C0020B045002046
:109B00000AD7233C4EB70B0830B52DED028B364CEF
:109B100094F8803D152B83B00546B0EE408A06D000
:109B2000324A042104F6783042F034FB19E0304820
:109B300065F038FBD4ED1C7AB4EEE70AF1EE10FACA
:109B400014DB9FED2C7A67EE877A17EE900AF6F712
:109B5000DBFC294ACDE90001042104F6783042F00B
:109B600019FB2846FFF77EFF002037E0B4F9003AE2
:109B700007EE903AF8EEE77AF4EEC87AF1EE10FAD2
:109B800001DD1E4ACDE7B4F9023A07EE903AF8EE4D
:109B9000E77AF4EEC87AF1EE10FA23D4DFED157A05
:109BA00085ED0F8A68EE277A17EE900AF6F7ACFC7F
:109BB000134ACDE9000104F67830062142F0EAFAB2
:109BC0000B4865F0EFFAD5ED0F7A30EE670A04F531
:109BD000F65484ED000A04ED010A012003B0BDEC47
:109BE000028B30BD074A9CE7B045002074B70B08D4
:109BF000005C00200AD7233C9BB70B08CDB70B08AD
:109C0000F7B70B0819B80B0838B504462DED028BD1
:109C10001C4800F0ABFC90B3D4ED0F7A1A4DF5EE72
:109C2000C07A05F60C23F1EE10FA93ED008A0FDCF2
:109C300005F6082393ED000AD5ED1C7AB4EEE70A89
:109C4000F1EE10FA04D530EE480A2046FFF75CFF2B
:109C5000D4ED0F7AF5EEC07AF1EE10FA0FDD78EE62
:109C6000277A95ED1C7A094BF4EEC77AF1EE10FADB
:109C7000A4BF77EE677A38EE278A83ED008ABDECC1
:109C8000028B38BDB0250020B04500206C64002058
:109C900030B52DED028B036A1B68B3F9083000EE76
:109CA000103A83B00446B8EEC00A4848F8F7A4F961
:109CB00046488DED010AF8F78DF963689DED010ABC
:109CC000B3F9283001EE103A434200EE903AB8EE74
:109CD000C11AF8EEE00A692016F0C6FCDFED3C7A06
:109CE000B0EEC07AB4EEE77AF1EE10FAB0EE408A48
:109CF00058D594F8403083B1E068D4ED0F8A65F010
:109D000051FAD4ED117A38EE800A204630EE670A17
:109D1000FFF7FAFE002384F840302E4B93F87C2D99
:109D200093F97C3D002B22DA6268236BD2ED2C7A0A
:109D300093EDD37AF1EE046A77EEE67AF4EE477AA1
:109D4000F1EE10FAC8BFF0EE477AC3EDD37A2046A1
:109D5000FFF788FE206BB0EE480A62F063FD206BCF
:109D600003B0BDEC028BBDE8304063F0B3BC5306DA
:109D700014D5E068256B65F015FA236BF2EE047AD2
:109D800030EE270AD3EDD37AB4EE670AF1EE10FA7B
:109D9000C8BFF0EE407AC5EDD37AD8E72046FFF78A
:109DA00033FFD7E7D4ED0F7AF5EEC07AF1EE10FA73
:109DB000D0DD94F84030002BCCD1E06865F0F2F9AA
:109DC000012384ED110A84F84030C3E7B025002058
:109DD000CDCC4C3DB045002010B50446FCF7FEFF4D
:109DE0002046FFF755FF2046BDE81040FDF7F4B8C8
:109DF00038B5044604F5A0456AF038FFD5F8AC3113
:109E000003F5FA7398421BD904F52D5004F500545C
:109E10000C4A0621383042F0BDF994F87C3D6FF3CE
:109E2000C30384F87C3D69F0A3FA036801225B68F0
:109E3000032198476AF01AFFC5F8A801002038BD31
:109E40000120FCE784B80B0870B52DED028B00F5FE
:109E5000405300F50054D3F8EC3ED3EDCD7AD3ED6A
:109E6000CE8AFDEEE77A1546B4F95C2017EE903AFB
:109E70000E46F1EE688A5142FDEEE88A09B218B248
:109E800016F030FCB4F95C2018EE903A514208EE1E
:109E9000100A09B218B216F025FCB4F95C3007EECE
:109EA000903AB8EEC88AF8EEE77A88EE277ABDECE9
:109EB000028B07EE900A86ED007AB4F95C30B8EEBA
:109EC000E77A07EE903AF8EEE77AC7EE276AC5ED33
:109ED000006A70BD70B52DED028B00F5804300F572
:109EE0000054D3F8F037D3EDCD7AD3EDCE8AFDEE22
:109EF000E77A1546B4F95C2017EE903A0E46F1EE7B
:109F0000688A5142FDEEE88A09B218B216F0EAFBFF
:109F1000B4F95C2018EE903A514208EE100A09B2EA
:109F200018B216F0DFFBB4F95C3007EE903AB8EEE9
:109F3000C88AF8EEE77A88EE277ABDEC028B07EE46
:109F4000900A86ED007AB4F95C30B8EEE77A07EE55
:109F5000903AF8EEE77AC7EE276AC5ED006A70BD61
:109F600070B52DED028B00F56C53D3EDD87AD3ED9F
:109F7000D98A00F50054FDEEE77A1546B4F95C2065
:109F800017EE903A0E46F1EE688A5142FDEEE88AED
:109F900009B218B216F0A6FBB4F95C2018EE903A9C
:109FA000514208EE100A09B218B216F09BFBB4F940
:109FB0005C3007EE903AB8EEC88AF8EEE77A88EEA1
:109FC000277ABDEC028B07EE900A86ED007AB4F991
:109FD0005C30B8EEE77A07EE903AF8EEE77AC7EE33
:109FE000276AC5ED006A70BD00F53650283065F06F
:109FF00013BA000070B504466AF038FE04F5A043B9
:10A00000D3F8A82102F51C53103383420AD94AB170
:10A01000164A04F52D500221383042F0BBF80025D5
:10A02000284670BD124B1B68D86A03681B6A9847A4
:10A03000012801D10F4AECE704F5005696F87B5E43
:10A040003DB904F52D500C4A0421383042F0A2F8F5
:10A05000E6E704F53650283065F0DEF996F87C3DE9
:10A0600043F0080386F87C3DDAE700BF9CB80B0894
:10A07000A8250020C9B80B08FEB80B0884B070B53D
:10A080002DED048B84B004460DA880E80E006AF024
:10A09000EDFD04F5A04304F50055C3F8AC0195F8B7
:10A0A0007C3D1B071DD44A4E6AF0E0FD336803F582
:10A0B000FA6398420DD92046FFF79CFF88B904F552
:10A0C0002D50444A0421383042F064F86AF0CEFD45
:10A0D0003060002004B0BDEC048BBDE8704004B0DB
:10A0E0007047129802280CD0F6F7ECF9CDE9000180
:10A0F00004F52D54384A38340421204642F04AF8F9
:10A10000E7E79DED0E0A9DED0D8A8DED030AF0EE59
:10A11000000ADDED0F8A16F0CDF99DED030A50B16E
:10A1200010EE100AF6F7F0F904F52D54CDE9000110
:10A130002A4A3834E0E7F7EE000A8DED030A16F0FC
:10A14000B9F99DED030AA8B1FDEEE88AFCEEC87AE4
:10A1500018EE903ACDED037A04F536509DF80C10C8
:10A160001AB2283004B0BDEC048BBDE8704004B0D6
:10A1700066F0D4BCDFED1A0A16F09CF90028A8D0CE
:10A180009FED189ADFED160A8020B0EE491AB0EE66
:10A19000680A16F069FAC0EE096AD5F8B828B2F96B
:10A1A0000A30B2F90E20D21A07EE902AB8EEE77AFA
:10A1B00007EE903AF8EEE77AE6EE877ABCEEC87AD8
:10A1C000FDEEE77A8DED037A17EE903AC4E700BF13
:10A1D000B07A002020B90B0842B90B0856B90B0819
:10A1E000000000000000C84210B500F5005304460E
:10A1F00093F8802D142A19D093F87C2D120703D5DB
:10A20000BDE81040FFF7F4BD012283F87C2E4BF02F
:10A2100031FC4BF0C5FB4BF06BF804F536502830A1
:10A2200067F058FCBDE810404BF02CBC10BD00009E
:10A23000024B01461868026812681047347F0020FC
:10A2400010B504460020FFF7F3FF04F50054C4F8EE
:10A25000B4080120FFF7ECFFC4F8B0080220FFF7B4
:10A26000E7FFC4F8B8080320FFF7E2FFC4F8BC0812
:10A270000420FFF7DDFFC4F8C0080520FFF7D8FF72
:10A2800041F29411C4F8C408D4F8B00849F0B6FEFD
:10A29000D4F8B40841F2941149F0B0FED4F8BC08E7
:10A2A00041F2941149F0AAFED4F8B8084FF47A713B
:10A2B00049F0A0FED4F8C00841F2941149F09EFE86
:10A2C000D4F8C40841F2941149F098FED4F8B008CB
:10A2D0001E2149F097FED4F8B4081E2149F092FEE1
:10A2E000D4F8B8081E2149F08DFED4F8BC08282106
:10A2F00049F088FED4F8C0081E2149F083FED4F846
:10A30000C4081E2149F07EFE0024E0B2002240F283
:10A31000DC51013449F0A6FD062CF6D1204600227E
:10A3200040F2DC5149F09EFDBDE81040002240F2B1
:10A33000DC51072049F096BD37B5044604F50055B9
:10A3400000F536502830B5F89E10019066F0BEF842
:10A3500095F814110198002266F0A4F8D5F8B838E1
:10A360000198B3F90A10B3F90E2067F0D7FB0198F2
:10A3700067F0D8F904F5575001210830F7F7D0F805
:10A3800010B12046FFF730FE03B0BDE830404BF07F
:10A3900021B9000013B5044600F58D60019005F069
:10A3A00043FB94F879340198242202FB0303D3ED94
:10A3B0000B7AF5EEC07AF1EE10FA02DD05F03CFC06
:10A3C000019804F5005494F87D3DDB0709D594F815
:10A3D000A51D05F019FB94F8A43D60F3000384F873
:10A3E000A43D02B010BD000038B5102300F648555A
:10A3F000C0F8F43F04461921284636F00DF804F55C
:10A400002850B5EE000A103041F0D2F904F500549E
:10A410001921284635F04CFB94F8FC3960F3000311
:10A4200084F8FC3938BD0000F8B500F648562DED2B
:10A43000028B0546304635F0F5FB1921304635F0E4
:10A440005DFB19210746304635F028FB042805F549
:10A4500000546FD0002094F8FC3960F3410384F875
:10A46000FC391921304635F039FBA4F8FE0905F511
:10A470005950103064F096FE04F6082383ED000A6C
:10A480001921304635F050FB1921A4F8000A304656
:10A4900035F040FB94F8FC39A4F8020A9B0725D557
:10A4A0006AF0E4FBD4F8043A0646F31AB3F57A7F6F
:10A4B000B4F9FE3905F5285000EE103A00F110000D
:10A4C00049D9B8EEC00A41F0E3F92648C4F8046A55
:10A4D0000346083093ED008A41F0D8F9D0ED007AB8
:10A4E00078EE677A04F60C23C3ED007A94F8FC3911
:10A4F00004F60C2405F5804205F58F452168C3F369
:10A500000006C3F3400013F0010382F88A6782F863
:10A510008C07296104D092F98B37003B18BF0123C7
:10A5200082F8353882F8360802F2E4725165BDECE3
:10A53000028BF8BD1921304635F012FB022889D96B
:10A540007A1C06D094F96C30BB42CCBF00200120AD
:10A5500081E701207FE7DFED040AB8EEC00A41F091
:10A560002BF9B2E7B84F0020CDCC4C3D10B50446D6
:10A570006AF07CFB04F5005393F8FC2912F001010A
:10A580000BD0C2F34001920707D5D3F8043AC01AA2
:10A59000B0F57A7F2CBF00210121084610BD0000D4
:10A5A00008B500F5005090F87C3DB1EBD31F13D0F7
:10A5B00061F3C713094A80F87C3D00211B06116036
:10A5C00006D53EF01FFDA321BDE808403EF0B2BA1B
:10A5D0003EF018FDA421F7E708BD00BFB87A0020BF
:10A5E00008B500F5005090F87C3DC3F380128A4214
:10A5F00013D061F38613094A80F87C3D00215B0685
:10A60000116006D53EF0FEFCA521BDE808403EF0F5
:10A6100091BA3EF0F7FCA621F7E708BDB47A002016
:10A6200070B500F5005586B095F87B1E044649B913
:10A630000191FFF7B5FF0199204606B0BDE87040D3
:10A64000FFF7CEBF00F58F50002303A90830039316
:10A650000493059302F096FFDDED057A9FED3F7AB6
:10A66000F4EEC77AF1EE10FA49DD9FED3D7AF4EE93
:10A67000C77AF1EE10FA4CBF0126002695F87D3D11
:10A68000DA0746D595F8A43DDB0742D594F879243E
:10A6900095ED446ADFED336A04F58D63242101FBF7
:10A6A000023393ED0B7A95F97C3D002BC6EE267AAA
:10A6B00027DADFED2B6A77EEE67AF4EEC77AF1EE71
:10A6C00010FA4CBF012100212046FFF769FF95F8E1
:10A6D000AF3D002B3FD0002E3DD0234A136807EE3C
:10A6E000903AB8EE677ADFED217AB4EEE77AF1EED0
:10A6F00010FA1FD401212046FFF772FF21E0002647
:10A70000BCE7B4EEE77AF1EE10FACCBF01210021EC
:10A71000DAE7E6B195F8B03DABB1154A136807EE3C
:10A72000903AB8EE677ADFED117AB4EEE77AF1EE9F
:10A7300010FA02D50133136003E001212046FFF730
:10A740002FFF06B070BD95F8AF3D002BC5D100219D
:10A750002046FFF725FF0021CDE700BFCDCC4CBD43
:10A76000CDCC4C3D0000C842B47A00200000C84364
:10A77000B87A0020F8F7E2BD0148FAF755BB00BFF0
:10A78000B025002038B500F58F5508350446284619
:10A7900001F0ECFD04F58053042283F8F423B4F9AE
:10A7A0009C3004F6D8001BB9B4F89A30A4F89C3059
:10A7B000B4F89C1015F0E8FA2846BDE8384001F0DE
:10A7C000CDBE00002DE9F3410446103006F06AF9D1
:10A7D00004F50450183058F00BFD04F58C5014307B
:10A7E00031F002F904F5445004F58D66083005F0A7
:10A7F00057FD304605F0D2FBB7EE000A6F4834F043
:10A800001DFA04F52D50383045F074FC2046F8F759
:10A81000ADFD49F0ABFB992229214AF071FB49F0CB
:10A82000A5FB49F07DFB2046FFF70AFD2046FFF718
:10A8300083FD2046FAF77CFF04F58B504DF094FB26
:10A840005F4B60491B68986A03684FF47A72DB6A51
:10A850009847042304F588510C31C4F8503104F5AD
:10A8600088700DF0EFF90BF033FF4FF400530363E2
:10A870000BF02EFF04F580570CF0F6FE802504F552
:10A8800090403C30C7F8505F06F0F0FE00213046A3
:10A89000C4F87C5405F00EFA304605F0C5F894F87B
:10A8A00078C4002304F27C4024225FFA83F8C44574
:10A8B00020D903FB02215D1C415C012979D104F5FB
:10A8C0000055694604F204508DF8003034F090FCD5
:10A8D00095F87D3D85F8A58D43F0010385F87D3D14
:10A8E0004146304605F090F895F8A43D60F300032A
:10A8F00085F8A43D04F5005604F58F5596F87D3D86
:10A9000013F0010305F10805E84654D1414604F26D
:10A9100004508DF8003034F06BFCB2EE040A284687
:10A9200002F0CCFD04F52750183064F07BFC04F5F0
:10A93000A043D7F8E023C3F89C212046FFF754FD3D
:10A9400004F5285020304BF08FFA04F52A500430DB
:10A950001AF0E6F91C4B00931C4B019304F52350AD
:10A9600098E8060008303DF02DFB2046FFF70AFF6F
:10A970002046FAF73FF94FF40023C4F8E03B2046A5
:10A98000F8F700FE04F521502430F9F713FB2046B8
:10A99000F8F72CFE2046F8F76FFE2046F8F7B0FED9
:10A9A00096F87C3D43F0100386F87C3D02B0BDE88C
:10A9B000F0812B4679E79FED060AB0E770B90B08E6
:10A9C000A825002079A70108B025002075A7010857
:10A9D000CDCCCC3D13B5044600F58F50083001F0C6
:10A9E000DDFE90B104F55950103004F5005464F0C8
:10A9F000CBFB94F87B2E0190C3B2C0F3001032B9A8
:10AA000018B99DF80500C0F3400002B010BD002841
:10AA1000FBD083F08000C009F7E7000038B500F5EF
:10AA20000053054693F8A03D5B070AD4FFF7D2FF19
:10AA3000044620B905F58F50083001F0AFFE2046DE
:10AA400038BD0024FBE7000037B500F52355083575
:10AA5000044604F50054284601913DF0FBFB94F8B0
:10AA60007C3D019960F34103284684F87C3D03B0A6
:10AA7000BDE830403EF0ECB837B500F591455035B3
:10AA8000044628463BF0FCFE012201A928463BF083
:10AA900077FE20B104F64854019BC4F89C3203B001
:10AAA00030BD000010B504210446FFF7CDFF30B1E2
:10AAB00004F591405030BDE810403BF02FBF10BD71
:10AAC00000F58053D3EDFB7A9FED227AF5EEC07A44
:10AAD000F1EE10FA04DBF4EEC77AF1EE10FA17D4B7
:10AAE000F4EEC77AF1EE10FA14DC9FED1B7AF4EE67
:10AAF000C77AF1EE10FA4CBF0223032300F5405051
:10AB000090F80826032A0ED8DFE802F006161B1F6D
:10AB10000023F3E70123F1E7012B07D1D0F8042646
:10AB20000132C0F8042680F808367047032BFAD1AA
:10AB3000D0F80426013AF4E7022BEFD0002BF7D02F
:10AB4000F1E7032BEAD0012BF1E7002BE6D0022B33
:10AB5000EDE700BFDB0FC93FDB0FC9BF13B50446EC
:10AB6000143000F0CFFE04F12C0000F0CBFE04F115
:10AB700074006BF003FB04F1F4006BF0FFFA4FF08C
:10AB8000FF331549C4F85031204633F0C3FC00238D
:10AB90000DF1070104F128008DF8073034F00AFBAD
:10ABA00001230DF1070104F129008DF8073034F07D
:10ABB00001FB0F230DF1070104F125008DF807308B
:10ABC00034F0F8FA054B1A6812B105486AF01CF81F
:10ABD00020461C6002B010BD08BB0B08BC7A0020E8
:10ABE00080B90B082DE9F0478CB003A932F068FF5B
:10ABF00060B300210D2208A807AF1C4CDFF870805D
:10AC0000DFF8709007910B2697F0ACF90697237A3E
:10AC1000DFF864A08DF81430002554F82530049333
:10AC2000D8F80000E368B5B90093C06A5346112212
:10AC3000394612F033FB0021B7EE000A03A833F0C7
:10AC40007BF935B1013E04F11004E0D10CB0BDE850
:10AC5000F0870125E1E701930223009311224B467F
:10AC60003946C06A12F01AFBE5E700BFA8BB0B0823
:10AC7000A8250020DDB90B08D4B90B082DE9F74F42
:10AC8000D0F8543104467BBBDFF86CA1074600F1D5
:10AC9000740800F5AA750126721ED2B297ED070A54
:10ACA000019240466BF08AFAFB69C8F83C304FF0DD
:10ACB0007E53C8F8483097F92830019A013B5FFA73
:10ACC00086FB0C2B1FD8DFE803F0123D49565F6866
:10ACD0001E1E1E1E1E1E7A00D4F8543103B9636175
:10ACE000D4F8583103B9E36203B0BDE8F08F4820CF
:10ACF000019208F0C9FB814618B1019A21466AF019
:10AD000001FAC5F80090286890B103689B689847DD
:10AD1000002866D147F068FC33465246032141F0D3
:10AD200039FA286810B103685B68984700232B60E4
:10AD3000022E07F1180708F1800805F10405CBD0B1
:10AD40000226A9E72820019208F09EFB81460028F0
:10AD5000D7D0019A21466BF0F9F9D2E76820019229
:10AD600008F092FB81460028CBD0FF23019A2146B0
:10AD70006AF06AFCC5E76820019208F085FB81460D
:10AD80000028BED00023F1E76820019208F07CFB88
:10AD900081460028B5D00123E8E74420019208F05D
:10ADA00073FB81460028ACD0019A214669F06CFF04
:10ADB0000F4BC9F800300023C9F84030A1E76020EC
:10ADC000019208F061FB814600289AD0019A214641
:10ADD00069F05AFF074BC9F800300023C9F8243046
:10ADE0008FE72B68002BA3D084F84FB1A0E700BFFA
:10ADF000B8E30C0868BC0B08BAB90B0813B50446D5
:10AE0000FFF7F0FE204632F0A9FF68B994F9283028
:10AE100013B994F940303BB101230DF107012046ED
:10AE20008DF8073034F0E4F994F90030002B08DD98
:10AE300094F928302BB1204602B0BDE81040FFF74E
:10AE40001DBF02B010BD00000346406C012807D0B2
:10AE5000032805D0986C012802D0032818BF0220CF
:10AE60007047000090F90030002B0ADD012908D856
:10AE7000182303FB010090F92800003818BF0120B7
:10AE8000704700207047000037B50446FFF7EAFF1F
:10AE90009FED0B0A0D4680B104EB81038DED010A95
:10AEA000D3F8540138B1036801A9DB68984704EB73
:10AEB000C51484F865009DED010A03B030BD00BFE4
:10AEC0000000000070B50446FFF7CCFF50B104EB62
:10AED0008104D4F8540128B10368BDE870401B69AF
:10AEE00011461847002070BD2DE9F04F2DED028B63
:10AEF00090F90030002B83B00646894653DD2C4B79
:10AF00001B68D86A03685B689847044650B147F0ED
:10AF10006BFB284A062103B0BDEC028BBDE8F04F65
:10AF200041F038B99FED248ADFF890A0DFF890B0A7
:10AF3000354606F14407B04621463046FFF792FFFA
:10AF400020B195F8643043B188ED068A8035043726
:10AF500008F118083CBB0124EEE7B9F1000F03D05B
:10AF600098F92630002BF1D1D7F81021631C0193FA
:10AF70003AB947F039FB019B5A46032141F00AF9DF
:10AF8000E4E769F073FE0022A5F87020A5F87220AE
:10AF90000122A86685ED1B8A3A6047F025FB019BDC
:10AFA00052460621EAE703B0BDEC028BBDE8F08F04
:10AFB000A8250020E8B90B080000000026BA0B08FD
:10AFC000FFB90B082DE9F0432DED028B83B0044649
:10AFD0000D46B0EE408AFFF745FF90B304EBC11772
:10AFE0004FEAC118BB6E63B369F040FEBB6EC01A76
:10AFF000B0F57A7F03D3B7F872300F2B0CD804EB7F
:10B00000080393F86520002A7AD14444B4F87230DA
:10B010000133A4F8723014E0B7F8703005F101097B
:10B0200005F1100693B947F0DFFA4B463C4A04217C
:10B0300041F0B0F804EB8606032344447360002318
:10B04000A36603B0BDEC028BBDE8F08347F0CCFAF9
:10B05000344A4B46062141F09DF8B7F87030D7EDE1
:10B060001B6AD4F85C2107EE903AF8EEE77A86EE98
:10B07000A77A8DED017ACAB394F90230002B35DD41
:10B0800007EE903AB2F906209FED275AF8EEE75AFC
:10B09000F7EE007AE5EE857A182101FB054506EE0C
:10B0A000902AF8EEE66A95ED066A67EEA67A37EE24
:10B0B000467A67EEA77AB0EEC77AE6EEE67AF6EE63
:10B0C000006A67EEA67AB4EEE77AF1EE10FA0DDDCB
:10B0D000B0EEC66AB5EEC06AF1EE10FA06DD47F0D2
:10B0E00083FA124A4B46042141F054F8182001A972
:10B0F00000FB094034F022F804EB860602239CE7AB
:10B10000B3F87220052A80D9D3ED1B7AB3F87020EA
:10B1100037EE880A013283ED1B0AA3F8702074E72A
:10B1200048BA0B085EBA0B080AD7233C75BA0B085D
:10B1300010B590F90030002B02460C461CDD90F84B
:10B140004D31CBB9FFF78EFEA8B1182101FB0422C7
:10B1500092F9243093B1022B0DD146204AF0D2F956
:10B16000DFED077AB0EEC00AB4EEE70AF1EE10FAAE
:10B170004CBF0120002010BD0020FCE71846FAE774
:10B18000000000342DE9F8432DED028B04460E46F5
:10B19000FFF768FEE8B104EB81090DB2D9F854312C
:10B1A000BBB169F063FD04EBC6174FEAC6183866F9
:10B1B000D9F8540103685B69984770B1D9F8540114
:10B1C000036839469B69503198473B6D87F86500A5
:10B1D000FB64BDEC028BBDE8F8833146204697F84E
:10B1E0006590FFF751FE182303FB064393ED068A93
:10B1F000BB6E30EE488A87ED178A1BB13146204678
:10B20000FFF7E0FEB9F1000F43D0DFED447A9FED88
:10B21000447A04EB080368EE277AD3ED166AE6EE6B
:10B22000877A182104EB080701FB0646C7ED167A5A
:10B2300096F9273083B3012B53D1DFED3A8AF1EE33
:10B24000487A05EB4505B4EEE88AC7ED157A04EBBC
:10B25000C505F1EE10FA95ED070A58BFF0EE687AD1
:10B2600027EE800A94F0B0FD87ED130A97ED160AD9
:10B27000B4EEE80AF1EE10FA48BFF1EE408A95ED1F
:10B28000070A28EE800A94F09FFD444484ED140AD6
:10B290009FE7F0EE487AC4E7B5EEC08A05EB4505B6
:10B2A000F1EE10FA87ED158A04EBC505D8BF9FEDC6
:10B2B0001D8A95ED070A28EE000A94F085FD04EB3F
:10B2C0000803D3ED167A83ED130AF5EEC07AF1EE9A
:10B2D00010FAD8BFDFED137A95ED070A27EE800A42
:10B2E000D1E7B0EEC88A05EB450587ED158A04EB7A
:10B2F000C50494ED070A28EE000A94F065FDD7ED29
:10B30000167A87ED130A94ED070AF0EEE77A27EE36
:10B31000800A94F059FD87ED140A5AE79A99993EEC
:10B320003333333F0000000038B500EBC11304464F
:10B3300093F865300A46CD0153B1FFF793FD0346FC
:10B3400030B104EB8103D3F85431003B18BF012323
:10B35000182101FB0242D2ED067AF0EEE77AF5EE13
:10B36000C07AF1EE10FA0ADC2C4494F8640020B99B
:10B3700092F92600003818BF0120184038BD01207E
:10B38000FBE7000010B500210446FFF76BFD18B184
:10B390002046FFF7C9FF50B101212046FFF762FDAB
:10B3A00030B12046FFF7C0FF003818BF012010BDA4
:10B3B0000846FCE710B50246FFF754FD20B102EB4A
:10B3C000C11292ED140A10BDBFEE000AFBE70000A7
:10B3D00010B50246FFF746FD20B102EBC11292ED17
:10B3E000130A10BDBFEE000AFBE7000010B50246CD
:10B3F000FFF738FD20B102EBC11292ED150A10BD26
:10B400009FED010AFBE700BF0000000010B50246F7
:10B41000FFF728FD20B102EBC11292ED170A10BD13
:10B420009FED010AFBE700BF000000002DE9F04F8F
:10B430002DED028B8DB0044669F020FC9FED3C8A17
:10B44000DFED3C8A80468946274625464FF0000BB3
:10B4500004F5AA7A5FFA8BF631462046FFF702FD23
:10B46000002858D05AF82B30002B54D06A4620467A
:10B47000FFF728FD08B9CDED008A1D22002104A8A0
:10B4800096F070FDA3238DF80430952331468DF896
:10B49000053020466E238DF80630CDF80780CDF8B4
:10B4A0000B908DF80F60FFF793FF20468DED040A97
:10B4B000FFF79CFFDDED007A8DED050A67EE887AD7
:10B4C0002046FDEEE77A17EE903AADF81830FFF718
:10B4D0009DFF10EE103A2046CDF81A30BB69CDF82A
:10B4E0001E30FFF725FE31468DF822002046FFF77B
:10B4F0001BFFD5F8BC300993D5F8C0300A9394F8F7
:10B500004E318DF823008DF82C303DF07BFD292243
:10B5100001A93CF07FFD18378035BBF1000F04D046
:10B520000DB0BDEC028BBDE8F08F4FF0010B91E741
:10B530000000C84200000000F8B590F90030002B70
:10B5400004464DDD0021FFF71DFE01212046FFF7D7
:10B5500019FE94F90030002B0DDD94F9403053B101
:10B5600047F042F8012105462046FFF723FF1D4919
:10B57000284641F063F8667894F84E7131462046CB
:10B58000FFF7D2FE054668B901462046FFF7CCFE1C
:10B5900028B901212046FFF7C7FE28B1012584F80C
:10B5A0004E5101E084F84E61204669F04BFD94F85D
:10B5B0004E31BB4204D03DF025FD5A213DF0BAFA90
:10B5C000D4F8503101330BD03DF01CFDD4F85011AC
:10B5D0003DF03EFB20B12046BDE8F840FFF726BF16
:10B5E000F8BD00BFA4BA0B08014B1868704700BF34
:10B5F000BC7A00200020704770470000012070478F
:10B60000436AC3B1B0F850301BB9436D0B600120E1
:10B61000704707EE903AD0ED136AF8EEE77A002310
:10B6200086EEA77A81ED007AA0F85030002380EDF5
:10B63000157AC364EBE718467047000070B50446FE
:10B640003AF010F900222221054639F06FFF6062BE
:10B6500020B300231A461946062011F08FFB01463D
:10B66000204669F04BFB002222212846666A39F009
:10B670007DFF0146304611F043FD94F82020E36938
:10B68000182101FB0233002283F82420E36994F897
:10B69000202003EBC213012083F8640070BD00007A
:10B6A00010B5034B0360044669F0FEFA204610BD56
:10B6B00068BC0B0810B50446FFF7F2FF204607F000
:10B6C000E9FE204610BD000073B590F845500446D1
:10B6D0003DB3012380F846300DF10601002390F8B8
:10B6E00028008DF806308DF8073007F085FB18B973
:10B6F0000025284602B070BD94F829000DF107011D
:10B7000007F07AFB0028F3D09DF806509DF807302B
:10B7100043EA051394F84450DBB2EB1A5D425D41F5
:10B72000E7E790F83830FBB990F82830413B192B07
:10B73000DFD890F82930413B192BDAD800F12A06DE
:10B7400017493046F5F7A4FE10B984F84850D0E701
:10B7500014493046F5F79CFE18B9012384F84830A7
:10B76000C7E784F84750C4E790F8482042B9012B56
:10B77000BFD12946283097F02FFF84ED100AB8E793
:10B78000012AB6D1072BB4D12946283097F024FFDF
:10B79000DFED057A20EE270A84ED0F0AA9E700BF46
:10B7A00058BC0B085CBC0B08E4388E3E242970B5ED
:10B7B00004460D4640D016DC0A291ED00D291CD0A7
:10B7C00094F837300D2B9FBF5A1C1B1984F8372073
:10B7D00083F8285094F8450090B994F844104D40EF
:10B7E00084F844500DE02A2907D02C29E8D190F89C
:10B7F000443083F02C0380F8443094F846600EB156
:10B80000002070BD94F84730002BF9D094F8373001
:10B810002344204683F82860FFF756FF94F8383019
:10B8200084F83760013384F83830A5F12A035D428B
:10B830005D4184F84550E4E700204FF0807384F8C0
:10B84000380084F837006364DBE700002DE9F0413D
:10B850002DED028B436A0446884623B90020BDECD7
:10B86000028BBDE8F08169F001FA0546606A9FED40
:10B87000248A03685B699847002687B23BB2002B95
:10B8800026DD606A03689B699847431CE6D041B295
:10B890002046FFF78BFF50B194F84830E565012B47
:10B8A00008D1D4ED0F7A013638EE278AB6B2013FBF
:10B8B000BFB2E3E7D4ED137A94ED107AB4F85030C8
:10B8C00077EE877A0133C4ED137AA4F85030EEE7AF
:10B8D00056B9A36DC8F80030E06D281AB0F5FA6FBC
:10B8E0002CBF00200120BAE707EE906AF8EEE77A55
:10B8F00088EE277A88ED007A84ED167AECE700BFAF
:10B900000000000010B50349044632F003FE204653
:10B9100010BD00BF88BC0B08F0B52DED048B91B0B5
:10B9200004466D46284607F0A1FA94F8B433002B7C
:10B9300072D004F578730FCB85E80F0094F8F033DC
:10B94000D4EDEA8A94EDEB8A94EDEC9A002B63D067
:10B9500094F8C833002B5FD02D22002104A8D4F81E
:10B96000B873D4F8BC63D4F8C053D4F8C44396F089
:10B97000F9FAA3238DF8103095238DF81130442364
:10B980008DF8123069F07AF99FED250A9FED257A3E
:10B99000CDF8171068EE807ACDF8130067EE877A3D
:10B9A000FDEEE77A17EE903A68EE007A29EE000A8B
:10B9B00067EE877AADF81B30FDEEE77A20EE070AD6
:10B9C00017EE903AADF81D3014F0E2FDDDED017A8E
:10B9D0009FED157ACDF82D70BCEEC00AF8EEE77A2F
:10B9E00010EE103A67EE877AADF81F3017EE903AF6
:10B9F000CDF82130029BCDF82530039BCDF82930BE
:10BA0000CDF83160CDF83550CDF839403DF0FAFA37
:10BA10002D2204A93CF0FEFA11B0BDEC048BF0BD60
:10BA2000E02E65420000C8420AD7233C30B52DED18
:10BA3000028B89B004461C220D4601A8002196F015
:10BA400091FAA3238DF8043095238DF80530462311
:10BA50008DF8063069F012F9D5ED007A95ED020AFD
:10BA6000CDF80B10FDEEE77ACDF8070017EE903A0F
:10BA7000D5ED017AADF80F30FDEEE77AD4F8F0316C
:10BA8000ADF8113017EE903AADF81330D4F8F43128
:10BA9000ADF8153014F07CFDBCEEC00AD4F8F80106
:10BAA0009FED168A10EE103AADF8173014F0B0FD85
:10BAB000ADF81900204600F089FD20EE080A204666
:10BAC000BCEEC00A10EE103AADF81B3000F084FD59
:10BAD00020EE080ABCEEC00A10EE103AADF81D3098
:10BAE00094F804338DF81F303DF08CFA1C2201A924
:10BAF0003CF090FA09B0BDEC028B30BD0000C842AA
:10BB000030B587B014460D4618220021684696F0DD
:10BB100029FAA3238DF8003095238DF801304723AF
:10BB20008DF8023069F0AAF8A3680393E3680493E0
:10BB30006368CDF807100593CDF803008DF80B501E
:10BB40003DF060FA182269463CF064FA07B030BD57
:10BB500010B58EB0044602A807F088F902A9204665
:10BB600001F0C0FC002845D001F0C6FE694601F096
:10BB700047FB1F22002106A896F0F4F9A3238DF8B5
:10BB8000183095238DF8193048238DF81A3069F054
:10BB900075F8DDED037A9FED1B7A049BCDF8233019
:10BBA000F8EEE77A059BCDF8273067EE877ACDF877
:10BBB0001B0017EE903ADDED007ACDF82B30F1EE58
:10BBC000677A17EE903ACDF81F10204601A9CDF8FC
:10BBD0002F3000F045FE78B1DDED017AF1EE677AA5
:10BBE00017EE903ACDF833303DF00CFA1F2206A93B
:10BBF0003CF010FA0EB010BD3DF004FADFED027A11
:10BC0000EEE700BF0AD7233C5241C07F2DE9F04345
:10BC10002DED048B0D469DB002F18801064602F120
:10BC20007C001446994617F03FF8B0EE409AF0EECB
:10BC3000608AB0EE418A8DED000ACDED010A8DEDEE
:10BC4000021A69F01BF8DFED657A96ED247AD5EDDE
:10BC5000066ACDF833000023CDE91933CDF86B30F7
:10BC6000A32329EE279A8DF8303095238DF83130B3
:10BC7000492327EE277A8DF8323019EE103ACDF8A5
:10BC80003B3017EE103A95ED057ACDF83F3037EEA0
:10BC9000267A68EEA78A17EE103A96ED257ACDF847
:10BCA000433027EE277A18EE903AD5ED086ACDF8A2
:10BCB000473017EE103A95ED077ACDF84B3037EE56
:10BCC000267A28EE278A17EE103A96ED267ACDF8D6
:10BCD0004F3067EE277A18EE103A95ED0A7ACDF8D4
:10BCE000533017EE903AD5ED097ACDF8573077EE0C
:10BCF000877A9FED3B7ACDF8371017EE903ACDF862
:10BD00005B30D9F87C33CDF85F30336AD3EDD47A29
:10BD100077EE877A9FED337A67EEC77A074617EE9C
:10BD2000903A05F144008846CDF863303FF0AEFD0F
:10BD30000346DFED2D0A93ED000AB7EE001A9E20B0
:10BD400014F092FC10EE103ACDF867306B6BCDF822
:10BD50006B303DF057F90CA93F223CF05BF92349C9
:10BD600004F1E80016F072FF78B3A3238DF80C30CD
:10BD700095238DF80D304A238DF80E30D4F8E83035
:10BD8000CDF81730D4F8EC30CDF81B30D4F8F030C3
:10BD9000CDF81F30D4F80031CDF82330D4F8043179
:10BDA000CDF82730D4F80831CDF80F70CDF81380D6
:10BDB000CDF82B303DF026F9232203A93CF02AF9D7
:10BDC0001DB0BDEC048BBDE8F083084904F580701C
:10BDD00016F03CFF0028C8D1F2E700BFE02E654214
:10BDE0000AE81C410000C84200000000A0C40C0882
:10BDF0007047000010B5044607F04CFB204610BD0C
:10BE00000023036043608360C36003614361836117
:10BE1000C3610362704700002DE9F041076A07F52E
:10BE20004676044600F16C050FCE0FC50FCE0FC548
:10BE300033682B6007F5437393E8070004F190081B
:10BE400088E8070094ED2E7AD4ED2D7A77EE877A84
:10BE50009FED367AF0EEE77AF4EEC77AF1EE10FA5B
:10BE60008EB004F16C0718D404F14802394604A8D6
:10BE700004AD14F0D7FE0FCD3E460FC60FCD0FC652
:10BE80002B683360414604F1240014F04DFE84ED2C
:10BE9000240AC4ED250A84ED261A04F10C0304F1EA
:10BEA0000802211D384615F077F89FED216AD4ED80
:10BEB000037A94ED017ADFED1F6A206A67EE867AD5
:10BEC00027EE067A67EEA67A27EE267AFDEEE77A67
:10BED000BDEEC77A17EE903A84ED047A94ED027ABB
:10BEE000002BB8BF03F50C4327EE067AB8BFA0338A
:10BEF00027EE267AA36104F1B003039304F1AC03A7
:10BF0000BDEEC77A029304F1A803019304F1A403E0
:10BF1000009384ED057A04F1A00304F19C023946F4
:10BF200001F0A8FD0EB0BDE8F08100BF00000034B4
:10BF3000E02E65420000C84210B504468AB0006A8F
:10BF400001F028FD04A904F124008DED040ACDEDD3
:10BF5000050A8DED061A14F0E7FD0AB010BD0000C9
:10BF600030B58BB0014604466D46684614F0CAFEF3
:10BF70000FCD0FC40FCD0FC42B6823600BB030BDA5
:10BF8000F8B50446244B036000F1240501620277F2
:10BF900004F148072846FFF733FF3846FFF730FF24
:10BFA00004F16C00FFF72CFF217F00231829C4F84F
:10BFB0009030C4F89430C4F8983026D0192926D08F
:10BFC00039BBC4F8B430D4ED2D7A84ED2E0A30EEAE
:10BFD000270A14F0B3FA9FED111ADFED110A284673
:10BFE00060EE200AB0EE410A14F076FF0FCD3E4617
:10BFF0000FC60FCD0FC62B6833603846FFF7B0FF72
:10C000002046FFF709FF2046F8BD064BD9E7064B4F
:10C01000D7E7064868F0F8FD6CBD0B08000000008B
:10C0200035FA8E3C0000B4420000874348BD0B083F
:10C030000023036043608360C360036143618361E5
:10C04000C36103627047000090F8B032B02202FB77
:10C05000030390F8562393F8913012B1012B28BFB7
:10C0600001231846704700002DE9F04304468BB0C9
:10C070000D4619F007FE002384F80C3204F5047015
:10C080004FF07E5767F022FD4FF47A73A4F85A32CE
:10C0900084F86052C4F84072C4F84472C4F848721C
:10C0A00004F51970002506F0E1FE04F52979032353
:10C0B000C4F8783204F53276C4F88C52C4F8905241
:10C0C000C4F89452C4F89852C4F89C52C4F8A052D0
:10C0D0004846FFF7ADFF3046FFF7AAFFC4F80C5300
:10C0E000C4F81053C4F8145304F54670FFF7A0FFCA
:10C0F000C4F83C53C4F84053C4F84453C4F84853FC
:10C10000C4F84C53C4F85053C4F85453C4F85853AB
:10C11000C4F85C53C4F86053C4F86453C4F868535B
:10C12000C4F88453C4F88853C4F88C53C4F8A0539B
:10C13000C4F89C53C4F89853C4F8A853C4F8AC533B
:10C14000C4F8B053C4F8C453C4F8C053C4F8BC53C3
:10C15000C4F89473C4F8B87304F5737006F086FEDF
:10C1600004F5787006F082FE04F58063C4F8F45399
:10C17000C4F8F85304F582601D605D609D6006F0B0
:10C1800075FE04F2244304F25C481D605D609D600E
:10C19000734BC4F8343404F50B73C4F8383404F525
:10C1A0000C73C4F83C3404F50D73C4F8403404F542
:10C1B0000E73C4F8443404F23D23C4F8483404F543
:10C1C0000F73C4F84C3404F58A6340461D605D600B
:10C1D0009D60FFF72DFF04F59060FFF729FF04F540
:10C1E000966304F234421D605D609D6004F2BC43BE
:10C1F00004F5B4601D605D609D6004F599631D6089
:10C200005D609D6004F2D4431D605D609D6004F23A
:10C21000E4431D605D609D6004F2F4431D605D6059
:10C220009D6004F5A363C2F8D470C2F8D8701D6095
:10C230005D609D6004F224531D605D609D6004F5A7
:10C24000A8631F605D6004F264531D605D609D60C3
:10C2500004F5AE631D605D609D6004F5B1631D6013
:10C260005D609D604FF07C53C2F8603106F0FEFDCA
:10C2700004F5B66304F5BC601D605D6004F5B7634A
:10C280001D605D6004F5B8631D605D60C8F808500E
:10C29000C8F80450C8F81450C8F80C50C8F81C501E
:10C2A000C8F81850C8F82070C8F81070C8F80070A6
:10C2B000FFF7BEFE04F2046304F234601D605D60AB
:10C2C0009D6004F5C2631D605D609D6004F21C63A7
:10C2D0001D605D609D6004F5C5631D605D609D60CF
:10C2E00006F0C4FD1F4B20491C60204632F012F9B5
:10C2F00094F86032C4F8205343F0010384F86032AC
:10C30000C4F81C53C4F82C53C4F82453C4F8345351
:10C31000C4F83053C4F83873C4F82873C4F81873D9
:10C3200004F5237207CA04F5267383E8070048461C
:10C3300094EDA81AD4EDA70A94EDA60A14F0CCFD4A
:10C340003546494668466E4614F0DCFC0FCE0FC5F4
:10C350000FCE0FC533682B6020460BB0BDE8F083CD
:10C360008CBF0B08C07A00207CBE0B0810B590F97A
:10C370002A32012B88B0044602D1274804F070FC11
:10C38000022B09D1032380F82A3204A901230D309E
:10C390008DF8103032F0FEFE94F82A3284F888329C
:10C3A00004F2344001F0E8FA94F92932642B30D1D8
:10C3B000652304A904F229208DF8103032F018FF0B
:10C3C00004A9204631F0B4FB18B304238DF81830CB
:10C3D0000023CDE9013303930F230593694604A895
:10C3E00031F05EFD059B28B108AA02EB830200999B
:10C3F00042F8581C0133112B0593EFD95DF0D4FCA2
:10C400009DED031ADDED020A9DED010A65215DF047
:10C4100089FC08B010BD00BF74BD0B0870B500F5F5
:10C42000237600F526758CB004463146284616F072
:10C43000F1FBE0B996E8070085E8070004F52971EB
:10C4400094EDA81AD4EDA70A94EDA60A0191084626
:10C4500014F042FD02AD019902A814F053FC0FCD77
:10C4600004F532740FC40FCD0FC42B6823600CB0D9
:10C4700070BD000013B54FF49F7200F504710446BF
:10C4800001A810F08DFD04F2344001F06FFC20464D
:10C4900019F01CFE01A810F0A5FD02B010BD0000AF
:10C4A000F8B50B68C0F8FC314B68C0F800328B68F7
:10C4B000C0F8043201F10C0607460C4600F546753B
:10C4C0000FCE0FC50FCE0FC533682B6004F13002BD
:10C4D00007CA07F5437383E8070004F13C0207CA63
:10C4E00007F54F7383E8070004F1480207CA07F510
:10C4F000527383E80700543494E8070007F5557336
:10C5000083E80700384601F0A7FB3846BDE8F8404D
:10C5100001F08ABB13B5044600F23440019003F0E9
:10C5200009F804F2D4510198009102F059FB0099E6
:10C53000204602B0BDE81040FFF7B2BF4A78064B74
:10C54000C2F340121A754A78C2F380125A750A78FB
:10C55000C2F300129A7570474D7B002013B540F26C
:10C56000C322044600F5047101A810F019FD002152
:10C5700004F2344001F04AFE94F8583223B12046C8
:10C580001AF068FB84F8580201A810F02BFD02B0E5
:10C5900010BD000038B590F8043305460C462BB1A9
:10C5A000032B0BD095F86032DB070CD405F2346313
:10C5B0000FCB84E80F0095F8440603E019F0FEFD68
:10C5C0000028EFD038BD0020FCE7000000F2344026
:10C5D00090ED350A7047000000F2344090ED360AC5
:10C5E0007047000010B490F804230C462AB1032AC7
:10C5F0000AD000205DF8044B704700F5B16007C811
:10C6000084E807000120F5E75DF8044B19F094BDBC
:10C6100038B590F804330D468BB900F2344001F080
:10C6200017FC044610B90024204638BD01F064FB15
:10C63000D5ED007A27EE800A85ED000AF4E790ED4B
:10C64000DE7A81ED007A90F87443002CEBD0D0EDC7
:10C65000DC7A67EE877AC1ED007AE5E790F804337B
:10C66000032B01D119F0E0BC0020704710B490F802
:10C670000443032C03D15DF8044B19F0E1BC002006
:10C680005DF8044B7047000090F80423032A01D1A1
:10C6900019F048BE00F2344002F01EB830B590F8F0
:10C6A000043385B004460D468BB1032B18D004F536
:10C6B000237016F0E9FA284601A98DED010ACDEDA7
:10C6C000020A8DED031A16F0D3F9012006E000F2FC
:10C6D000344001F067FB0028E9D1002005B030BDEF
:10C6E00090F85832002BF8D019F004FEDFE7000074
:10C6F0007FB590F8042332B1032A4FF0000309D02C
:10C70000039304930CE000F2344007B05DF804EBAF
:10C7100001F0FEBB03A903930493059319F07AFC7F
:10C720009DED030ADDED040A07B05DF804FB00008F
:10C7300007B590F8043333B100F57D7003B05DF8B0
:10C7400004EB15F029BB00F2344001F0E1FB684630
:10C750008DED000ACDED010A15F01EFB03B05DF86A
:10C7600004FB000037B5044640F27F520D4600F549
:10C77000047101A810F014FC2046294619F048FD68
:10C7800094F80433032B08BF044601A818BF002403
:10C7900010F028FC204603B030BD000090F80403E0
:10C7A000003818BF0120704708B590F80423032A09
:10C7B00005D0BDE8084000F2344001F093BB19F009
:10C7C00029FC012008BD000010B590F804230C4698
:10C7D0001AB1032A07D0002010BDBDE8104000F2B6
:10C7E000344001F047BB19F03BFC012084ED000A06
:10C7F000F2E7000030B590F8043385B005460C46EA
:10C8000023B1032B09D0002005B030BD00F2344025
:10C8100005B0BDE8304002F013BA002302A902932C
:10C82000039319F0DFFB0028EDD001A9284619F089
:10C83000E5FB0028E7D0029B2360039B6360019B1C
:10C84000A360E1E790F804231AB1032A05D0002081
:10C85000704700F2344002F027BA19F0C3BB000061
:10C8600090F804231AB1032A05D00020704700F283
:10C87000344002F00BBA19F0C1BB000090F92A3223
:10C880003BB990F8603213F0010F14BF0320002071
:10C890007047032070470000F7B50446FFF7EEFF2E
:10C8A0000546002862D0032839D194F858326BB37A
:10C8B00094F86032D8072BD501A9204619F058FD0D
:10C8C000BDF80430002B18BF002594F80C6206F068
:10C8D000FD06012E4AD10023032D019307D101A9A2
:10C8E000204619F051FD204619F034FD064604F2A9
:10C8F000344002F057FA08B994F801039DF8043067
:10C90000D90703D55A0701D59F0632D400252DE05B
:10C91000204619F0E5FA002808BF0025D5E70025D4
:10C92000D3E713F0020F2EE094F93C3223B99DF8BF
:10C930000430DB092FD0E9E7002EF8D00DF002F922
:10C94000FFF782FB022807D99DF805309806DDD550
:10C950009DF80430D906D9D5FB6A93F89C30002B9A
:10C96000E5D118E0DA0601D41B0718D5284603B034
:10C97000F0BD0028FAD094F80123B4F94836002A13
:10C98000CFD013F0010FF1D1154B1F68FB6A93F85C
:10C990009C30002BC8D19DF804309C07E2D409F0EC
:10C9A00097FE09F093FD0028B0D10DF0CBF8FFF70A
:10C9B0004BFB0228AAD90DF0C5F890F8B032B0228E
:10C9C00002FB030090ED2B7AF0EE007AB4EEE77AEA
:10C9D000F1EE10FA9AD59DF80530DB09C6D195E73E
:10C9E000A82500202DE9F04790F8583292B004466F
:10C9F000002B00F08680204619F08AFE2046FFF7C3
:10CA00004BFF032840F0AC8004F5467800274146F0
:10CA1000204600970197029719F042FC694620468C
:10CA200019F034FC009BC4F8FC31019BC4F80032BF
:10CA3000029BC4F80432204601F00EF9204601F0B2
:10CA4000F3F813F02FF90546204619F0BDFA002837
:10CA5000A8BFC6B203AA4FF0FF312046BCBF95F86D
:10CA6000029395F803630397A8BFB146049705970F
:10CA700019F004FB03A816F007F94FF00C0A0AFBA3
:10CA8000095084EDCF0AC4EDD00A84EDD11A04F523
:10CA90004F7100F50D7016F007F904F555770AFB94
:10CAA000065584EDC30AC4EDC40A84EDC51A3A469E
:10CAB00020464FF0FF3105F5BC7519F0F3FA95E803
:10CAC000070006AE86E807003946304616F052F9F0
:10CAD00004F52972414609A814F0A4F8314609A8C2
:10CAE00014F022F809A9204684EDD20AC4EDD30A35
:10CAF00084EDD41A19F048FC09A92046FFF71EFD61
:10CB00002EE0D0F85C321BB968F0B0F8C4F85C02D3
:10CB1000154B1B68D86A03685B68984788B168F052
:10CB2000A5F8D4F85C32C01AB4F85A32984204D945
:10CB300020461AF08FF884F8580294F858327BB1E6
:10CB400059E768F093F8D4F85C32C01A41F28733A1
:10CB50009842E4D83CF056FA3CF096F80028DED132
:10CB600012B0BDE8F08700BFA825002090F804337C
:10CB700023B1032B4FF0000007D0704790F92A2211
:10CB8000032A04D10A70012070470870FBE7184699
:10CB90007047000073B50D460DF107010446FFF71D
:10CBA000E5FF064628B19DF807302BB1032B09D0CD
:10CBB0000026304602B070BD04F234630FCB85E826
:10CBC0000F00F6E72946204619F0F8FA94F8586263
:10CBD000EFE700007FB50E460DF103010446FFF7B5
:10CBE000C5FF054618B90025284604B070BD9DF85C
:10CBF000033083B1032B16D004F5237016F044F8EC
:10CC000001A930468DED010ACDED020A8DED031A22
:10CC100015F02EFFE8E7314604F2344001F0C2F887
:10CC20000028E9D1DFE794F85832002BDBD03146F9
:10CC3000204619F05FFBDFE737B50D460DF1070120
:10CC40000446FFF793FF28B19DF8073023B1032B6B
:10CC50000FD0002003B030BD04F2D4531B682B600A
:10CC600004F5BB6304F2DC541B686B602368AB60A3
:10CC7000F0E72046294619F009FB94F85802E9E745
:10CC800010B50446FFF7FAFD18B1032807D00020BD
:10CC900010BD04F23440BDE8104001F0ADB894F886
:10CCA0005832002BF3D0204619F01AF90028EED0A4
:10CCB00094F80C3203F0FD03012BE9D194F804033E
:10CCC000C31E58425841E3E710B50446FFF7D6FDAE
:10CCD00080B1032810D194F8580250B167F0C6FF14
:10CCE000D4F85C32C01A44F62063984294BF002006
:10CCF000012010BD0120FCE70020FAE708B502463C
:10CD0000FFF7BCFD032804D1104619F03DFB0120BC
:10CD100008BD0020FCE7000030B585B00446019155
:10CD2000FEF762FC0199054610B9002005B030BD40
:10CD30000191FEF7FDF901990028F6D02846FEF78B
:10CD4000F3FA0028F1D094F80133002BEED00B4A0F
:10CD50001268D26A92F89C506DB103A92046FFF781
:10CD6000CDFF30B19DF80E309A07DFD5C3F38000B8
:10CD7000DCE72846DAE71846D8E700BFA8250020F8
:10CD800010B490F8044324B1032C08D05DF8044B90
:10CD900070475DF8044B00F2344000F0F9BF5DF8D5
:10CDA000044B19F0AFB9000090F80433F5EE007AA7
:10CDB000002BB7EE000A08BFB0EE670A704700000C
:10CDC00010B50446FFF75AFD032804D12046BDE8FC
:10CDD000104019F0C9B9002010BD00002DE9F04144
:10CDE00090F804338CB00027032B06460C461546FA
:10CDF00000970197029719D119F0E6F86A46804624
:10CE00004FF0FF31304619F04DF9B8F1FF3FA76000
:10CE1000676027600DD112F045FF2B4690F8031391
:10CE2000224611F0EFFF0CB0BDE8F0814FF0FF3863
:10CE3000EBE712F037FF2B4622465FFA88F111F03C
:10CE4000E1FF95ED000A684615F05AFF03A9204658
:10CE50008DED051A8DED030ACDED040A15F08AFF5C
:10CE600006F5297206F5467103A813F0DBFE21468C
:10CE700003A813F059FE84ED021A84ED000AC4EDF4
:10CE8000010A95ED007ADFED037AA7EE271A84ED0B
:10CE9000021AC8E70AE81C411FB5DFED0B7A20EE45
:10CEA000270A0C461946094BCDE90042BDEEC00ADF
:10CEB00018688DED020A064B9DF81820C06A10F024
:10CEC000EDF904B010BD00BFE02E6542A82500209A
:10CED00088BD0B082DE9F0472DED028B92B000259F
:10CEE00004460F464FF07E5A00F5467106A890465C
:10CEF000CDF818A009950895079515F0BFF909F028
:10CF0000E7FB09F0E3FA81462046FFF7B7FC032868
:10CF100003D094F80433032B4FD19FED558ADFEDF6
:10CF2000558A00262378F2B2934247D90AAA71B2F1
:10CF30002046CDF828A00D950C950B9519F0BAF95F
:10CF40000AA906A815F006FEB4EEC80AF1EE10FA1A
:10CF50000DDD494ACDF800803B4648492046FFF7A1
:10CF60009BFF002012B0BDEC028BBDE8F0870AA940
:10CF700006A803950495059515F0D6FD03A90EA8FE
:10CF80008DED0E0ACDED0F0A8DED101ACDED111AB3
:10CF900015F0FAFAB9F1000F0DD09DED050AB0EECB
:10CFA000C00AB4EEE80AF1EE10FA04DD344ACDF816
:10CFB00000803B46D1E70136B4E7002394F8606275
:10CFC00016F0010001D0012BCCD104F5BC610AA8F8
:10CFD000CDF828A00D950C950B9515F04FF90AA9E1
:10CFE00006A815F0B7FDDFED227AB4EEE70AF1EE00
:10CFF00010FA05DD204ACDF800803B462149ADE717
:10D000002046FFF73BFC03282DD1204619F096F966
:10D0100094F86032DB0728D438BB0AA906A8039528
:10D020000495059515F080FD03A90EA88DED0E0A57
:10D03000CDED0F0A8DED101ACDED111A15F0A4FAF1
:10D04000B9F1000F11D09DED050ADFED0A7AB0EEBF
:10D05000C00AB4EEE70AF1EE10FA06DD084ACDF890
:10D0600000803B46CAE70020D2E701207AE700BFF4
:10D07000C2B8323EC2B8B23EB4BD0B08BFBD0B0849
:10D080007FBF0B08C4BD0B082DE9F74314460546C6
:10D0900088460193FFF7F4FD019A074638B9244802
:10D0A000244B00682146C06A10F0F8F8019A0192FA
:10D0B00021462846FFF70EFF064630B32846FFF705
:10D0C000DDFB95F80433019A83420DD009F000FB93
:10D0D00009F0FCF9019A38B1174B15480068214650
:10D0E000C06A10F0DBF810E02846FFF7C7FB18B164
:10D0F00003280FD0114BF0E713464146224605F2B4
:10D10000344000F08DFE00B107B90026304603B070
:10D11000BDE8F08395F85892B9F1000F01D1084BA2
:10D12000DBE7134641462246284618F0E5FEEAE7CB
:10D13000A8250020C8BD0B08D4BD0B0804BE0B08F1
:10D14000F3BD0B0890F80433032B01D119F032B969
:10D150000020704790F80433032B01D119F06AB90D
:10D160000020704790F80433032B01D119F0AAB9BD
:10D170000020704708B50246FFF780FB10B1032876
:10D1800006D008BDBDE8084002F2344000F0FEBD04
:10D19000BDE80840104619F003B900000B4610B472
:10D1A00011462BB1032B09D000205DF8044B7047CA
:10D1B0005DF8044B00F2344000F0FEBD5DF8044B16
:10D1C00019F008B813B50446FFF758FB0A460146A4
:10D1D00020460192FFF7E2FF70B9084B019A1B68E5
:10D1E000DB6A93F89C0038B194F80413204602B02F
:10D1F000BDE81040FFF7D2BF02B010BDA825002047
:10D2000070B590F87432DB0786B004460D460CD436
:10D2100002F0AAFE437C242202FB0300D0ED0B7A2D
:10D22000F1EE677AC5ED007A3BE002A805F01EFE3C
:10D2300001A92046FFF714FBE8B90CF083FC94F930
:10D240003C32022B0646E3D1FEF7FEFE0228DFD970
:10D2500096F8B0029FED147AB02303FB0066D4F871
:10D260006832D6F8A0209B1A07EE903AF8EEE77ADB
:10D2700067EE877AD6E702A92046FFF7A3FF0028CA
:10D28000DBD0D4F86822039BDFED076A9DED017ABD
:10D290009B1A07EE903AF8EEE77AA7EEE67A85ED6C
:10D2A000007A06B070BD00BF0AD7233CF0B50C462B
:10D2B00087B000F50471064640F6473201A80FF02A
:10D2C0006FFEA36853B9E36843B9636833B90027B5
:10D2D00001A80FF087FE384607B0F0BD204605F0E4
:10D2E000B9FE0028F3D094E80F0002AD85E80F00E6
:10D2F0000021284605F084FE07460028E7D096F86E
:10D300007432DB0704D43BF07DFE19213BF012FCA4
:10D3100095E80F0006F5197C8CE80F0096F874323A
:10D3200043F0010386F87432304600F0C5FC45F046
:10D330005BF9432145F006FD45F056F9422145F0E1
:10D3400001FD054BA2681B68DB6A1A61E2685A613D
:10D3500062689A61BCE700BFA825002038B5144B6D
:10D360001B68DD6A2B6804465B6828469847F0B165
:10D370002B690BB96A69D2B1C4F86C326B69C4F815
:10D380007032A969002204F5197005F075FD94F852
:10D39000743223F0030343F0030384F8743245F03E
:10D3A00023F9BDE83840034A06213EF0F3BE38BDFC
:10D3B000A825002018BE0B0810B588B004460593B8
:10D3C000FFF75CFA0328059B4FF000000AD1069096
:10D3D000079006A802900B9801900A9800902046AA
:10D3E00018F092FF08B010BD38B50446FEF7FCF8FF
:10D3F0000546D0B194F80433032B03D095F84E4181
:10D40000204638BD204618F0A3FEFF280446F5D07C
:10D4100001462846FDF788FF0028EFD02146284620
:10D42000FDF786FE0028E9D0EAE70446E8E70000B9
:10D4300008B590F80433032B05D012F033FC90F9B3
:10D440000203C0B208BD18F0BFFD431CF9D1F4E7D8
:10D4500008B590F8043383B1032B03D1BDE808402D
:10D4600018F0AABD39F09EFF40F6AE424FF480118D
:10D4700039F04EFF4FF0FF3008BD1846FCE70000C2
:10D4800090F80433032B01D119F096BA70470000CD
:10D4900090F80433032B01D118F0A4BC70470000AE
:10D4A00018F004BD10B504461BF08CFC2046FEF7B6
:10D4B00033FA2046BDE81040FEF74ABB07B51C30E2
:10D4C00001A98DED010A31F039FE03B05DF804FBCE
:10D4D00090F804330BB1032B01D119F0EBBA002003
:10D4E0007047000030B500F5737304460D460FCB4E
:10D4F00085E80F0094F8DC0330BD00007FB50546D9
:10D5000068460E4605F0B2FC95F87432DB0703D48A
:10D510000024204604B070BD69462846FFF7E2FFAC
:10D5200004460028F4D0694605F5197005F076FE2A
:10D5300086ED000AC6ED010AEBE70000D0F878336B
:10D540000B6090F874037047D0F880330B6090F84C
:10D550007D03704730B500F5657304460D460FCB6B
:10D5600085E80F0094F8A40330BD000030B500F545
:10D57000826304460D460FCB85E80F0094F8200423
:10D5800030BD000010B500F2244203460C4607CA25
:10D5900084E8070093F8300410BD00002DE9F04343
:10D5A0002DED028B8BB005460E461746FFF71CFF8C
:10D5B000014680462846FFF7AFFB0446B0B3FEF7AE
:10D5C00013F84146FDF7F6FE86ED000A95F928327C
:10D5D000002B28DD0CF0B6FAFEF736FD012822D923
:10D5E0000CF0B0FA90F8B03295EDDC7A96ED000AC6
:10D5F000B02202FB030095F92832D0ED2B0A07EE8A
:10D60000903AF8EEE77A20EE070A37EEA01A40F2D9
:10D61000833070EEE70A13F027F895EDDC7AC0EE60
:10D62000077AC6ED007A01233B7003E095F80033DA
:10D6300033B9387020460BB0BDEC028BBDE8F083E7
:10D6400095F804334FF00009CDF80490CDF8089018
:10D65000CDF80C9043B1032B10D0CDF81090CDF83D
:10D660001490CDF818907CB902233B7032464146A5
:10D6700005F2344001F05AFB0446DBE701A92846D5
:10D6800018F05AFD0446E8E795F80433002BEBD078
:10D6900004A92846FFF776FF04460028E4D001A934
:10D6A00004A815F017FB07A8CDED080A8DED091A9F
:10D6B0008DED070A15F022FF04A8B0EE408A15F0A0
:10D6C0001DFF95F92832002B25DD07EE903AF8EE84
:10D6D000E77A40F2C93070EE670A37EE801AF5EE4D
:10D6E000C00AF1EE10FA48BFDFED0F0AF4EE410A6E
:10D6F000F1EE10FAB0EE480AC8BFB0EE601A12F0B0
:10D70000B3FFB0EE408A95EDDC7AC8EE077A0323CA
:10D71000C6ED007A88E7B5EEC08AF1EE10FA48BF90
:10D720009FED018AEFE700BF0000000010B504463E
:10D73000FFF77EFE84F805032046FFF779FE84F8A4
:10D7400006032046FFF774FE84F807032046FFF720
:10D750007FFE04F5587184F808032046FEF742FF67
:10D7600084F86C0300F0C8FA04F55F7284EDDC0AFB
:10D7700004F55E712046FFF711FF04F5607184F82F
:10D7800074032046FEF744FF04F5617184F87D03BD
:10D790002046FEF763FF04F5657184F89003204688
:10D7A000FEF77CFF04F56A7184F8A4032046FFF7B6
:10D7B00043FA04F56E7184F8B4032046FFF70AFAC1
:10D7C00004F5737184F8C8032046FEF7E3FE04F500
:10D7D000787184F8DC032046FFF7DCF984F8F00365
:10D7E0002046FEF785FF2046C4EDFE0A84EDFD0AC3
:10D7F000FEF79EFF04F20C4284EDFF0A04F58061FF
:10D800002046FFF7EBFA04F582612046FFF7DAFCC9
:10D8100004F2244184F820042046FEF7C5FF84F872
:10D82000300410BD37B50D46044600F003F91DB9AC
:10D8300012F038FA11F016FA40F2791204F5047178
:10D8400001A80FF0ADFB94F861322BB92046FFF729
:10D8500085FD012384F86132224B1D68A86A0368A4
:10D860009B6998472046FEF7D9FD2046FEF752FEF9
:10D87000204600F053FA2046FFF7B4F8286B30B189
:10D880000368D4EDD00ADB6894EDCF0A9847D4F84A
:10D89000080208B1FEF7C0FA204600F06DF82046F5
:10D8A000FEF7FAFF94F8883284F8040383420ED01E
:10D8B00084F8880298B10C4D0C4B032808BF1D4614
:10D8C00044F092FE0A4A2B4606213EF063FC2046B5
:10D8D000FFF72CFF01A80FF085FB03B030BD054D0D
:10D8E000EEE700BFA8250020457C0B08BFBD0B0854
:10D8F00030BE0B08C4BD0B08014B1868704700BF51
:10D90000C07A00204FF0FF307047000001207047C0
:10D9100070470000002070470020704770470000EB
:10D9200070470000002070470020704700207047BB
:10D93000002070470020704700207047002070478B
:10D94000012070470368D3F89430184700207047CF
:10D95000002070470020704700207047002070476B
:10D96000002070470020704700207047002070475B
:10D9700000207047704700007047000008B512F0A3
:10D9800091F990F8030308BD08B512F08BF990F8EF
:10D99000020308BD30B585B090F80653044612F076
:10D9A00081F90C2303FB050004F54F7100F50D70A0
:10D9B00005B0BDE8304015F077B9000030B52DED69
:10D9C000028B9FED1A1ADFED1A0A91ED000A87B05B
:10D9D00005462D200C468DED011ACDED000A12F002
:10D9E00043FE9DED011ADDED000AF0EE408A2E2087
:10D9F00094ED010A12F038FE9DED011ADDED000AEA
:10DA0000B0EE408A2F2094ED020A12F02DFE03A9F9
:10DA100005F52370CDED038A8DED048A8DED050AA1
:10DA200031F0CAFC07B0BDEC028B30BDC2B8323E4B
:10DA3000C2B832BE10B5044667F018F9D4F8EC321B
:10DA4000C21AB2F57A7F12D3094A1268D26A92F8E2
:10DA50009C2002B15BB9C4F8EC0294F8294212F0A0
:10DA600021F980F8FD4208F033FE80F8254010BD12
:10DA7000A82500202DE9F0432DED028B91ED007AD1
:10DA8000D1ED037A87B08DED047AB0EEC77AB5EEAA
:10DA9000C07AF1EE10FADDE91087DDF84C90CDED9B
:10DAA000057A0C4615461E4606DCF0EEE77AF5EEE2
:10DAB000C07AF1EE10FA02DD04A814F0EBF96A2046
:10DAC000B7EE001AFFEE000A9DED050A12F0CCFD3C
:10DAD0006B2089ED000AB7EE001AFFEE000A9DEDFB
:10DAE000040A12F0C1FD04A888ED000A14F02EF912
:10DAF000B7EE008A002852D00023C9F8003088ED24
:10DB0000008AD4ED067A67EEA77AF4EEC87AF1EED1
:10DB100010FA4ADB0023336085ED008ADFED3F0A0F
:10DB200096ED000A7B20B7EE001A12F09DFD86EDFF
:10DB3000000A95ED000A7C20B7EE001AFFEE000AFD
:10DB400012F092FD85ED000AD4ED067A129BDFED0E
:10DB5000346AF1EE677AC3ED007A96ED007AF0EE62
:10DB6000C77AF4EEE67AF1EE10FA2BD503AB02AAEF
:10DB700001A9204613F010FA9DED018AB0EE480A83
:10DB800091F0B6FD85ED000AB0EE480A91F006FF6F
:10DB900087ED000A07B0BDEC028BBDE8F08304A856
:10DBA00014F0C0F80028A7D1ABE738EE670A12F0EE
:10DBB000B5FC86ED000A94ED087AC7EE007AC5ED53
:10DBC000007AABE794ED076AC6EE077AC7ED007AF4
:10DBD00096ED007AB0EEC77AB4EEE67AF1EE10FA7E
:10DBE000C4D495ED007ADFED0F6AB0EEC76AB4EEEB
:10DBF000666AF1EE10FAB9DCB4EE477AF1EE10FA8B
:10DC0000B4D6B0EEE77AB4EE667AF1EE10FAADDC97
:10DC1000F4EE677AF1EE10FABCD7A7E70000000037
:10DC200000000034FFFF7F7F1FB500F515730393DD
:10DC300000F51473029300F51373019300F512734A
:10DC4000009300F5107200F5117300F54671FFF7AF
:10DC500011FF05B05DF804FB9FED156A90ED7F7A2A
:10DC6000DFED146AD0ED817A27EE067A67EE867AC8
:10DC700027EE267A67EEA67ABDEEC77AFDEEE77A42
:10DC800080ED7C7A90ED807A27EE067A17EE903A56
:10DC900027EE267A002BB8BF03F50C43BDEEC77AFA
:10DCA000B8BFA03380ED7D7AC0F8F831704700BF6F
:10DCB000E02E65420000C8421FB50E4B1B680446AB
:10DCC000B3B1684605F0D2F869462046FFF74EFC2E
:10DCD00020B16A4600212046FDF712FF94F8743205
:10DCE000DB0705D504F5197201212046FDF708FF71
:10DCF00004B010BD607D002008B502F035F9BDE824
:10DD0000084001F093BD000010B580F8F012044601
:10DD100066F0ACFFC4F8F40210BD000010B590F836
:10DD2000F032044653B166F0A1FFD4F8F432C01AC1
:10DD3000B0F57A7F84BF002384F8F03294F8F8328B
:10DD400053B166F093FFD4F8FC32C01AB0F57A7F75
:10DD500084BF002384F8F83210BD000000F5AA70DB
:10DD60000B4607C883E80700012070470023C0F86E
:10DD70009C30C0F89830C0F89430C0F8A830C0F893
:10DD8000A430C0F8A030C0F8AC3070477047000035
:10DD9000024B0B604FF07C53136070470000484209
:10DDA0007047000008B50B4600F12801184614F032
:10DDB00065FA012008BD000010B500F5B6700C46EC
:10DDC0000FC884E80F00204605F040F830B1FFF797
:10DDD00093FD00F519700FC884E80F00204605F088
:10DDE00035F880F00100C0B210BD000010B5044647
:10DDF00005F050FB204610BD10B5D0F86431044644
:10DE00005BB166F033FFD4F86431C01A41F2883355
:10DE1000984294BF0020012010BD0120FCE70000C3
:10DE200013B5009303680192D3F890309847DDE969
:10DE30000021044628B90448044B0068C06A0FF06A
:10DE40002DFA204602B010BDA8250020C8BD0B0841
:10DE500013B504460191FDF7C7FB2368019A1B6DBA
:10DE6000014608B190F84E11204602B0BDE81040BE
:10DE70001847000030B585B0002301930293039347
:10DE800003680D46DB6D01A99847044620B1039B4A
:10DE90002B60204605B030BD02F066F8417C01F0F1
:10DEA000B3FD04460028F4D002F05EF801F046FC11
:10DEB000B1EE400A85ED000AEBE7000010B5FDF772
:10DEC00093FB044658B190F84E11FDF731F930B18B
:10DED00094F84E112046BDE81040FDF725BA002009
:10DEE00010BD000038B50D460BF02CFE0446FEF7C1
:10DEF000ABF8022881BF94F8B002B02303FB0040C6
:10DF0000C43089BF07C8002085E80700012038BD5C
:10DF10002DE9F0432DED028B8FB003680025DB6CFB
:10DF20000395049505950695029502A90446984720
:10DF3000064638B1FFF7E0FEDDED027A27EE800AF3
:10DF40008DED020A0BF0FEFDFEF77EF80746002E6F
:10DF500051D0DDED027AD4ED656A94ED667A2368DE
:10DF60000B9527EE877A67EEA67A8DED097ACDEDCF
:10DF70000A7A0C950D959B6C0BA9204609AD984724
:10DF80000BA9284613F02AFE012F8DED030ACDEDD3
:10DF9000040A40F2B4800BF0D5FD90F8B032DFED0A
:10DFA0005C7AB02503FB0553034493ED008A28EE09
:10DFB000278AB0EE480A91F09BFBF0EE408AB0EE63
:10DFC000480A91F0EBFCCDED0B8A8DED0C0A0BF0BD
:10DFD000B9FD90F8B03205FB030090ED2B0A0BA8B9
:10DFE00013F01CFE09AD8DED050ACDED060A05A85E
:10DFF00096BB03C885E00128CDD89DED020AB5EE99
:10E00000C00AF1EE10FA7FDD07AED4F89821D4F8FB
:10E01000943107923046089313F03CFE23680B9529
:10E020000C950D959B6C0BA920469847DDED077A62
:10E030009DED0B7A77EE877A9DED0C7ACDED077A20
:10E04000DDED087A77EE877A09ABCDED087A96E8B0
:10E05000030083E8030049E0236993ED000AB7EE6B
:10E06000008A38EE408A13F0D9FD04F5BE798DEDB3
:10E07000090A4846B0EE480ACDED0A0A13F0CEFD73
:10E080000BA92846CDED0C0A8DED0B0A13F0A6FD69
:10E0900004F5C67603AFC4ED600A314684ED5F0A2D
:10E0A000384613F0ABFD04F5C2788DED090A404601
:10E0B000B0EE480ACDED0A0A13F0B0FD0BA92846D0
:10E0C0008DED0B0ACDED0C0A13F088FD97E80300E7
:10E0D00084ED610AC4ED620A86E8030049464046C1
:10E0E00013F07CFD8DED090ACDED0A0A9DED090ABC
:10E0F000DDED0A0A0FB0BDEC028BBDE8F083DDE96F
:10E10000030185E80300F1E709950A95EEE700BFF2
:10E1100035FA8E3C10B590F84213044607F002FF22
:10E120007C23C0B203FB0044D4F8A00010BD000063
:10E13000044B026F1B68DB6A5A60426F9A60826F01
:10E14000DA607047A8250020F0B58FB0044611F0C2
:10E15000A9FD002302930393049390F8021301ABEB
:10E1600002AA054610F0F4FD04F19407D8B39DED22
:10E17000010AB5EEC00AF1EE10FA34DD02A814F07F
:10E18000CFFD04F1B00684ED2C0AC4ED2D0A84ED18
:10E190002E1A3946304614F0D3FD04F17C01304686
:10E1A00014F082FD04F1880105A88DED050ACDED7E
:10E1B000060A8DED071A14F077FD08A88DED080A00
:10E1C0009DED010ACDED090A8DED0A1A14F098FDB6
:10E1D0000BA904F128008DED0B0ACDED0C0A8DED95
:10E1E0000D1A12F085FF95F802030C2303FB005073
:10E1F000394600F50D7014F057FD84ED2C0AC4ED7E
:10E200002D0A84ED2E1A0FB0F0BD00002DE9F04765
:10E21000824B00251F682DED028BC0F89C50C0F882
:10E220009850C0F89450C0F88450C0F88050C5672A
:10E23000C0F89050C0F88C50C0F88850C0F8B85062
:10E24000C0F8B450C0F8B0500446F86A03688AB009
:10E250005B680E46984704F12809002854D066F000
:10E2600005FD42F20F7398424ED8FB6A9FED6C8A0F
:10E2700093ED010A84ED1C0AD3ED020AC4ED1D0AD8
:10E2800093ED031A484684ED1E1A12F025FE44F061
:10E29000ABF9D4ED1E7A67EE887A054617EE900A40
:10E2A000F2F732F9D4ED1D7A67EE887ACDE90401F0
:10E2B00017EE900AF2F728F9D4ED1C7A67EE887A07
:10E2C000CDE9020117EE900AF2F71EF9554ACDE9A1
:10E2D0000001062128463DF05DFF94ED1E8AB0EE58
:10E2E000480A91F005FA84ED660AB0EE480A91F00A
:10E2F00055FB84ED650A66F0B9FCC4F868010AB004
:10E30000BDEC028BBDE8F087A6B194ED1C0AB4EE1B
:10E31000400AF1EE10FA0DD6D4ED1D0AF4EE600AB3
:10E32000F1EE10FA06D694ED1E1AB4EE411AF1EE93
:10E3300010FA52D711F0B6FC90F803334FF00C0AE4
:10E340000AFB030303F5BC73074693E8070007AE17
:10E3500086E807004FF01508B2EE028AF2EE068A50
:10E36000304615F0CBF8B4EEC80AF1EE10FA38D505
:10E3700008F1FF3818F0FF083CD1304615F0BEF820
:10E38000F1EE047AB4EEE70AF1EE10FA43DD9DED0A
:10E39000090ADDED087A9DED078A20EE000AA7EE56
:10E3A000A70A91F011FDF0EE400AB0EE480A91F094
:10E3B000C1FBDDED090A84ED1D0A9DED080AF1EEB1
